:020000022000DC
:106000000000042041AD02001D8E0200C1A202006A
:106010001D8E02001D8E02001D8E02000000000079
:106020000000000000000000000000001D8E0200C3
:106030001D8E0200000000001D8E02001D8E020059
:10604000EDAB02001D8E020091B1020095AD020081
:10605000A5AD02001D8E0200E9A002001D8E020007
:106060001D8E020071B1020081B1020011AD02006B
:106070001D8E02001D8E02001D8E02001D8E02006C
:10608000B9B1020021AD02001D8E02001D8E02007A
:106090001D8E02001D8E0200CDAE02001D8E02007C
:1060A0001D8E02001D8E02001D8E02001D8E02003C
:1060B0001D8E02001D8E0200000000000000000086
:1060C0001D8E02001D8E02001D8E0200B5AD020065
:1060D00031AD02001D8E02001D8E0200B1B1020022
:1060E000A1B10200EDAC02001D8E02003DAE020027
:0860F000000000001D8E0200FB
:10700000DC760B004CB10B00DC760B00A8B90B0052
:10701000DC760B00B0B90B00DC760B00B8B90B00C6
:10702000DC760B0060BB0B00DC760B0068BB0B0052
:10703000DC760B000CC00B00DC760B0024C00B00D0
:10704000DC760B00C8C00B00DC760B008CCC0B0090
:10705000DC760B0094CC0B00DC760B009CCC0B0098
:10706000DC760B0074CD0B00DC760B007CCD0B00C6
:10707000DC760B00E4CE0B00DC760B00ECCE0B00D4
:10708000DC760B00F4CE0B00DC760B000CCF0B0093
:10709000DC760B0014CF0B00DC760B00D8CF0B0096
:1070A000DC760B0070D00B00DC760B0088D00B0078
:1070B000DC760B0090D00B00DC760B0098D00B0038
:1070C000DC760B00A0D00B00DC760B005CD10B0053
:1070D000DC760B0064D10B00DC760B00FCD10B00DE
:1070E000DC760B0004D20B00DC760B0090D20B0098
:1070F000DC760B0098D20B00DC760B00A0D20B00E4
:10710000DC760B00A8D20B00DC760B00B0D20B00B3
:10711000DC760B004CD30B00DC760B0054D30B0059
:10712000DC760B005CD30B00DC760B0064D30B0029
:10713000DC760B00E8D30B00DC760B00F0D30B0001
:10714000DC760B00F8D30B00DC760B00B8D50B0017
:10715000DC760B00C0D50B00DC760B00B4D80B003E
:10716000DC760B00DCD80B00DC760B0054DB0B006C
:10717000DC760B005CDB0B00DC760B00A8DB0B0085
:10718000DC760B00ECDB0B00DC760B0048DC0B0044
:10719000DC760B0050DC0B00DC760B00ECDD0B002A
:1071A000DC760B0004DE0B00DC760B00BCDE0B0093
:1071B000DC760B001CE00B00DC760B0024E00B00FF
:1071C000DC760B0050E10B00DC760B0058E10B0085
:1071D000DC760B00E4E10B00DC760B00F8E20B0040
:1071E000DC760B0000E30B00DC760B00F4E30B0015
:1071F000DC760B000CE40B00DC760B0020F00B00BF
:10720000DC760B0038F00B00DC760B0040F00B0056
:10721000DC760B0038F30B00DC760B00F4F40B008B
:10722000DC760B0084F90B00DC760B008CF90B008C
:10723000DC760B0094F90B00DC760B0050FC0B00A5
:10724000DC760B0058FC0B00DC760B0060FC0B00BE
:10725000DC760B0030FE0B00DC760B0038FE0B00FA
:10726000DC760B0040FE0B00DC760B0048FE0B00CA
:10727000DC760B008C000C00DC760B00A4000C000C
:10728000DC760B00AC000C00DC760B00B4000C00CC
:10729000DC760B00BC000C00DC760B0058010C0007
:1072A000DC760B0080030C00DC760B0098030C00EE
:1072B000DC760B00A0030C00DC760B0094050C00C0
:1072C000DC760B009C050C00DC760B00A4050C00A2
:1072D000DC760B00AC050C00DC760B00BC050C006A
:1072E000DC760B00C4050C00DC760B00CC050C0032
:1072F000DC760B00D4050C00DC760B005C060C0081
:10730000DC760B006C080C00DC760B0074080C00BB
:10731000DC760B007C080C00DC760B0084080C008B
:10732000DC760B00F0080C00DC760B001C0B0C006C
:10733000DC760B00240B0C00DC760B008C0C0C00B4
:10734000DC760B00540F0C00DC760B005C0F0C009D
:10735000DC760B00640F0C00DC760B006C0F0C006D
:10736000DC760B00740F0C00DC760B0050160C0062
:10737000DC760B0058160C00DC760B00C8190C00EC
:10738000DC760B00D0190C00DC760B007C1F0C00A7
:10739000DC760B00841F0C00DC760B008C1F0C00CD
:1073A000DC760B00941F0C00DC760B009C1F0C009D
:1073B000DC760B00DC220C00DC760B0034240C00A5
:1073C000DC760B003C240C00DC760B00A4240C00C3
:1073D000DC760B0050250C00DC760B006C270C00D3
:1073E000DC760B00782A0C00DC760B00882A0C0077
:1073F000DC760B00F82C0C00DC760B00002D0C006A
:10740000DC760B009C2D0C00DC760B00A42D0C0010
:10741000DC760B00AC2D0C00DC760B00B42D0C00E0
:10742000DC760B00482F0C00DC760B00502F0C0094
:10743000DC760B0044B10B003CB10B00DC760B009A
:1074400080B90B0078B90B00DC760B0090B90B000B
:1074500088B90B00DC760B00D4CC0B00CCCC0B0035
:10746000DC760B00E4CC0B00DCCC0B00DC760B00F4
:10747000F4CC0B00ECCC0B00DC760B0004CF0B0043
:10748000FCCE0B00DC760B0078D00B0068D00B0034
:10749000DC760B0054D10B004CD10B00DC760B00DA
:1074A000D0D50B00C8D50B00DC760B00C4D80B0080
:1074B000BCD80B00DC760B00D4D80B00CCD80B006A
:1074C000DC760B0004DA0B00FCD90B00DC760B0039
:1074D0000E000000ACDC0B00DC760B0014E00B00AF
:1074E0000CE00B00DC760B00F4E10B00ECE10B0090
:1074F000DC760B0004E20B00FCE10B00DC760B00F9
:1075000014E20B000CE20B00DC760B0018E30B001E
:1075100010E30B00DC760B0018F00B0010F00B00F2
:10752000DC760B0030F00B0028F00B00DC760B0053
:1075300050F00B0048F00B00DC760B0060F00B0005
:1075400058F00B00DC760B00ECF40B00E4F40B00BD
:10755000DC760B0004F50B00FCF40B00DC760B0072
:107560001CF60B0014F60B00DC760B0080F70B000A
:1075700078F70B00DC760B0090F70B0088F70B0018
:10758000DC760B00A0F70B0098F70B00DC760B0005
:10759000B0F70B00A8F70B00DC760B0010FA0B001D
:1075A00008FA0B00DC760B00D4FB0B00CCFB0B00C5
:1075B000DC760B00E4FB0B00DCFB0B00DC760B0045
:1075C000F4FB0B00ECFB0B00DC760B0004FC0B0067
:1075D000FCFB0B00DC760B00F0FC0B00E8FC0B0066
:1075E000DC760B00E0FD0B00D8FD0B00DC760B0019
:1075F000F0FD0B00E8FD0B00DC760B0008FE0B0035
:1076000000FE0B00DC760B0018FE0B0010FE0B00DA
:10761000DC760B0028FE0B0020FE0B00DC760B0056
:1076200058FE0B0050FE0B00DC760B0068FE0B00D2
:1076300060FE0B00DC760B0078FE0B0070FE0B008A
:10764000DC760B0084000C007C000C00DC760B0068
:107650009C000C0094000C00DC760B006C030C000A
:1076600064030C00DC760B0090030C0088030C0014
:10767000DC760B00B0030C00A8030C00DC760B00DA
:10768000C0030C00B8030C00DC760B0080110C006A
:1076900078110C00DC760B0090110C0088110C00A6
:1076A000DC760B00BC170C00B4170C00DC760B006A
:1076B000CC170C00C4170C00DC760B00E8190C008A
:1076C000E0190C00DC760B009C1A0C00941A0C00DC
:1076D000DC760B00AC1A0C00A41A0C00DC760B0054
:1076E000281B0C00201B0C00DC760B00381B0C0048
:1076F000301B0C00DC760B00441F0C003C1F0C0000
:10770000DC760B00541F0C004C1F0C00DC760B00C9
:10771000641F0C005C1F0C00DC760B00741F0C0057
:107720006C1F0C00DC760B0020210C0018210C00D3
:10773000DC760B0030210C0028210C00DC760B00DD
:10774000B4220C00AC220C00DC760B00C4220C002E
:10775000BC220C00DC760B00D4220C00CC220C00E6
:10776000DC760B004C240C0044240C00DC760B006F
:107770005C240C0054240C00DC760B006C240C0000
:1077800064240C00DC760B007C240C0074240C00B8
:10779000DC760B008C240C0084240C00DC760B00BF
:1077A0009C240C0094240C00DC760B0060250C005B
:1077B00058250C00DC760B0070250C0068250C00A9
:1077C000DC760B0080250C0078250C00DC760B00A5
:1077D00090250C0088250C00DC760B007C270C0023
:1077E00074270C00DC760B0034280C002C280C00CD
:1077F000DC760B0044280C003C280C00DC760B00E7
:1078000054280C004C280C00DC760B0064280C007B
:107810005C280C00DC760B0074280C006C280C0033
:10782000DC760B0084280C007C280C00DC760B0036
:1078300094280C008C280C00DC760B00A4280C008B
:107840009C280C00DC760B00B4280C00AC280C0043
:10785000DC760B00C4280C00BC280C00DC760B0086
:10786000D4280C00CC280C00DC760B00E4280C009B
:10787000DC280C00DC760B00F4280C00EC280C0053
:10788000DC760B0004290C00FC280C00DC760B00D5
:10789000982A0C00902A0C00DC760B00402F0C007C
:1078A000382F0C00DC760B00A0300C0098300C0058
:1078B000DC760B00B0300C00A8300C00DC760B003E
:1078C00064310C005C310C00DC760B0074310C0070
:1078D0006C310C00DC760B0038320C0030320C00BE
:1078E000DC760B0048320C0040320C00DC760B00DA
:1078F00058320C0050320C00DC760B009C320C002D
:1079000094320C00DC760B00AC320C00A4320C007C
:10791000DC760B00BC320C00B4320C00DC760B00C1
:10792000CC320C00C4320C00DC760B00DC320C00D4
:10793000D4320C00DC760B000C340C0004340C0048
:10794000DC760B001C340C0014340C0040F8044BA3
:1079500040F8045B40F8046B40F8047B40F8048B6B
:1079600040F8049B40F804AB40F804BB40F804CB5B
:1079700040F804DB6846704781F0004102E000BF38
:1079800083F0004330B54FEA41044FEA430594EADF
:10799000050F08BF90EA020F1FBF54EA000C55EA1A
:1079A000020C7FEA645C7FEA655C00F0E2804FEAEB
:1079B0005454D4EB5555B8BF6D420CDD2C4480EACD
:1079C000020281EA030382EA000083EA010180EAFD
:1079D000020281EA0303362D88BF30BD11F0004F4B
:1079E0004FEA01314FF4801C4CEA113102D0404281
:1079F00061EB410113F0004F4FEA03334CEA1333BC
:107A000002D0524263EB430394EA050F00F0A780D3
:107A1000A4F10104D5F1200E0DDB02FA0EFC22FACE
:107A200005F2801841F1000103FA0EF2801843FAC2
:107A300005F359410EE0A5F120050EF1200E012AB3
:107A400003FA0EFC28BF4CF0020C43FA05F3C018F1
:107A500051EBE37101F0004507D54FF0000EDCF16A
:107A6000000C7EEB00006EEB0101B1F5801F1BD313
:107A7000B1F5001F0CD349085FEA30004FEA3C0C17
:107A800004F101044FEA445212F5800F80F09A800D
:107A9000BCF1004F08BF5FEA500C50F1000041EB11
:107AA000045141EA050130BD5FEA4C0C404141EB15
:107AB0000101013C28BFB1F5801FE9D291F0000F10
:107AC00004BF01460020B1FA81F308BF2033A3F1BF
:107AD0000B03B3F120020CDA0C3208DD02F1140CB6
:107AE000C2F10C0201FA0CF021FA02F10CE002F1F1
:107AF0001402D8BFC2F1200C01FA02F120FA0CFCEA
:107B0000DCBF41EA0C019040E41AA2BF01EB045132
:107B1000294330BD6FEA04041F3C1CDA0C340EDC30
:107B200004F11404C4F1200220FA04F001FA02F373
:107B300040EA030021FA04F345EA030130BDC4F131
:107B40000C04C4F1200220FA02F001FA04F340EA26
:107B50000300294630BD21FA04F0294630BD94F0D7
:107B6000000F83F4801306BF81F480110134013DBE
:107B70004EE77FEA645C18BF7FEA655C29D094EA2F
:107B8000050F08BF90EA020F05D054EA000C04BFAD
:107B90001946104630BD91EA030F1EBF0021002098
:107BA00030BD5FEA545C05D14000494128BF41F037
:107BB000004130BD14F580043CBF01F5801130BD9B
:107BC00001F0004545F0FE4141F470014FF0000026
:107BD00030BD7FEA645C1ABF194610467FEA655CD7
:107BE0001CBF0B46024650EA013406BF52EA033579
:107BF00091EA030F41F4002130BD00BF90F0000F67
:107C000004BF0021704730B54FF4806404F13204A2
:107C10004FF000054FF0000150E700BF90F0000F5B
:107C200004BF0021704730B54FF4806404F1320482
:107C300010F0004548BF40424FF000013EE700BF52
:107C400042004FEAE2014FEA31014FEA02701FBFE2
:107C500012F07F4393F07F4F81F06051704732F014
:107C60007F4208BF704793F07F4F04BF41F400216B
:107C7000704730B54FF4607401F0004521F00041C9
:107C80001CE700BF50EA010208BF704730B54FF053
:107C900000050AE050EA010208BF704730B511F054
:107CA000004502D5404261EB41014FF4806404F18C
:107CB00032045FEA915C3FF4D8AE4FF003025FEA12
:107CC000DC0C18BF03325FEADC0C18BF033202EB96
:107CD000DC02C2F1200300FA03FC20FA02F001FAF0
:107CE00003FE40EA0E0021FA02F11444BDE600BF93
:107CF0004FEA4102B2F1E04324BFB3F5001CDCF1CE
:107D0000FE5C0DD901F0004C4FEAC0024CEA507005
:107D1000B2F1004F40EB830008BF20F00100704734
:107D200011F0804F21D113F13872BCBF01F0004037
:107D3000704741F480114FEA5252C2F11802C2F169
:107D4000200C10FA0CF320FA02F018BF40F00100EA
:107D50004FEAC1234FEAD32303FA0CFC40EA0C009C
:107D600023FA02F34FEA4303CCE77FEA625307D1D9
:107D700050EA01331EBF4FF0FE4040F44000704710
:107D800001F0004040F0FE4040F40000704700BFAA
:107D900080F0004002E000BF81F0004142001FBFC0
:107DA0005FEA410392EA030F7FEA226C7FEA236CC9
:107DB0006AD04FEA1262D2EB1363C1BFD2184140BE
:107DC00048404140B8BF5B42192B88BF704710F054
:107DD000004F40F4000020F07F4018BF404211F0F7
:107DE000004F41F4000121F07F4118BF494292EA5F
:107DF000030F3FD0A2F1010241FA03FC10EB0C008B
:107E0000C3F1200301FA03F100F0004302D5494217
:107E100060EB4000B0F5000F13D3B0F1807F06D3C4
:107E200040084FEA310102F10102FE2A51D2B1F1BC
:107E3000004F40EBC25008BF20F0010040EA0300B1
:107E40007047490040EB0000013A28BFB0F5000F31
:107E5000EDD2B0FA80FCACF1080CB2EB0C0200FAE7
:107E60000CF0AABF00EBC25052421843BCBFD04036
:107E70001843704792F0000F81F4000106BF80F4B0
:107E800000000132013BB5E74FEA41037FEA226C73
:107E900018BF7FEA236C21D092EA030F04D092F03E
:107EA000000F08BF0846704790EA010F1CBF002072
:107EB000704712F07F4F04D1400028BF40F00040CF
:107EC000704712F100723CBF00F50000704700F0EF
:107ED000004343F0FE4040F4000070477FEA226216
:107EE00016BF08467FEA23630146420206BF5FEAE7
:107EF000412390EA010F40F4800070474FF00003E7
:107F000004E000BF10F0004348BF40425FEA000CAD
:107F100008BF704743F0964301464FF000001CE055
:107F200050EA010208BF70474FF000030AE000BFAB
:107F300050EA010208BF704711F0004302D54042E9
:107F400061EB41015FEA010C02BF8446014600205B
:107F500043F0B64308BFA3F18053A3F50003BCFA76
:107F60008CF2083AA3EBC25310DB01FA02FC634423
:107F700000FA02FCC2F12002BCF1004F20FA02F22A
:107F800043EB020008BF20F00100704702F120021D
:107F900001FA02FCC2F1200250EA4C0021FA02F27E
:107FA00043EB020008BF20EADC7070477BB972B96E
:107FB0000029BEBF00204FF0004106E008BF0028A6
:107FC0001CBF6FF000414FF0FF3000F081B9ADF100
:107FD000080C6DE904CE002909DB002B1ADB05F043
:107FE00001FEDDF804E0DDE9022304B07047404201
:107FF00061EB4101002B1BDB05F0F4FDDDF804E033
:10800000DDE9022304B0404261EB4101524263EBDF
:1080100043037047524263EB430305F0E3FDDDF891
:1080200004E0DDE9022304B0404261EB4101704706
:10803000524263EB430305F0D5FDDDF804E0DDE9D2
:10804000022304B0524263EB4303704753B94AB969
:10805000002908BF00281CBF4FF0FF314FF0FF3050
:1080600000F036B9ADF1080C6DE904CE05F0BAFDAB
:10807000DDF804E0DDE9022304B0704770B54FF08D
:10808000FF0C4CF4E06C1CEA11541DBF1CEA1355A4
:1080900094EA0C0F95EA0C0F00F0DEF82C4481EA0C
:1080A000030621EA4C5123EA4C5350EA013518BF2C
:1080B00052EA033541F4801143F4801338D0A0FB19
:1080C00002CE4FF00005E1FB02E506F00042E0FBC6
:1080D00003E54FF00006E1FB03569CF0000F18BFCC
:1080E0004EF0010EA4F1FF04B6F5007F64F5407474
:1080F00004D25FEA4E0E6D4146EB060642EAC62107
:1081000041EA55514FEAC52040EA5E504FEACE2E73
:10811000B4F1FD0C88BFBCF5E06F1ED8BEF1004F76
:1081200008BF5FEA500E50F1000041EB045170BDF2
:1081300006F0004646EA010140EA020081EA030136
:10814000B4EB5C04C2BFD4EB0C0541EA045170BD32
:1081500041F480114FF0000E013C00F3AB8014F1AC
:10816000360FDEBF002001F0004170BDC4F10004F5
:10817000203C35DA0C341BDC04F11404C4F1200576
:1081800000FA05F320FA04F001FA05F240EA0200D1
:1081900001F0004221F0004110EBD37021FA04F607
:1081A00042EB06015EEA430E08BF20EAD37070BDC1
:1081B000C4F10C04C4F1200500FA04F320FA05F020
:1081C00001FA04F240EA020001F0004110EBD37022
:1081D00041F100015EEA430E08BF20EAD37070BD92
:1081E000C4F1200500FA05F24EEA020E20FA04F36B
:1081F00001FA05F243EA020321FA04F001F000411A
:1082000021FA04F220EA020000EBD3705EEA430E8A
:1082100008BF20EAD37070BD94F0000F0FD101F0B9
:108220000046400041EB010111F4801F08BF013CF2
:10823000F7D041EA060195F0000F18BF704703F030
:108240000046520043EB030313F4801F08BF013DB7
:10825000F7D043EA0603704794EA0C0F0CEA135573
:1082600018BF95EA0C0F0CD050EA410618BF52EA2D
:108270004306D1D181EA030101F000414FF0000033
:1082800070BD50EA410606BF1046194652EA430641
:1082900019D094EA0C0F02D150EA013613D195EAB5
:1082A0000C0F05D152EA03361CBF104619460AD1FD
:1082B00081EA030101F0004141F0FE4141F4700107
:1082C0004FF0000070BD41F0FE4141F4780170BDF7
:1082D000704700BF4A0011D212F5001211D20DD51D
:1082E0006FF47873B3EB62520ED44FEAC12343F0BC
:1082F000004343EA505323FA02F070474FF0000066
:10830000704750EA013002D14FF0FF3070474FF014
:1083100000007047000000009FED197B70B51A4CFB
:1083200084ED007B41B30023DFF868E0101F1D4699
:108330009C4602E0013399420FD050F8042F960773
:10834000F8D116687645F5D1BCF1000F15D101338F
:10835000994215464FF0010CEFD1BCF1000F0BD044
:1083600095ED017ADFED097A67EE277A17EE900A2C
:1083700004F020FAC4E9000170BD05487AF0F2F972
:1083800000000000000000001012012000007A44EC
:1083900088A10B0074DB0B0090F8743043F000737D
:1083A00003F17E43033B102B05D8DFF83CC05CF89B
:1083B00023309A4213D310B59FED097BA0B00C4631
:1083C000043004A98DED047B019265F029FB019A2C
:1083D00003AB214604A865F047FB20B010BD7047F1
:1083E0000000000000000000DC360C00000000006F
:1083F00010B584B004469DF820E09DF828C0039392
:1084000008469DF81C1084F8371000216EF3070110
:108410006CF30F21BDF818C084F832C0CCF1080C01
:1084200084F836C09DF82CC09FED0F7B6CF317418C
:10843000E163002121609DF8241084F8331084ED5D
:10844000027B1146CDE9010272F006FB0198029A07
:108450000399A0852046E28504B0BDE810402DF0C8
:10846000E3BF00BFAFF30080000000000000000089
:1084700000B59FED0D7B89B00923016802904FF094
:108480000A0C039302A800238DED007BCDF810C0E9
:10849000CDF814D08DF8183046F092FC00980038D2
:1084A00018BF012009B000BD00000000000000005E
:1084B00010B5144686B017A3D3E90023FFF776FD65
:1084C00003A9019075F09EFC9DF80F309DF80E20D9
:1084D00001980F491B0443EA42539DF8102043EAD8
:1084E000C2239DF8112043EA42139DF8122043EA6B
:1084F0005203BDF80C2020F00100A2F2BC72A0FBD8
:10850000010143EA4263236006B010BDAFF300806F
:1085100000CA9A3B00CA9A3B00000000000000001D
:108520002DE9F04F87B0044600AF8A4690460025FB
:1085300041F086F807F10801204601223D7267F0FC
:10854000CFF997F90800397AA84234DA01F0E0034C
:10855000E02B30D0A02B36D001F0F003902B00F0B0
:10856000A881802B00F0AE81A1F1C0031F2B00F287
:108570009D81DFE813F097019B0199019501580057
:10858000580058008A008A008A002101CB00E900C7
:10859000F600050134014501530161016F018001BD
:1085A00087018E0113011A0141004100410096002C
:1085B0009600A300A300400040F0010318461C37BA
:1085C000BD46BDE8F08F01F01F02D31D03F0380354
:1085D0006D46ADEB030D6B463AB169462046C7E9DF
:1085E000003267F07DF9D7E900321846114649F0AC
:1085F00059FE0346AD46E1E72731C9B2204667F090
:1086000033FA0546014607F108007EF001FE25B168
:1086100039692A46204667F063F907F1080049F0F6
:108620008FFE0346CAE73C31C9B2204667F01CFA08
:1086300005468046014607F108007EF0E9FDF5B1E8
:108640003969206866687960B8F5807F454628BF3B
:108650004FF4807504F10C032A46B0470346E068E6
:108660007968002840F05581002B00F04E819D4232
:1086700000F24881B8EB050329449846E1D107F19F
:10868000080049F09FFA034698E73931C9B22046FD
:1086900067F0EAF95246014620467AF0D3F80346DD
:1086A0008CE72531C9B2204667F0DEF94346014622
:1086B000524620467AF088F803467FE72331C9B254
:1086C000204667F0D1F9B0F1005F834680F0238146
:1086D00049F006FB0346BBF1000F3FF46FAF0025E6
:1086E0004246514620467B60FFF71AFF42468146CC
:1086F00051462046FFF714FF013502464946786887
:1087000046F040FEAB457B68EAD157E79FED847B9E
:108710000822B918204687ED027B67F0E1F8D7E917
:10872000023210BA19BAFFF7E3FA07EE900AF4EE34
:10873000677AF1EE10FA50D6034623F0030343F0B4
:108740000203A3F1FF4339E70023012207F10801E7
:1087500020463B7267F0C4F83B7A5B0043F00103AC
:108760002CE70023022207F1080120463B8167F035
:10877000B7F83B895BBA9BB25B0043F001031DE78E
:108780000023042207F108012046BB6067F0A8F827
:10879000B86800BA49F09CFC03460FE7524608212E
:1087A00020467AF04FF8034608E75246102120464B
:1087B0007AF048F8034601E70023042207F1080194
:1087C0002046BB6067F08CF8BB681BBA07EE903A96
:1087D000F4EE677AF1EE10FAAFD7534BEEE69FED69
:1087E000507B0822B918204687ED027B67F078F8A5
:1087F000D7E9021009BA00BA49F08CFC0346DDE65D
:108800000023012207F1080120463B7267F068F857
:1088100097F908305B0043F00103CFE60023022202
:1088200007F1080120463B8167F05AF83B89DBBA23
:108830005B0043F00103C1E60023042207F10801B5
:108840002046BB6067F04CF8B86800BA49F09AFB64
:108850000346B3E69FED327B0822B918204687ED28
:10886000027B67F03DF8D7E9021009BA00BA49F077
:10887000F3FB0346A2E652460121204679F0E2FFCF
:1088800003469BE652460221204679F0DBFF034671
:1088900094E652460421204679F0D4FF03468DE643
:1088A0003E238BE60E2389E61E2387E61F4879F0D8
:1088B00059FF4346524601F00F01204679F084FFEC
:1088C00003467BE601F00F06304649F009FAB3464D
:1088D0000346002E3FF472AE4246514620467B606E
:1088E000FFF71EFE4246814651462046FFF718FE1E
:1088F000013502464946786846F044FDAB457B6841
:10890000EAD15BE60A4879F02DFF0A48194685F05E
:108910000EFA79F0CFFE0848722179F02BFF00BFE4
:10892000000000000000000002004000F0A30B0067
:10893000C48E0B005C6C0B00C8AA0B00D2B32DE9EF
:10894000F0436FF00E0885B00646174601F10F049C
:10895000A8EB010854F80F0C54F80B1C54F8072C22
:1089600054F8033CEC46ACE80F003146A4F10F008C
:1089700001F0AAFCA4F1100306F1EF0213F8011FA5
:1089800012F8010FA34281EA00011970F6D1EC46FA
:10899000BCE80F00103408EB040C6745C6F8F00083
:1089A000C6F8F410C6F8F820C6F8FC30D2D805B0E6
:1089B000BDE8F083704700BF2DE9F041044682B363
:1089C0006FF00E05164601F10F0700F1F0086D1A61
:1089D00008F1FF31A7F11003A7F10F0813F8012FD9
:1089E00011F801CFBB4282EA0C021A70F6D121467F
:1089F0004046103700F018F9EB199E42E8D8D8F835
:108A00000010D8F80420D8F80830D8F80C00C4F8C2
:108A1000FC00C4F8F010C4F8F420C4F8F830BDE845
:108A2000F08100F1F008EAE7002A44D070B54C1E4E
:108A300084B0064615194FF0100C01E00CF1010C42
:108A4000BCF1100F0BD00DEB0C0214F8013F1278A3
:108A5000AC4283EA02032370F0D104B070BDD6F8B3
:108A6000F000D6F8F410D6F8F820D6F8FC30EC4632
:108A7000ACE80F003146684600F0D6F80F2206F544
:108A8000807111F8013DFF2B0FD03244013382F881
:108A9000F03014F8013F9DF80020AC4283EA020355
:108AA0002370DAD04FF0010CCDE70023013A0B70B0
:108AB000531CE6D1EDE7704703460846194601F01E
:108AC00003BC00BF03460846194600F0ADB800BF1E
:108AD000182A2DE9F04F0546C0F800217ED0202A43
:108AE00076D0102A7ED1834640F20A43A5F804319D
:108AF000AC4600200B788CF800304B788CF80130B5
:108B00008B788CF80230CB788CF8033095F80531EF
:108B1000013098421A4601F104010CF1040CE9D32A
:108B200095F804110131B3EB810F55D20BEB8201A3
:108B3000501E11F802EC1BF8204011F803CC11F87C
:108B4000010C2B4FDFF8AC802DE017F80CA018F8C3
:108B5000099017F80EC017F800E0385D8AEA09049A
:108B6000A2EB03090BEB89031BF8299084EA0904A3
:108B70000C7093F8019004318CEA090C01F803CCD5
:108B800093F802908EEA090E01F802ECDB78584067
:108B900001F8010C95F8043101320133B2EB830F77
:108BA0001AD295F80531B2FBF3F903FB192ABAF191
:108BB000000FCAD0D5F80061202ED1D1BAF1040F30
:108BC000CED13C5D17F80CC017F80EE0385CC7E753
:108BD000834640F60E0389E7BDE8F08F834640F2F6
:108BE0000C6383E700239B46A0F804311A469DE7F7
:108BF000BC350C00B0340C0000B583B0CDE90030BA
:108C0000FFF766FF009B0198D3F800C059689A6887
:108C1000DB68C0F8FC30C0F8F0C0C0F8F410C0F851
:108C2000F82003B000BD00BF2DE9F04FD1F80031AE
:108C3000103B102B85B08946864600F2E980754AC4
:108C400022FA03F313F0010F14BF0D4600250EF1B5
:108C50000406344600270EEB070379191A7811F839
:108C6000010B424003F8012B9C42F7D10437102F2F
:108C700004F10404EFD10EF11008674FCDF8048021
:108C80004FF0010C0EF11402AB46CA4671460023A8
:108C900011F82300385C01F823000133042BF7D1CD
:108CA00001318E42F3D19EF805409EF809109EF8DE
:108CB00001309EF80D509EF802008EF801408EF8AB
:108CC00005109EF80A409EF806108EF809508EF89E
:108CD0000D309EF80E509EF803308EF802408EF84C
:108CE0000A009EF80F409EF80B008EF80E109EF8BA
:108CF00007108EF806508EF803408EF80F008EF89D
:108D00000B108EF807309AF8043163456AD0CDE92C
:108D100002CB7046047845788178C37884EA0509E7
:108D20004FEAD9184D404FEAD51C08EB4808594086
:108D30005C4008EBC8080CEB4C0C00230CEBCC0C93
:108D400068F307036CF30F234FEAD11C0CEB4C0CB8
:108D50000CEBCC0C89EA010B6CF317434FEA490981
:108D60004FF0000C6D0069F3070C490065F30F2C00
:108D700061F3174C0021E5096BF3070164006BF305
:108D80000F2105EB450564F31F6C6BF31741046875
:108D900005EBC5056BF31F6165F31F6383EA0C03E5
:108DA00061404B4040F8043B019B8342B2D1DDE976
:108DB00002CB34464FEA0C15231F0BEB0500197844
:108DC00010F8018B81EA080103F8011B9C42F6D1DF
:108DD0000434A24205F10405EED10CF1010C5FFA56
:108DE0008CFC53E75D464FEA0C1C331F05EB0C006F
:108DF000197810F8014B614003F8011B9E42F7D12E
:108E00000436B2420CF1040CEFD105B0BDE8F08F8E
:108E100000251CE701010100BC350C00FEE700BF86
:108E20002DE9F04F4FEAA3095C4FDFF8ACB1DFF852
:108E3000ACA103F0030486464B4659488BB007EBC0
:108E400084171C2B50F824000090A8BF1C237868BE
:108E50000197033323EAE37318410790B868184178
:108E60000890F86818410990B9F11F0F4FF0000001
:108E7000C8460690A8BF4FF01F080BE00DEB850514
:108E8000AC69002B40EA0400B8BF6442013A41F8E3
:108E9000044B75D05EF8043B13EA0B0F23F000453A
:108EA000ECD013EA0A0F0BD1019CB9F1000F54F872
:108EB0002540BABFC8F10005AC4044FA08F4E0E729
:108EC000384C23420DD1103D374C54F82540009DBD
:108ED00084FB0565A8F10304002C47DB45FA04F484
:108EE000CFE76C04B4F1006FBABF6C05042600260E
:108EF000B4F1005FBCBFA40002362C4DB4F1804F2A
:108F0000BCBF64000136AC423DDD294D294FCDE99F
:108F1000045705F1F95505F5CE2505F29B15039586
:108F2000254F264D0295254687FB05C5029F3D44EA
:108F3000274685FB07C7039D2F44254687FB05C5AC
:108F4000049F3D4485FB0474059D2C441C4D55F83D
:108F5000265084FB0575EC00009D84FB0575194CBB
:108F600054F82640A8EB0404002CB7DA66426FF0F0
:108F7000004444FA06F7AF4283DB05FA06F480E7C3
:108F80000BB0BDE8F08F104D104FDFF854C0CDE9A5
:108F900004570F4D0F4FCDE9025CC4E7284D0C007C
:108FA000284E0C00C0FFFF7F684C0C009979825A54
:108FB000F0CEC227B477F5FE63218510A4F633D333
:108FC000284C0C00484C0C008D496C23591858FF54
:108FD00028482EB0A9BDA029FCFFFF7FF0FFFF7F2E
:108FE0001BAA5759844602F001007BBB60B3DCF832
:108FF0008034DCF88001DCF88012DCF880235B42EE
:10900000CCF88034DCF880384042494252425B421E
:10901000CCF88001CCF88012DCF88005DCF88016F2
:10902000CCF88023CCF88038DCF88027DCF880305E
:109030004042494252425B42CCF88005CCF880164F
:10904000CCF88027CCF88030002070472DE9F0471D
:10905000C3F11F04002847D04FF00047DF40002035
:109060000CF18006013F0CF51069804656F8802C03
:1090700042FA04FEBEEBE27F87EAE27E18BF724648
:109080009A40454646F8802C82EAE275A5EBE275E7
:10909000DCF88020C2F1000E4EFA04F2B2EBEE7F53
:1090A00087EAEE7218BF96460EFA03F2CCF88020DB
:1090B000C64682EAE27EAEEBE27E0A6845EA0E052B
:1090C000284342FA04F5B5EBE27F87EAE27518BF60
:1090D0002A460CF5807C9A40E14541F8042B06F5C0
:1090E0008076C3D1BDE8F0874FF00046DE40013EF8
:1090F0000CF180050CF5106E074655F8802C42FAED
:1091000004F9B9EBE27F86EAE27918BF4A469A4051
:10911000B84645F8802C82EAE278A8EBE278DCF8E1
:10912000802042FA04FABAEBE27F86EAE27A18BFBC
:1091300052469A40B946CCF8802082EAE279A9EBFF
:10914000E2790A6848EA090840EA080042FA04F8A5
:10915000B8EBE27F86EAE27818BF42460CF5807CE5
:109160009A40E64541F8042B05F58075C5D1BDE868
:10917000F08700BF2DE9F041436903F5A04307469E
:10918000D3F8C46DD3F8C08DEEB1046A0025033462
:1091900014F8023C14F8031C14F8012C1B0203EB16
:1091A00001431A44294630461BF004FB2946304649
:1091B00001351BF0EDFAB5F5807F04F10304E7D12A
:1091C00097F825303BBBF9683868B8F80420431895
:1091D0009342D7E901342344B8F80640C8BF111AB6
:1091E000A34216DA904214DA002912DDB8F80C20F6
:1091F00002FB03F3D8F8082002EB8302BB6986B1B7
:109200000244013A194413F8010B02F8010F8B4292
:10921000F9D1BDE8F08197F8241030461BF0C2FA6E
:10922000D1E702EB400297F82500FC69012809D03C
:10923000194413F8010B34F8100022F8020B8B428A
:10924000F7D1E6E797F82450194413F8010B85424B
:109250001CBF34F8100010808B4202F10202F4D1DE
:10926000D7E700BF2DE9F04100F5A04882B098F89B
:10927000AE1D426B01238DF80730036B51BBD11A31
:109280004C1E40F2F942944224D833BB044640F2CB
:10929000FA4600F1540514E0636BB3421ADC236C08
:1092A0009847616B236C9DF8072001F5BD5114317F
:1092B000214428469847636B9DF807201344636355
:1092C000D2B1D4E915739F424FF001020DF10701AD
:1092D0002846E1DB02B0BDE8F08100F5BD52133253
:1092E0001344551813F8014F02F8014FAA42F9D15F
:1092F0000023C0E90C31C9E7012388F8AE3D02B074
:10930000BDE8F08170B500F5A042002382B043654E
:1093100082F8B43D82F8AE3D826D4FF0FF310B2AEA
:10932000D8BF5218C0E90831C8BF0C22036C0192A3
:1093300000F5DA71044654309847019A824227D1E9
:109340001849052204F5DA703CF04EFC30B116499C
:10935000052204F5DA703CF047FC00BB94F8BE31FE
:10936000B4F8BA11B4F8BC212160C3F3021301337D
:10937000C4E90121E260A3610146626C04F154007A
:109380009047A368B3F5A07F07DC012002B070BD51
:1093900006230020E36102B070BD0223F9E7082331
:1093A000F7E700BF68330B0070330B0041F2167C07
:1093B000614500F276812DE9F04F00F58D5A0AF1F2
:1093C000140A00F5ED5700F59B460368856A91B0D5
:1093D0000E372E3600F5DA7E5446A64500F0BD80E5
:1093E000725C04F8012D37F811106145F5D95B1B4B
:1093F00000F17408BAEB0407434400F0AE80C16A80
:1094000000F5A5521432039200293A460546474614
:109410004FF0000B00F5A046904640F39A80A86AF2
:10942000404500F32E811A1893420BD2013B04EB06
:10943000000C14F8012B03F8012FA445F9D1D5E94C
:109440000A0164462A682B69AA6202930593A8EB75
:109450000008039B96F8B40D0B9700280CBFD1466B
:1094600099460892D5F804C096F8B3EDCDF824C01B
:109470000138CDE90C9918BF01208DF83C00D5F8D2
:109480001490CDF81890ACEB01011EF0400F07913D
:109490000CD00CF1FF3000EBD07EB1EB6E0F40F33F
:1094A000B58040F00100C0EB4100079096F8AF0D89
:1094B00096F8B11D96F8B03D01934FF0000E00F004
:1094C000010C61F3070EC0F382006CF30F2E60F302
:1094D000174E63F31F6ECDF838E0D5E9193E0A93B5
:1094E000BEF1000F23D0079B02999944AB68022874
:1094F00003FB09130EEB830332D0BCF1000F3AD00B
:10950000002A0FDD9DF838C0394611F8010B84455B
:1095100018BF18700898A1F17402521B904203F111
:109520000103F2DC96F8B6EDBEF1010F2CD0AB6C66
:1095300005A89847E96A013911F0030FE96208BFED
:109540004BF0010BB8F1000F03D000293B463FF769
:1095500066AFBBF1000F40F08E8011B0BDE8F08F18
:10956000184601993CF03AFD9DF839C0089A034627
:10957000BCF1000FC4D1184639463CF04BFB96F8BD
:10958000B6EDBEF1010FD2D1DDE906329918AA6815
:10959000059BE86896F8B5CD02FB0131AB6E00FB88
:1095A00002F2BCF1010F03EB81010C9803EB820383
:1095B0002A6850D9002A27DDCDE9017403334FF022
:1095C000000C4FF0030911F8012B02EB42070333A3
:1095D000C75D03F8067C12FB09E70224C75D03F8A8
:1095E000057C12FB09420CF1010C825C03F8042C8F
:1095F0002A689445E7DBDDE90174D5E9023203FB13
:1096000002F2AB6E03EB82030B9390E700288646D1
:10961000B8BF0CF1020EB1EBAE0F07DD20F0030076
:1096200040F00200C0EB810107913FE7002884462B
:10963000B8BF00F1070CB1EBEC0F4FEAC10E07DD2C
:1096400020F0070141F00401AEEB010107912DE785
:10965000CDF81CE02AE7002AD6DD4FF0000C11F807
:10966000012B30F8122023F8022B2A680CF1010C90
:109670009445F4DBC1E7284611B0BDE8F04FFFF791
:10968000F1BD4746DA19934208D2013BE11914F8BB
:10969000012B03F8012FA142F9D1A86AC01BA862CF
:1096A00057E7704730B5D0E900431B1B9342B8BF62
:1096B00003F1FF3283B012B9104603B030BDC36866
:1096C00005461C4603F1080001AB83F039FA20B9C6
:1096D000236C01982B6003B030BD052078F0EAFFC1
:1096E00038B5C56804460A46CB1705F1080082F074
:1096F000B3FE286C206038BD10B545F6B8520C4654
:1097000000213CF06BFC00F5A04383F8B54D10BD83
:109710002DE9F04F0646436C856D87B00F465430F7
:10972000002106F5DA749847336C4FF480522146D5
:1097300006F15400984796F9BE1196F8BE2100290B
:109740000346A5EB0005C0F2F0804FF00D094FF085
:10975000000E42F21072CDE901E24FF0020BF24628
:109760001A4603970BF1FF339145049329DA4846D3
:10977000171AB7F5817F034604EB000131DB097846
:109780002C2942D03B291CD021291AD12344811CE9
:109790005F789878F92F00F0FD8008442318023094
:1097A0005F7867B101460F44791CE75DA2EB0109C0
:1097B00007F201134B455FDA002FF4D108469042BF
:1097C000D6DB039FD646ABF1020C019BBB60029B2C
:1097D000C7F800C00120FB60C7F804E007B0BDE88F
:1097E000F08F3A4620463CF049FA336CC7F5805278
:1097F000E11906F15400984721463A1809782D1AC4
:109800002C294FF000000346BCD19042D9DA234402
:1098100000F10A0993F909105B7A002953DB09F179
:10982000010103F20113571ABB4239DA631809F137
:1098300002091F787FB14946A946B1F5406F6EDD38
:10984000B9F1000F07EB01034DDCE75C591C002F59
:10985000F6D14D46894614F809303B2B04EB09013B
:1098600000F0B580002D6CD1A2EB09031F2B40F353
:10987000AE800BF1010B75E74A46214420463CF0CF
:10988000FDF9C9F5805204EB0901336C06F154006F
:109890009847002109EB00022D1A002F83D18DE794
:1098A0008A426BDC891A01F1010963184FF4805276
:1098B00021460027059306F15400336C9847059B19
:1098C0003A182D1AB5E703F00703022199404FF02B
:1098D000030011FB009909F1010103F20113571A6A
:1098E000BB42DDDAA2E7551A2A46214420463CF065
:1098F000C5F9C5F580524A45A8BF4A46336C61197F
:1099000006F154009847E35D2A18A9EB0009791C79
:10991000002B9ED00B44591CE75C002F99D00F44BC
:10992000791CE75D002F88D193E702F007024FF022
:10993000020909FA02F94FF003010D2219FB01296E
:1099400005E7B36DB3F5805F93DD002D91DDA2EBEC
:1099500009094A4620463CF091F9C9F58052AA42CD
:10996000A8BF2A4604EB0901336C06F1540098475E
:1099700009EB00022D1A4FF000097AE721443A461C
:1099800020463CF07BF94FF00109E119C7F5805200
:1099900023468FE704287FF400AF1F795B7947EAFD
:1099A0000323022BB8BF0223019F03EB8303B7EB12
:1099B000430F0AEB430A4FEA430C02DACDF804C026
:1099C000EBE6029B6345A8BF63460293E5E6DDF83C
:1099D00010C0039FD646F8E6FFF794BC2DE9F04F80
:1099E0008BB004460491934609B100230B60D4E97F
:1099F00015735A1E974227DA04F15402009204F5B7
:109A0000A041002281F8B42D81F8AE2D22624FF0E2
:109A1000FF32626207F1FF029A42C6BFDB1B03F10D
:109A2000FF394FF0FF0904F5DA750591236C0098B2
:109A30004A4629469847814506460ED00623E361EB
:109A400000200BB0BDE8F08F636C04F154000021DE
:109A500000909847D4E91573D1E7002F00F0978064
:109A600000212B4689461A782C2A22D0DA46B346A2
:109A70003B2A00F0E581212A40F0E78105EB09024D
:109A800009F102085278FE2A00F0F980FF2A00F05E
:109A9000A980012A6FD0F92A40F0EE8015F808203D
:109AA000042A00F055814146C1462C2AE0D15E4689
:109AB000D346294405EB090388785A7802EB002243
:109AC00022610879CA7802EB0022626188794A79BA
:109AD00002EB00222260087ACA7902EB002262605F
:109AE0005B7A059A82F8B33D1A0609F10A0800F17B
:109AF0006381059A15F8083082F8B23DAA4A0297A8
:109B0000D35CA361002308F10101009F636341F26C
:109B1000B478AA46CDF804B009E03CF07BF8626B5B
:109B20000BEB05012A446263002D00F0C382B142B1
:109B300001F1010B80F291811AF80150606BA6EBE4
:109B40000B0940444D4520442A460AEB0B01E4DD55
:109B50004A463CF05FF8616B236C49446163A5EBB6
:109B60000909414421444A4638469847636B3146C7
:109B700009EB0302D7E715F8083008F1010898440B
:109B8000002BF8D115F808204146C1468DE78749DA
:109B9000052228463CF028F838B185490522284698
:109BA0003CF022F8002840F0EE8094F8BE31B4F882
:109BB000BA212260A260C3F302120132A2610599A8
:109BC000B4F8BC216260E26094F8BF2181F8B02D46
:109BD0001A0681F8AF0D00F181800D2104F2C11346
:109BE000894640E75B46A34615F8086008F101097D
:109BF000A3EB090406F11F02A24227DA09EB0608CB
:109C00000B2E08D0002EEFD15C4615F808209B469D
:109C10004146C14649E7A944664901933246484650
:109C20003BF0E2FF019B0028DED199F80B20032ACC
:109C3000DAD199F80C20012AD6D199F80E1099F8AA
:109C40000D2002EB0122CBF82420CDE708F2B5115C
:109C50005944224628463CF011F804F5DA71DBF845
:109C600040300098594406F1200298474F44231889
:109C70004FF00009B046C3E70123E361E0E6414647
:109C8000A1466C5C4E1CABEB060804F11F03434578
:109C90000EDA3119D9F838303E441BB9C9F83860AA
:109CA000A9F83C40002CECD14C466A5C8946FCE6A5
:109CB00001F2B5114944424628463BF0DFFF08F562
:109CC000DA714944D9F84030009804F120029847ED
:109CD000374408EB000B00262146DBE703F00703BF
:109CE00003F101084FF0030906F5DA7109FA08F9E2
:109CF000236C009821444A469847059B064493F8F4
:109D0000B50D012842D804F58D514FF0020C1231E7
:109D10000CFA08FC8C44224692F8C23192F8C1E158
:109D20009B084FEADE0E5B0143EACE2392F8C3E1C3
:109D3000033243EADE0300B15BBA21F8023F61451A
:109D4000EAD1032101FA08F10D3189466B188AE640
:109D50002944059BC87883F8AF0D4E790A7902EB48
:109D6000062202EB82025200012AD8BF642222623C
:109D7000C00744BF8A7983F8B12D09F10809494623
:109D800015F8092091E60823E36159E604F58D50A2
:109D90004A4604F2C11109F10D0914303BF03AFFB3
:109DA000494605EB09035EE6107F0C0068330B00A3
:109DB00070330B0020310B0003F00703013306F56D
:109DC000DA7103229A4001932144236C0098029295
:109DD0009847059A92F8B51D029A0129064404F5A0
:109DE000A55000F27781019A02239340123003EBD1
:109DF000000E012303FA02FC04EB090292F8BF31C2
:109E000092F8BE819B084FEAD8085B0143EAC82359
:109E100092F8C081033243EAD80301B15BBA20F85B
:109E2000023F8645EAD10CF1FF3303EB430309F10E
:109E30000D0903EB0908059A012382F8B43D58E6A1
:109E40000723E361C4F864A0FAE5A36DDB1B1F2BB5
:109E50003FF712AF0723E361F2E5DDF804B0E369F1
:109E6000C4F864B0072B3FF4EBAD059B93F8B23D0B
:109E70004FF6FF7601339E4004F5BD53143336B2DE
:109E800003936368E3626FEA66062368A362B31C08
:109E90009BB2019304F5ED530E330025721C06931B
:109EA00004F576531FFA82FA2E3325632046029377
:109EB000FFF7D8F9BAF1000F14D02B4604F5ED5096
:109EC00004F5765504F59B412D350C302D3141F2CA
:109ED000187701F8013F05F8013F0133534520F899
:109EE000027FF6D1CAF580535B000993069BCDF83B
:109EF00000A003EB4A03F51C08930026A246059B2D
:109F0000099A93F8B28D08984FF6FF7308F101098A
:109F100041F2177108F1010803FA09F93CF05EF803
:109F2000DAF83000039BC8F12002B242B8BF00EB60
:109F3000E60003EB0001B8BFCAF830001F5C4878A8
:109F4000009B07EB00278878C97807EB0047B8BF6C
:109F500006F007060FFA89F907EB016727FA06F101
:109F60006FEA090909EA010189B28B42464400F00F
:109F7000818050460791FFF719FA019B07998B42A0
:109F800000F0A6804FF0010B0BFA08FB5346444645
:109F90001FFA8BFB07951FFA85FA98462EE0DA45E3
:109FA00015D2069B029A23F81A10515C02F80A1087
:109FB00033F815E041F217739E4518BF029B0AF56E
:109FC000805C16BF595D02F80C1003F80C100AF102
:109FD00001031FFA83FADA450BD30B2C09D8621C54
:109FE0004FEA4B0B4FEA490994B21FFA8BFB49F039
:109FF000010929464046FFF7D9F92946D8F82C50DF
:10A00000002D27DDC4F12005B54217DAD8F830500D
:10A01000039B05EBE60503EB050CC8F830505F5DCC
:10A020009CF8015007EB05279CF8025007EB054709
:10A030009CF8035006F0070607EB056727FA06F5BC
:10A04000009B09EA0505ADB2AB4226442FD0019B27
:10A05000AB42A4D14446049B13B1049A236A136013
:10A06000D4E91503013B9842ACBF002001200BB09E
:10A07000BDE8F08FB24213DADAF83020039B02EB2E
:10A08000E6029918CAF830209F5C4A7807EB02274D
:10A090008A7807EB0247CA7806F0070607EB0267E3
:10A0A00027FA06F109EA010189B2464461E7079DF2
:10A0B000C24624E7059A01238E42DDE901B782F802
:10A0C000AE3D7FF7CCAE0098636C39449847C6E646
:10A0D0005446C0E705EB0801143001923BF09AFDAD
:10A0E000019A9044A7E600BF2DE9F04F00221646E2
:10A0F00089B06C4B6C4C6D48CDE90222354601228B
:10A10000196841B1D4F80413114204D01D601968D4
:10A11000009100991643043383424FEA4202EFD183
:10A12000614BD3F87C21F1B2002A6ED00022C3F833
:10A130007C21D3F87C3101934FF0A042019BD2F8EF
:10A1400010255B4B0292D3F81035039300297DD183
:10A150000DF1100A00224FF0FF33564DDFF8508109
:10A160000492CAF804200693534C07934FF0000B57
:10A1700014F9013F5F1C31D0C3F3C20E0EF120026F
:10A180000DEB020C03F007021CF8086CD640F60732
:10A19000D9B203F03F0021D5484F3E18890996F9FE
:10A1A000286057F82660002E5BD003295BD01F285B
:10A1B00087BF03F01F03C64603464FF0A04E1CF8AE
:10A1C00018CC0EEB83032CFA02FCD3F800271CF00A
:10A1D000010FC2F301423CD0022A4FD0A542C7D1A1
:10A1E000BBF1000F2FD04FF0A0430299D3F81035E8
:10A1F000D8F81025994202D10399914223D0CDE994
:10A200000232DDE904230692AEE7D1B12B4F0125DE
:10A210000024A30003F180432E4203F5C0430BD07A
:10A22000D3F8100557F82420D3F81015C0F30520F3
:10A23000C1F3014102B190470134082C4FEA4505B2
:10A24000E7D1002E84DB09B0BDE8F08F46F0004670
:10A25000DCE7032AC2D1032921D0002EBED0B047AB
:10A26000BCE70329BAD11AF80E704FF0010909FAB8
:10A2700002F947EA09090AF80E9098E70329ECD198
:10A280004FF4403CD3F8002722F440320BF1010B8D
:10A2900042EA0C025FFA8BFBC3F80027DDE74FF4BC
:10A2A000003CEFE70061004000600040206100409A
:10A2B00000030050C1110120BF11012068110120CD
:10A2C00008B5042066F018FA2DE9F04FD1F80031F6
:10A2D000103B102B8BB0064600F25681AC4A22FA96
:10A2E00003F313F0010F14BF8A464FF0000A91F8F0
:10A2F00004C1351D4FEA0C1C06F114092C46231F1E
:10A300000CEB0A001A7810F8017B7A4003F8012B55
:10A310009C42F7D10434A1450CF1040CEFD191F823
:10A320000431013B06F11002DBB20492AC469A0004
:10A33000B6469EF80D309EF809609EF805509EF8CE
:10A3400001409EF802109EF80A008EF80D608EF80B
:10A3500009509EF80E609EF806508EF805408EF863
:10A3600001309EF807409EF803308EF802008EF808
:10A370000A109EF80B009EF80F108EF80B108EF846
:10A3800006608EF80E508EF803408EF807008EF8A7
:10A390000F307146002311F823007E4C205C01F839
:10A3A00023000133042BF6D101318C45F2D1960004
:10A3B00065462B1F0AEB0600197810F8014B614027
:10A3C00003F8011BAB42F7D11D1DA94506F1040698
:10A3D000EFD1002A00F0D580CDE905A9CDE907C26B
:10A3E000F346CDF824E09BF803E09BF800A09BF82F
:10A3F00001809BF802904FEADE164FEADA1706EB6F
:10A40000460606EBC60607EB470786EA4E0007EB53
:10A41000C70787EA4A074FEAD815C0F3C01CC7F33D
:10A42000C01205EB45050CEB4C0C4FEAD91405EBBB
:10A43000C50502EB42020CEBCC0C85EA48058CEA20
:10A44000400C009004EB44048AEA080002EBC202CC
:10A450008AEA090A82EA47028EEA0A06C5F3C013AD
:10A4600004EBC40484EA490488EA0908029689EAEC
:10A4700000098EEA000603EB4303C2F3C01003EBAE
:10A48000C30300EB400083EA4503C4F3C01100EBB3
:10A49000C00080EA42008EEA08085FFA87FAC3F338
:10A4A000C01E574001EB4101474001EBC1010EEBDB
:10A4B0004E0E81EA440101970EEBCE0EEFB28EEA0A
:10A4C000430E8AEA090A87EA08075D40C1F3C0180B
:10A4D000DBB283EA0A0308EB4808434008EBC808EC
:10A4E00088EA410803968EEA0303029E5FFA84F924
:10A4F00088EA030A009B89EA06094C40039EC9B218
:10A500007940DFB27740D2B27A405FFA8CF787EABF
:10A51000090742407840CCF3C01707EB47078EEAA3
:10A52000010107EBC70787EA4C0783EA0C0688EAB4
:10A530000101019B8EEA020288EA0000794078401E
:10A540007A40774059408EEA05058AEA070388EA8F
:10A5500004048BF803306840049B8BF800106240C1
:10A560008BF801008BF802200BF1040B9B457FF464
:10A570003AAFDDE907C2DDE905A9DDF824E0043AD8
:10A58000D7E60BB0BDE8F08F4FF0000AAFE600BF92
:10A5900001010100BC340C002DE9F04F89B0129E7E
:10A5A000002800F047820F4609681D469046824603
:10A5B00080F080FCB0F10009C0F2018239684944A2
:10A5C0003960504681F01AF9021EC0F2768239686D
:10A5D00011443960D8F8000009EB020CA0EB0C0024
:10A5E000C8F80000DAF8B817DAF8B037002956D101
:10A5F000002B55D10121CAF8B017D8F80010D7F8B0
:10A6000000E00129CDE903E9AEEB0C0C704622DD38
:10A6100001F1FF3B4FF0000E03E00EF1010EDE45AD
:10A6200019D0044610F8019BB9F1FF0FF5D194F849
:10A63000019009F0E009B9F1E00FEED19CF80000BB
:10A64000FF2800F0C5800EF1030EA1EB0E010129D9
:10A6500004F10300DCDC4FF0FF32DAF8C817DAF857
:10A66000C4C7CAF8B4270CFB01F2DAF8BC1701FB27
:10A6700002F2002A10DDA91E002021F8020FDAF8EC
:10A68000C847DAF8C42704FB02F2DAF8BC47013302
:10A6900004FB02F29342F0DB6FF0020095E04BB155
:10A6A000DAF8B44750467DF035FB2044CAF8CC07B1
:10A6B000D8F80000002E00F0BA80DAF8D827CAF8DF
:10A6C000CC07002A40F05D81904240F35A81CAF8DD
:10A6D000DC073E6830443860D8F80020DAF8CC1740
:10A6E000521AC8F80020DAF8C417002291420792E3
:10A6F00040F34581DAF8DC4703924FEAC4080AF2D6
:10A70000DC77D1462C46D9F8BC27002A40F3BD801F
:10A71000DDF81CA00597BB46002537460494564635
:10A72000DDF80CA020E05BF8043F43452BDC079FDD
:10A7300001953E449B1BCDF800A048467DF0F6FAFB
:10A740000028C7EBC003D9F8BC17A8EB060805F131
:10A75000010504EB0007C0F2D680079E8D4233440A
:10A76000A8EB030880F28E8007AA3946CDE900A540
:10A770004346484680F08EFC041EC6EBC4063C44AB
:10A7800007AA2146CFDAD9F8C427D9F8C807D9F8DB
:10A79000BC17049D00FB02F201FB02F2002ACA462C
:10A7A00011DD0021A81E0E4620F8026FDAF8C4372A
:10A7B000DAF8C847DAF8BC2704FB03F3013102FBDF
:10A7C00003F39942F0DB6FF0070009B0BDE8F08FAA
:10A7D00094F801909CF8010081457FF434AF9CF817
:10A7E00002B0A0788BEA000003283FF62CAFDDE929
:10A7F00003E91BF0020F18BF04F1FF34A4EB0E04B1
:10A80000DAF8C817DAF8C4C7CAF8B447002C0CFB4A
:10A8100001F0FFF628AFDAF8C017A1444A4401FB63
:10A8200002F2D20092FBF0F2CAF8B8273AE7DAF85F
:10A83000CC47844200F32181DAF8DC17DAF8D82714
:10A840009142C0F2BF80891A0AF11C063144304699
:10A850003BF014FADAF8D807DAF8CC273968304434
:10A860003BF0D8F9DAF8CC17DAF8D8270A44CAF856
:10A87000DC273A680A443A60D8F80020DAF8CC17A6
:10A88000521A2EE73E46DDE90447039948467DF01B
:10A890006BFF0028D9F8BC27C0F2CF80002A55DD15
:10A8A000DDF80CA0002501E095424FDA2A4651461A
:10A8B00048467EF095FC0028D9F8BC2705F1010533
:10A8C000F2DAD9F8C417D9F8C80700FB01F101FB87
:10A8D00002F2002ACA4611DD0021A01E0D4620F812
:10A8E000025FDAF8C827DAF8C43702FB03F3DAF8B4
:10A8F000BC27013102FB03F39942F0DB6FF00A0041
:10A9000009B0BDE8F08FD9F8C427D9F8C807049D6D
:10A9100000FB02F201FB02F2002ACA4611DD00210F
:10A92000A81E0E4620F8026FDAF8C437DAF8C847D6
:10A93000DAF8BC2704FB03F3013102FB03F399426D
:10A94000F0DB6FF0080009B0BDE8F08FD9F8C81748
:10A95000039B03FB01F102FB01F104EB41014846BB
:10A9600080F020FA0028D9F8C427C0F2C780039BE2
:10A9700001339342039307F10807FFF6C4AE0020AA
:10A9800023E7DAF8C427DAF8C807DAF8BC1700FBBF
:10A9900002F201FB02F2002A11DD0021A81E0C4682
:10A9A00020F8024FDAF8C827DAF8C43702FB03F3BD
:10A9B000DAF8BC27013102FB03F39942F0DB6FF0B8
:10A9C000050002E70AF11C002246084439683BF002
:10A9D00021F9DAF8CC17DAF8DC270A44CAF8DC27C0
:10A9E0003A680A443A60DAF8CC17D8F80020521ACC
:10A9F000C8F80020DAF8C817DAF8C42701FB02F219
:10AA0000DAF8BC1701FB02F2002A10DDA91E30465D
:10AA100021F8020FDAF8C827DAF8C43702FB03F38B
:10AA2000DAF8BC27013602FB03F39E42F0DB6FF03D
:10AA30000100CAE66FF00400C7E6D9F8C417D9F8D8
:10AA4000C80700FB01F101FB02F2002ACA4611DD32
:10AA50000021A01E0C4620F8024FDAF8C827DAF8C9
:10AA6000C43702FB03F3DAF8BC27013102FB03F31E
:10AA70009942F0DB6FF00900A7E6DAF8C817DAF8B8
:10AA8000C42701FB02F2DAF8BC1701FB02F2B24262
:10AA900010DDA91E304621F8020FDAF8C827DAF8CF
:10AAA000C43702FB03F3DAF8BC27013602FB03F3D9
:10AAB0009E42F0DB4FF0FF3087E6DAF8C827DAF87D
:10AAC000C407DAF8BC1700FB02F201FB02F2002A0D
:10AAD00011DD0021A81E0C4620F8024FDAF8C82725
:10AAE000DAF8C43702FB03F3DAF8BC27013102FBC2
:10AAF00003F39942F0DB6FF0060066E6D9F8C80769
:10AB0000D9F8BC1700FB02F201FB02F2002ACA4688
:10AB100011DD0021A01E0C4620F8024FDAF8C827EC
:10AB2000DAF8C43702FB03F3DAF8BC27013102FB81
:10AB300003F39942F0DB6FF00B0046E6012913DDC9
:10AB4000821E431E114401E08B420DD09C4613F837
:10AB5000012FFF2AF8D15A7802F0E002E02AF3D15F
:10AB6000C0F10100604470474FF0FF30704700BFF4
:10AB700008B17EF087BA704788B338B50D461146E4
:10AB8000044680F097F9013026D0D4F8D037032B53
:10AB900022D1D4F8B8372B60D4F8BC376B60D4F826
:10ABA000C02710491023C5E9022394F8D437D4F8FC
:10ABB000D02703EB4303013A1344D4F8BC2731F9FF
:10ABC000133002FB03F32B61D4F8D0376B6194F898
:10ABD000D437AB61002038BD6FF0050038BD6FF091
:10ABE0000400704778750C007DF042B810B54FF046
:10ABF000804386B0D3F80443620703D5D3F8082115
:10AC0000002A62D1A30605D54FF08043D3F8142162
:10AC1000002A4FD1600605D54FF08043D3F81821A4
:10AC2000002A3BD1210604D54FF08043D3F81C21E4
:10AC30004ABBE20504D54FF08043D3F82021B2B9D6
:10AC4000A30512D54FF08043D3F824216AB1002226
:10AC5000C3F82421D3F82421214B0592059A1B68BF
:10AC6000022006B0BDE81040184706B010BD002213
:10AC7000C3F820211A4AD3F8203104930120136825
:10AC8000049A9847DCE70020C3F81C01144AD3F863
:10AC90001C3103931368039A9847CAE70022C3F84C
:10ACA0001821104AD3F81831029301201368029A30
:10ACB0009847B7E70020C3F814010A4AD3F81431C3
:10ACC00001931368019A9847A4E70022C3F808216A
:10ACD000054AD3F8083100931368009A984791E722
:10ACE0009C7001209870012094700120064BD3F8CD
:10ACF00000213AB1054A00205071C3F800011368E1
:10AD000091681847704700BF00900240747001209E
:10AD100002480322002135F04DBB00BF00B00040C7
:10AD200002480422012135F045BB00BF001001405C
:10AD300002480422022135F03DBB00BF0040024022
:10AD400008B50F4A0F4B934208D2013AD21A22F0AB
:10AD500003020D49043218463AF05CFF0B4A0C4BD3
:10AD6000934208D2013AD21A22F00302043200219F
:10AD700018463BF033F900F0FBF86BF083FE00BFA0
:10AD8000AC0601200000012070870C009C7B012094
:10AD9000C00601200149024876F0BCBEB06F012018
:10ADA0000030004002494FF0402076F0B3BE00BFB3
:10ADB000E46F01201D4BD3F8182102B9704700B58C
:10ADC00000211B4A83B0C3F81811D3F8181192F868
:10ADD00020300191FF2B01990FD0917F69B9D17F6C
:10ADE000B1B11F2B86BF134803F01F034FF0A040E3
:10ADF000012101FA03F3C0F80C35D2E900E1002388
:10AE00000D4853771372734603B05DF804EB18478F
:10AE10001F2B86BF074803F01F034FF0A0400121FE
:10AE200001FA03F3C0F80835E7E700BF003002403D
:10AE3000506F012000030050586F01201F4BD3F8C2
:10AE4000182102B9704700B500211D4A83B0C3F82C
:10AE50001811D3F8181192F844300191FF2B019981
:10AE600011D092F8421071B992F84310C1B11F2B62
:10AE700086BF144803F01F034FF0A040012101FAE0
:10AE800003F3C0F80C35D2E909E100230E4882F83B
:10AE9000413082F82C30734603B05DF804EB18475C
:10AEA0001F2B86BF074803F01F034FF0A04001216E
:10AEB00001FA03F3C0F80835E5E700BF00F00240EF
:10AEC000506F0120000300507C6F012070B5234CAF
:10AED00082B00226002501A866F0A4FD05280BD04B
:10AEE000019B032B2CD01ED8022BF4D101A8257076
:10AEF00066F098FD0528F3D1194E4FF40C751948EA
:10AF0000ADF802500DF1020166F018FDE0B9D6F877
:10AF1000B440002CF3D0D4E90112246811489047C2
:10AF2000002CF8D1EBE7A3F10902022AD3D80A2BAF
:10AF300008D0092B14BF0120022076F0B7FCCAE725
:10AF40002670C8E70020F8E70C2801D002B070BDD9
:10AF5000054906484AF00EFF02B070BD887B01200B
:10AF6000A4700120206D0120182F0B00C85B0B007E
:10AF700008B54FF08053D3F83021082A1FD0754A06
:10AF8000D2F8883043F47003C2F88830BFF34F8F93
:10AF9000BFF36F8F4FF01023D3F80C22D20700F1CC
:10AFA000BB80D3F80022002AC0F29080D3F804328C
:10AFB000002BC0F28B80684B684A1A6008BD4FF0C6
:10AFC00080400021C0F80C11654AC0F81011C0F88B
:10AFD0003815D3F80414C2F82015D3F80814C2F8B1
:10AFE0002415D3F80C14C2F82815D3F81014C2F89D
:10AFF0002C15D3F81414C2F83015D3F81814C2F86D
:10B000003415D3F81C14C2F84015D3F82014C2F834
:10B010004415D3F82414C2F84815D3F82814C2F8FC
:10B020004C15D3F82C14C2F85015D3F83014C2F8CC
:10B030005415D3F83414C2F86015D3F83814C2F894
:10B040006415D3F83C14C2F86815D3F84014C2F85C
:10B050006C15D3F83411D3F844C4C2F870C5F1B1FB
:10B0600051B14FF08043D3F80024D10787D56FF05A
:10B070000102C3F8002482E74FF08053394AD3F825
:10B0800030314FF40071082BC2F840167FF477AFCF
:10B090004FF08043D3F80024D107E8D46FE7A2F53E
:10B0A000E042DFF8C8C0C2F88CC602F520424FF07B
:10B0B000FB0CC2F818C5D0F8E42ED3F8583263F36D
:10B0C0000302C0F8E42E0029D6D0CAE7264A01239D
:10B0D000C2F80435D2F80034002BFBD04FF0102317
:10B0E0001221214AC3F80012D2F80034002BFBD001
:10B0F0004FF0102312211C4AC3F80412D2F8003476
:10B10000002BFBD000231849C2F80435D1F80034D5
:10B11000002BFBD001F036FB134A0123C2F80435A3
:10B12000D2F80034002BFBD04FF010210E4AD1F89A
:10B130000C3223F00103C1F80C32D2F80034002B9A
:10B14000FBD000230849C2F80435D1F80034002BA5
:10B15000FBD0DFE700ED00E0000001200090D0030D
:10B1600000C000400090024000E001404881030020
:10B170000149024835F076B9986F012000900040EF
:10B180000149024835F06EB9A46F012000A00040CB
:10B190000149024876F0C8BF187001200020004025
:10B1A0000149024876F0C0BF3C7001200080024097
:10B1B000002079F0E3BA00BF094BD3F8002172B147
:10B1C00000B5084A83B052689047054B0022C3F887
:10B1D0000021D3F800310193019B03B000BD7047FB
:10B1E000000001406C700120022A2DE9F0431ED0BE
:10B1F000444C02EBC20204EB021404F1480601F1D4
:10B2000044058C3400F1240750F8043B54F804C979
:10B2100056F804EB1A468EFB028241F8042B8CFB95
:10B220000323B84245F80439EED1BDE8F083354B2D
:10B230008268D3F838C18CFB02428469D3F820516C
:10B2400085FB046422440A60D3F83C71426887FBA2
:10B250000242C469D3F8245185FB046422444A6045
:10B260000268D3F8406186FB0242056AD3F82841A0
:10B2700084FB05E52A448A600268D3F84491964627
:10B2800089FB0E2E026AD3F82C4184FB02827244A1
:10B29000CA604268D3F848E18EFB0242C469D3F821
:10B2A000305185FB048422440A618268D3F84C81C2
:10B2B00088FB0242D3F83451836985FB03431A4467
:10B2C0004A6143698CFB03238B61036987FB03237A
:10B2D000CB61C36886FB03230B62C36889FB03232E
:10B2E0004B6203698EFB03238B62426988FB023247
:10B2F0000023C1E90F33C1E90D33CA624B640B630C
:10B30000BDE8F083D07C0C002DE9F047B0F85E304A
:10B310000446002B71D0434E434D0F46904646F0F5
:10B3200001064FF0000A4FF0010994F8622072B351
:10B330000AF00F034FF40041194101EA080100230C
:10B3400013E01F2A86BF02F01F0228464FF0A040DC
:10B3500009FA02F2C0F8082594F862200133DBB242
:10B3600002EB4202B3EB420F0FDA2269D25C0029F2
:10B37000E7D11F2A86BF02F01F0228464FF0A040E7
:10B3800009FA02F2C0F80C25E6E7B4F85E30DB1BE0
:10B3900053450CDA94F834301F2B86BF03F01F039B
:10B3A0002A464FF0A04209FA03F3C2F8083594F890
:10B3B00061301F2B8ABF2A464FF0A04203F01F03C3
:10B3C00009FA03F3C2F808354020B04794F8613019
:10B3D0001F2B8ABF2A464FF0A04203F01F0309FA31
:10B3E00003F3C2F80C354020B0470AF1010AB4F863
:10B3F0005E301FFA8AF2934297D894F834201F2ABD
:10B4000007D84FF0A04101239340C1F80C35BDE8A7
:10B41000F087054902F01F0201239340C1F80C3563
:10B42000BDE8F08730850C0000030050054B18681C
:10B430000368D3F8402112B10022C3F8402100F084
:10B440003DBF00BF18120120002800F05E822DE9E8
:10B45000F84304460069002800F01A8294F861302D
:10B4600094F862101F2B8CBFDFF82CC34FF0A04C58
:10B47000002900F0F2810FFA81F901EB4101490046
:10B480000022C54E884615464FF0010E01E08A4263
:10B4900013DA835C1F2B88BF374603F01F0398BF66
:10B4A0004FF0A04701320EFA03F3BC45D2B245EA91
:10B4B0000305ECD00120BDE8F883B5F1807F34BFEF
:10B4C00000230123DB0015F47F0F43F0040218BFB3
:10B4D000134615F47F4FEAB200F0DF81002A00F036
:10B4E000B18143F00303012202FA03F341F208029F
:10B4F000134200F0B48109EB4902022302FA03F877
:10B500001A4694F86310B4F85E6084F86030012342
:10B510008B40073606F4FF6684F86630DBB216FB14
:10B5200003F694F8653003FB06F694F8683002FBE6
:10B5300006F6E66403B17600012108EB060061F02F
:10B5400037FC6062002800F0A381831932466361F2
:10B5500000213AF043FD94F8610094F8603094F8CB
:10B560006260012100F01F0201FA02F28B4245EAFB
:10B57000020500F09781022B00F0C981C4E906257D
:10B58000002284F864209EB1D4E904359B5C03F06A
:10B590001F0301FA03F345F8223094F86230501C7F
:10B5A000C2B203EB4303B2EB430FEDDB94F861004F
:10B5B00094F8653094F8341094F8665001229A405B
:10B5C000013A4FF47A43B3FBF5F3B3FBF2F3642B88
:10B5D00038BF64231F29C4E914338CBF6E4B4FF06E
:10B5E000A043002284F86A2003F5A162A26201F060
:10B5F0001F01012202FA01F194F8442003F20C53D6
:10B600001F2AC4E90B318CBF634B4FF0A04302F0FB
:10B610001F0103F5A16503F20C5203461F2B4FF0E7
:10B62000010000FA01F188BF03F01F03C4E90F21F4
:10B6300003F5E07388BF584AA56398BF4FF0A04256
:10B6400040F2033142F8231094F861201F2A86BF8C
:10B6500002F01F0250494FF0A04101239340C1F86E
:10B660000C3594F834301F2B86BF03F01F034A4A71
:10B670004FF0A04203F5E07340F2033142F823108B
:10B6800094F834201F2A86BF02F01F0242494FF06F
:10B69000A04101239340C1F80C3594F844301F2B8E
:10B6A00086BF03F01F033C4A4FF0A04203F5E0734E
:10B6B00040F2033142F8231094F844301F2B86BF28
:10B6C000354A03F01F034FF0A042012606FA03F3A8
:10B6D000C2F8083594F862303BB32F49002340F29A
:10B6E00003372269D25C1F2A88BF02F01F020D4671
:10B6F00002F5E07298BF4FF0A0454FF0A04045F82A
:10B7000022702269D25C1F2A84BF02F01F02084601
:10B7100006FA02F2C0F80C2594F862200133DBB27D
:10B7200002EB4202B3EB420FDBDB47F6FF720C2168
:10B730002046FFF7E9FD40220D212046FFF7E4FDFA
:10B7400094F86230C3B11449002301252269D25C08
:10B750001F2A08468CBF02F01F024FF0A04005FAD6
:10B7600002F2C0F80C2594F862200133DBB202EB40
:10B770004202B3EB420FE9DB94F86320012000FAA8
:10B7800002F3023B84F86D30002A6FD0024D002195
:10B79000844640F2033714E0000300501F2B86BF9D
:10B7A00003F01F032A464FF0A0420CFA03F3C2F83D
:10B7B000083594F863200131CBB29A424FEA400039
:10B7C00054D9A66C06EB01120B01127B1F2A8CBF09
:10B7D0002A464FF0A04202F5A162F250A26C1A4430
:10B7E000167B1F2E8CBF2E464FF0A04606F20C563D
:10B7F0005660A66C1E44327B02F01F020CFA02F265
:10B80000B260A26C1A44127B1F2A86BF02F01F028C
:10B810002E464FF0A04602F5E07246F82270A26C68
:10B8200094F86D601A440642137BB7D11F2B86BF74
:10B8300003F01F032A464FF0A0420CFA03F3C2F8AC
:10B840000C35B6E743F00203DBB2012202FA03F340
:10B8500013F48B7F03D0134653E60D46894609EB5C
:10B86000490204234FEAC2081A464AE694F86130B6
:10B870001F2B10D84FF0A04303F5A16203F20C5325
:10B880002046C4E9012300F0A7FC0020BDE8F883AE
:10B890000220BDE8F8833D4BEEE7002A6CD043F070
:10B8A0000103D1E727693978C1F3C101C4E906254D
:10B8B00084F86410002E3FF47BAE3A78606902F0A1
:10B8C0001F0203FA02F2C900CA40027094F8622013
:10B8D00002EB42025200012A7FF768AE1D46226940
:10B8E00094F86410D25C606902F01F0205FA02F25B
:10B8F000C900CA40C25494F862200133DBB202EBA3
:10B900004202B3EB420FEADB50E60320704727699F
:10B910003B78C4E90625C3F3001284F86420002EA6
:10B920003FF446AE3B78606903F01F0301FA03F36E
:10B930001201D340038094F8623003EB43035B00B1
:10B94000012B7FF733AE0A460D46236994F8641045
:10B950009B5C606903F01F0305FA03F30901CB4008
:10B9600020F8123094F862300132D2B203EB430374
:10B97000B2EB430FE9DB19E6012202FA03F313F4F9
:10B980008B7F3FF4B3AD1346BBE500BF000300500F
:10B9900090F86030012B05D0022B01D000F000B9E7
:10B9A00000F046BA00F000B82DE9F04F8FB090F8E3
:10B9B0006830446A03910546924633B190F86A3084
:10B9C000C26CC3F1010302FB034495F86560062EC7
:10B9D00000F0E080C6F10503DBB24FF4006202FA2A
:10B9E00003FC402202FA03F1012202FA03F095F867
:10B9F0006670002F00F0CB80B5F85E30D5F814B03B
:10BA0000CDF82CC000220492DA1D4FEAD208C3EB15
:10BA1000C80354FA83F20AF1FF3300241BB20894DE
:10BA20008E460993A94634465146002C00F0858085
:10BA30000023CDE90CE0CDE905230B9DCDF828804E
:10BA40008246F446079399F967000028B8BF404240
:10BA5000013840B2421C55D0059C039B01FB00F607
:10BA600007FB06F610F0010E03EB860607FB01F359
:10BA70006ED099F96720002A74DB002900F08480D9
:10BA8000049A164406EB43070022CDE9000904EBB3
:10BA90000108029136F8121037F8120011EA050376
:10BAA00018BF9BF8003011EA0C0F1CBF9BF80190E7
:10BAB00043EA090311EA0A0F1CBF9BF802100B436B
:10BAC00028421CBF9BF803100B4310EA0C0F1CBF4D
:10BAD0009BF804100B4310EA0A0F1CBF9BF80510DB
:10BAE0000B4304F8013B7244444512B2D2D1DDE964
:10BAF0000009029999F86670431E58B2431CACD1F4
:10BB000099F86540079B4FEA4C0C002B38D1052C67
:10BB100036D94FF0010A4FF40065069B059A0A9842
:10BB200001330693DBB202EBC002A34205920793F6
:10BB300089D3DDE90CE0DDF82880089B0133089308
:10BB4000DBB29F4223D9049B03EB410304936CE7D0
:10BB50000029D1D0049A164406EB43074FF0010E9A
:10BB6000002292E781B1089A013FBF1A01FB07F753
:10BB700006EB4707099A07EB43064FF0FF3E84E7C1
:10BB80006D004FEA4A0AC8E7431E58B265E70FB096
:10BB9000BDE8F08F102020214FF4004C27E700BFB4
:10BBA0002DE9F04F95B09246059190F868104569DF
:10BBB000436AC26C0E9061B1014690F86A0091F838
:10BBC0006010B2FBF1F1C0F1010000FB01F103EBE9
:10BBD00081030E9890F86510B0F85E40062900F0D9
:10BBE0002081C1F10501C9B24FF400608840109076
:10BBF000402000FA01F6012000FA01F71846002162
:10BC00003AF0ECF903460E9890F86220002A00F012
:10BC1000FD80E11D4FEAD10CC4EBCC01C9B205F1A6
:10BC2000180B03EB81050AF1FF339BB2002111933E
:10BC300090F8669004910133069331460895CDF84B
:10BC400034C0B9F1000F00F0D8800E9ACDF83CA0B6
:10BC5000002392F8652007930B930B46002A00F00F
:10BC6000BB80BDF944100C91CDE912370024494640
:10BC7000DDF84080DDF83890DDF83CC009949A4644
:10BC8000BE460A9499F9674084EAE473A3EBE4732F
:10BC9000013B5BB2581C00F08480089E274660463A
:10BCA00087EAE772049CA2EBE772D2B204FB02328D
:10BCB00000FB02F2059C01FB02F213F0010504EB0C
:10BCC000820201FB00F451D0002F58DB002800F065
:10BCD000A5800799571807EB440C0022CDE9029084
:10BCE000CDE9003631462C4606EB800637F8129037
:10BCF0003CF8125019EA080318BF5BF8183C19EA1F
:10BD00000A0F1CBF5BF8140C034319EA0E0F1CBF8B
:10BD10005BF8100C034315EA080F1CBF5BF80C0C12
:10BD2000034315EA0A0F1CBF5BF8080C034315EA2E
:10BD30000E0F1CBF5BF8040C034351F8040B2244A4
:10BD400018438E4212B241F8040CCFD1DDE90290C3
:10BD5000DDE90036069A99F8661006EB8206013B8B
:10BD60005BB25A1C1AD099F9677099E70028F6D08F
:10BD70000799571807EB440C01250022AEE700286D
:10BD80004CD00B9D0139491B00FB01F102EB410C2A
:10BD90000CEB44070C9A4FF0FF359FE799F86520AC
:10BDA00084460A9B4FEA4A0A002B32D1052A30D931
:10BDB0004FF0010E4FF40068099B08980D9C013369
:10BDC0000993DBB200EB4410934208900A93FFF40E
:10BDD00059AFDDE9123789460B9907980F9C01315D
:10BDE0000B91C9B200EB4400894507903FF636AF8E
:10BDF00019460E9B93F86220A246049B01330493DC
:10BE0000DBB29A420BF1180B3FF61BAF15B0BDE841
:10BE1000F08F4FEA48084FEA4E0ECDE7013B5BB288
:10BE20003EE74FF40041102720261091E6E600BFC0
:10BE30002DE9F04F95B04569059190F86810109282
:10BE4000466AC26C834659B190F86A009BF860104C
:10BE5000B2FBF1F1C0F1010000FB01F106EB41067C
:10BE60009BF86510BBF85E40062900F01E81C1F109
:10BE70000501C9B24FF4006000FA01F340200E93AF
:10BE800000FA01F301200F9300FA01FA0021304675
:10BE90003AF0A4F89BF86220002A00F0FC80E31D31
:10BEA000DF08C4EBC703DBB206EB4304109B9BF82F
:10BEB00066800894013B1FFA83FC002304930CF175
:10BEC0000103CDF844B00693644605F10C0B0D97C1
:10BED0004046002800F0D680119991F86530002284
:10BEE00007920B921A460B461099D046002A00F092
:10BEF000BA80DDE90E594FF0000C26B2C246CDF8EB
:10BF000048800C96CDF824C01394CDF828C08846FC
:10BF100093F9677087EAE771A1EBE77101394CB2D9
:10BF2000611C00F084800899049A87EAE776A6EB02
:10BF3000E776F6B202FB064608FB06F6059A00FB1A
:10BF400006F614F0010C02EB860600FB08F251D055
:10BF5000002F5ADBB8F1000F00F0A48007980644C8
:10BF600006EB42070022CDE90041CDE9023801EBA2
:10BF7000480E084636F8121037F8124011EA050349
:10BF800018BF3BF80C3C11EA090F1CBF3BF80A8CA8
:10BF900043EA080311EA0A0F1CBF3BF8081C0B43D5
:10BFA0002C421CBF3BF8061C0B4314EA090F1CBFB4
:10BFB0003BF8041C0B4314EA0A0F1CBF3BF8021C9D
:10BFC0000B4330F8021B62440B43864512B220F843
:10BFD000023CCFD1DDE90238DDE90041069A93F851
:10BFE000660001EB4201621E54B2621C1DD093F93F
:10BFF000677099E7B8F1000FF5D00798064406EB93
:10C0000042074FF0010C0022ADE7B8F1000F49D014
:10C01000471E0B983F1A08FB07F706EB470707EB8D
:10C0200042064FF0FF3C0C9A9DE793F865200A9971
:10C030004FEA4909002931D1052A2FD94FF0010AC9
:10C040004FF400650999089C0D9E01310991C9B210
:10C0500004EB0614914208940A91FFF459AF41464B
:10C06000139CDDF848800B9D079E01350B95EDB2C2
:10C0700006EB4106A84207963FF638AF119B93F8AE
:10C080006220C246049B01330493DBB29A420BF157
:10C090000C0B3FF61EAF15B0BDE8F08F6D004FEAF8
:10C0A0004A0ACFE7621E54B23EE74FF40043202015
:10C0B000CDE90E304FF0100AE8E600BF90B110B5A0
:10C0C00000F0AAFA0446406A08B160F089FDA06C4D
:10C0D00008B160F085FD206918B160F081FD002392
:10C0E000236110BD704700BF2DE9F04182B09DF87B
:10C0F0002C409DF824609DF830709DF834E09DF848
:10C1000038C09DF93C500194002857D0109C002D58
:10C1100008BF0125002C51D00446052B28BF05235C
:10C12000002D84F8675084F86520B8BF6D42019AED
:10C1300084F86120EDB203EB4302052E109884F8D9
:10C140003470A4F85C104FEA420215FB01F1374647
:10C150004FF0000528BF05272060A4F85E10D0B27C
:10C1600084F844E084F868C084F86230A5646562AD
:10C1700084F863700121804660F01AFE206130B3BC
:10C180000121380160F014FE0346A0642069CBB1A0
:10C190000899424639F03EFD66B10A9B591E2B466E
:10C1A000A26C11F8015F02EB03120133D8B287428F
:10C1B0001573F5D8002002B0BDE8F081032002B06D
:10C1C000BDE8F081019360F00BFD019B236102202B
:10C1D00002B0BDE8F08100BF00286BD070B590F8C8
:10C1E000662090F86530511E013B82B0012A80F82C
:10C1F0006B3080F86C1088BF90F86C3090F863104A
:10C200004FF000028CBF03F1FF33012380F86D3043
:10C2100080F86E20826500293DD04FF0010C264940
:10C2200040F20334E64612E01F2B86BF03F01F03E3
:10C230000D464FF0A0450EFA03F3C5F8083590F807
:10C2400063500132D3B29D424FEA4C0C23D9836C28
:10C2500003EB021316011B7B1F2B86BF03F01F038A
:10C260000D464FF0A04503F5E07345F82340836C7D
:10C2700090F86D50334415EA0C0F1B7BD4D11F2B63
:10C2800086BF03F01F030D464FF0A0450EFA03F3DF
:10C29000C5F80C35D3E7019000F030FA0198036837
:10C2A00001224FF47A715A60DA60C3F840151A60BF
:10C2B00002B070BD704700BF000300502DE9F0418F
:10C2C000836B026C1A60D0E90B321A60836A026BCE
:10C2D0001A600368A54F01265E6003685E64D3F8A8
:10C2E0004435C26A90F86B30016B1160054603F06B
:10C2F000FF0837433BBB90F863104446F9B195F80B
:10C300006C3095F86D2053401E424FEA041010D057
:10C31000AA6C95F86CC002EB04131CEA060F99682E
:10C3200014BF13585B684FF400701960B84795F854
:10C3300063100134E3B299424FEA4606DFD895F81C
:10C340006C3085F86D3095F86B3095F865200133C9
:10C35000DBB29A4285F86B300DD8002285F86B204D
:10C3600095F86C3095F866100133DBB2994285F888
:10C370006C3040F298802A6D2B6802FA08F1012295
:10C380005A604020DA60C3F840151A60B847D5E912
:10C390000F321A60B5F85E2095F86C1095F865C0FC
:10C3A00095F86B3095F860E007320CFB0133D6103E
:10C3B000D10895F86820C9000EFB03F301FB03F3D5
:10C3C00022B195F86A20E96C01FB02336A6ABEF17A
:10C3D000010F02EB0307D5E90640D5E9013100F072
:10C3E000C780F2B2561EBEF1020FF6B26CD0002A20
:10C3F00041D007EB461607F12002403652F8207C68
:10C400001F601C6000BF00BF086052F81C7C1F60EA
:10C410001C6000BF00BF086052F8187C1F601C60E1
:10C4200000BF00BF086052F8147C1F601C6000BF92
:10C4300000BF086052F8107C1F601C6000BF00BF86
:10C44000086052F80C7C1F601C6000BF00BF0860D1
:10C4500052F8087C1F601C6000BF00BF086052F8E3
:10C46000047C1F601C6000BF00BF2032B242086025
:10C47000C4D195F865C0BCF1010F12D995F86B30A5
:10C480007BB92A68012353642B6DD2F84425C3EB92
:10C49000C303134404336A6DDB08934238BF134669
:10C4A0002B65BDE8F08185F86C2095F86E303BB1C6
:10C4B00095F86A30C3F1010385F86A3085F86E207B
:10C4C000AB6D0133AB6556E7002AD4D007EB0616F7
:10C4D00007F1100206F1200795F8646003EB4606A9
:10C4E00032F810CCA6F800C01C6000BF00BF086086
:10C4F00032F80ECCA6F800C01C6000BF00BF086078
:10C5000032F80CCCA6F800C01C6000BF00BF086069
:10C5100032F80ACCA6F800C01C6000BF00BF08605B
:10C5200032F808CCA6F800C01C6000BF00BF08604D
:10C5300032F806CCA6F800C01C6000BF00BF08603F
:10C5400032F804CCA6F800C01C6000BF00BF086031
:10C5500032F802CCA6F800C01C6000BF00BF103249
:10C5600097420860BCD195F865C084E730850C001F
:10C57000002E80D0013EB6B207EBC60607F10802D6
:10C5800006F1100795F864601E4412F808CC86F88E
:10C5900000C01C6000BF00BF086012F807CC86F81E
:10C5A00000C01C6000BF00BF086012F806CC86F80F
:10C5B00000C01C6000BF00BF086012F805CC86F800
:10C5C00000C01C6000BF00BF086012F804CC86F8F1
:10C5D00000C01C6000BF00BF086012F803CC86F8E2
:10C5E00000C01C6000BF00BF086012F802CC86F8D3
:10C5F00000C01C6000BF00BF086012F801CC86F8C4
:10C6000000C01C6000BF00BF083297420860BCD168
:10C6100095F865C02FE700BF002860D0436A002B63
:10C620005DD010B490F86E30002BFBD102684FF053
:10C63000010CC2F804C00268C2F844C0816BD2F891
:10C640004425026C0A6090F86220C2B1244903F0CC
:10C65000FF030269D25C1F2A0C468CBF02F01F0246
:10C660004FF0A0440CFA02F2C4F80C2590F86220B6
:10C670000133DBB202EB4202B3EB420FE9DBB0F86D
:10C680005E3023B3164C00224FF0010C90F861305D
:10C690001F2B21468CBF03F01F034FF0A0410CFA63
:10C6A00003F3C1F8083500BF00BF90F861301F2BBD
:10C6B00021468CBF03F01F034FF0A0410CFA03F397
:10C6C000C1F80C35B0F85E3001329A42DED3836A8D
:10C6D000026B1A60D0E90B321A6010BC70477047C9
:10C6E0000003005090F8683033B1012380F86E30B9
:10C6F00090F86E30002BFBD1704700BF1E4A0368D4
:10C70000934212D002F5805293422ED002F580520D
:10C7100093422CD002F5803293422AD002F5805207
:10C72000934208BF042201D070470022134B03EB51
:10C73000C201002091F9041053F832304FF4803CCC
:10C74000012281425A60C3F80405DA60C3F8080583
:10C75000C3F81005C3F804C3E6DB4809084B01F031
:10C760001F018A4043F8202070470122DEE70222A1
:10C77000DCE70322DAE700BF0080004038850C00C8
:10C7800000E100E0BFF34F8F0549064BCA6802F491
:10C79000E0621343CB60BFF34F8F00BFFDE700BFE4
:10C7A00000ED00E00400FA05014B1868704700BF77
:10C7B0005000012007EE900AF5EEC07AF1EE10FA73
:10C7C00001D400F009B808B580F0004000F004F88A
:10C7D000404261EB410108BD70B5FBF731FA0C4BEB
:10C7E000002204460D46FBF749FCFBF773FD0646A5
:10C7F000FBF704FA074B0022FBF740FC02460B460E
:10C8000020462946FBF7BCF8FBF764FD314670BDB6
:10C810000000F03D0000F04110EE101A21F000433E
:10C820000122B3F1FF4FF0EE407A026015D2002BE7
:10C8300072D000B5B3F1E45F87B013D20029BEBF58
:10C840004FF0FF330360B1EE400A37F0D1FAB1EE9A
:10C85000407AB0EE470A07B000BD20EE007AB0EE95
:10C86000470A704700295EDBB3F17E5F68D0B3F101
:10C87000804F65D04A0000F19F809FEDDD6ADD4A60
:10C88000934240F2A382DC4A934240F24A82F0EEA5
:10C89000005A75EEE75A9FEDD67A9FEDD85ADFED34
:10C8A000D86ADFEDD84A9FEDD84A65EEA57AE7EE63
:10C8B000856AA7EEA44A9FEDD55ADFEDD54AA6EECC
:10C8C000A75AE4EE274ADFEDD36A9FEDD34AE5EE9F
:10C8D000276AA4EEA74A9FEDD15ADFEDD14AA6EE12
:10C8E000A75AE4EE274ADFEDCF6AE5EE276A9FED0F
:10C8F000CE5AA4EEA75A66EEA56AB6EE004AE5EE59
:10C90000276AF0EE667AE5EEC47A37EE877A002978
:10C910009FDA36EE477A9CE7DFEDB57AF7EE006AEC
:10C9200086EEA77A9BE7B3F1964F0CD3DFEDB07A92
:10C93000F7EE006A86EEA77AB0EE470A07B000BDB0
:10C940009FEDAB7A85E7B3F17A5FC0F05982B1EE23
:10C95000407A8DED020AB0EE470ACDE90410039348
:10C960008DED017A2FF05EFA9DED017ADDED027A10
:10C97000059AB4EE407AF1EE10FADDE9033140F0A9
:10C980009A819FEDAA7A37EE677A17EE100A00F0C7
:10C99000010007EE100AB8EEC77A8000CDE9013138
:10C9A0000492CDED037A062800F28A82DFE800F0D7
:10C9B0005DDFDF5959ECEC00B3F1824F80F09B81D1
:10C9C0009FED8B6ADFED9A6ADFED9A5ADFED9A4AA6
:10C9D000BDEEE77AB8EEC75A17EE103A77EEC57A91
:10C9E0009FED965AE7EEA65A033BA7EEA45ADFED59
:10C9F000946ADFED944AE5EEA76AE5EE274ADFED9B
:10CA0000925A9FED925AE6EEA75AA4EEA75ADFED8E
:10CA1000906ADFED904AE5EEA76AE5EE274ADFED82
:10CA20008E5A9FED8E5AE6EEA75AA4EEA75ADFED76
:10CA30008C6AE5EEA76AF7EE005AE5EE275A66EE35
:10CA4000A76AF6EE004A86EEA57AA7EEA47A042B32
:10CA50003FF65DAFDFE813F0C900AC002701180115
:10CA60002A01F7EE006A36EEC77A9FED7E0ADFED07
:10CA7000600A27EE000A002000F06CFFDDE90131BA
:10CA8000DDED037A049AF1EE406AF5EE406AF1EECC
:10CA900010FA3FF44BAF27EEA67A9FED720ACDED68
:10CAA000026AB0EEC77A80EE070ACDE9033105923B
:10CAB000CDED017A37F09CF9DDED026ADDED017A0A
:10CAC000F5EEC06AF1EE10FADDE90331B0EE407A1E
:10CAD00003D5059A4FF0FF301060B3F17E5F3FF44D
:10CAE000B8AEB3F1804F3FF4B4AE4800F1EE677AD0
:10CAF000B0EE476A7FF5C3AEB3F1824FFFF462AF89
:10CB0000B0EE670A8DED036A0291CDED017A37F040
:10CB10006FF9DDED017A9FED542ADFED542A9FED88
:10CB2000543ADFED543A9FED544ADFED544A9FEDFD
:10CB3000547A02999DED036AF7EE006A86EEA75AD1
:10CB4000F6EE005A77EEE55A65EE057A70EE666A03
:10CB5000E7EE822AA2EEA73AE3EE273AA3EEA74A2F
:10CB6000E4EE274AA4EE857AA5EEA67ACFE6F6EEA5
:10CB7000006A36EEC77A9FED3B0ADFED1D0A27EE0D
:10CB8000000A00F029FB79E7F7EE086A37EE667ACB
:10CB90009FED340ADFED160A27EE000A00F01CFBB9
:10CBA000DDE90131DDED037A049AF0EE406A6CE7CD
:10CBB000F7EE006AB0EE080A37EE800A20EE260A89
:10CBC000F0EE006A77EEA67A8DED037A27EE800A02
:10CBD0008DED026A019137F00BF99DED037A019911
:10CBE0009DED026A37EE007A91E6B7EE000AE7E7BC
:10CBF000000000006666663F17A6DD3FA283D337BC
:10CC000067976739752C3C384584E238A1549C3AC3
:10CC100034B6053A7E02F23BC66E3D3B01F0893DDB
:10CC20001599A83C3F239E3D661AA53E0000004B87
:10CC300067FF0538B435F13ABDD7F536D6EE4B3A35
:10CC4000E440DA3C54BF983CE6DC153E6E0F303EC3
:10CC50007ACCA63EC5D0383F5A245C3E3B2DB23F2D
:10CC60003F239EBDDB0F4940E8C4D5BAD23D5B3AB5
:10CC70005C061CBAFD0C503A610B36BBABAAAA3D50
:10CC80001D7FD63E00000000F7EE006AF1EE045A68
:10CC900077EEA55A65EEA65AF1EE006A77EEA66A1F
:10CCA00066EEA56A86E7F7EE005AF5E7F1EE086A48
:10CCB00077EEA66AEAE7F6EE006A27EE267ACDE975
:10CCC0000231B0EE470ACDED047A8DED017A2FF0F6
:10CCD000A9F89DED017A059A37EE407ADDE9023137
:10CCE00037EE077AF0EE477AFEEECF7A17EE900A2B
:10CCF000DDED047A52E6B3F1B94FC0F097808DEDC7
:10CD0000020A8DED010A37F073F8B7EE007A30EEC3
:10CD1000477ADDED027A1FED256A019927EE277A21
:10CD2000F5E5724A934240F28480DFED716A9FED2F
:10CD3000717A77EEE66A66EEA62A9FED6F4ADFED1E
:10CD40006F5ADFED6F4A9FED6F5ADFED6F3A9FED3F
:10CD50006F3A62EEA67AE7EE844AA7EEA55A9FEDF7
:10CD60006C4ADFED6C5AA4EEA74AE5EE275ADFEDD8
:10CD70006A4A9FED6A5AE4EE274AA5EEA75AA7EE43
:10CD8000A33ADFED675A9FED674ADFED673AA5EEFC
:10CD9000274AE4EEA75AE3EE273ADFED644A9FED17
:10CDA000645AE4EE265AE3EEA74ADFED626A9FED8D
:10CDB000624AE5EEE76AA4EEA75AF0EE667AD2EE92
:10CDC000857A77EEC47A37EE877AA0E5B0EE670A07
:10CDD000CDE902318DED046ACDED017A37F008F826
:10CDE000564A029BDDED017A03999DED046A934258
:10CDF000B1EE407A5CD9F7EE005A75EEE75A4CE591
:10CE00009FED4F0ADFED3B0A0293CDE9031027EEB9
:10CE1000800A0020CDED017A00F09CFDDDE90231B1
:10CE2000DDED017A049AF0EE406A2EE69FED316A5C
:10CE300066E6B7EE007A77EEC77A9FED2E7A9FED21
:10CE4000415ADFED416ADFED415ADFED414AE7EE3D
:10CE5000856AE7EEA54A9FED3F5ADFED3F5AA6EE01
:10CE6000A75AE4EEA75ADFED3D6ADFED3D4AE5EE55
:10CE7000276AE5EEA74A9FED3B5ADFED3B5AA6EE47
:10CE8000A75AE4EEA75ADFED396AE5EE276AB7EE56
:10CE9000005AA5EEA75A66EEA76AFEEE004AC6EE55
:10CEA000855AF0EE656AE7EEA46A36EE877A2EE5DB
:10CEB0002F4A9342C3D9DFED2F6A77EEE66A3AE74D
:10CEC000F0EE006A37EE667A9FED1D0ADFED090A83
:10CED00027EE000A002000F03DFDDDE90131049A53
:10CEE000DDED037AF1EE406ACFE500BF1FA69D3F5E
:10CEF000C316BB3F0000000027F9A3B9F7E9AF391B
:10CF000067F8663A85300DBA6B7BA53976F4B7BA07
:10CF1000FE7771BB9916143B3D37933CFEFC28BC51
:10CF20003C2117BE155A843D07E7C73B474D06BD58
:10CF30005EB9F73E521CE631CDCDF83D1F4A3B3F6E
:10CF4000DB0F49405E3C5B3C78756A3EDBD5523B6B
:10CF5000AF72D53DB24B7A3FDFEF443FE73ABA3F7D
:10CF60002D390840F400223FBE2E1D403F239EBDB8
:10CF700007336D3E0C5BEC3E10B510EE104A884A4C
:10CF800024F00043934288B0014662D9854A934217
:10CF900022D824F00043002CDFED837A834A23F06B
:10CFA0000F0340F3E380934230EE670A09BFDFEDE1
:10CFB000807A9FED807A9FED807A30EE670A70EE7E
:10CFC000477A30EE670AC0ED007A30EE470A80ED0E
:10CFD000010A012008B010BD784A934240D89FED65
:10CFE000787A9FED716AB0EEC00AF6EE007AE0EE54
:10CFF000077A9FED707AFDEEE77AF8EEE76A17EEB2
:10D00000900AA6EEC60A1F2866EE877A30EE677A87
:10D010006BDCDFF8C0C100F1FF3E24F000425CF899
:10D020002EC022F0FF0262455FD081ED007A30EE23
:10D03000470A002C30EE670A81ED010ACADAB1EE28
:10D04000477AB1EE400A81ED007A81ED010A404253
:10D05000C0E7002380ED000A4360002008B010BD47
:10D06000B3F1FF4F72D2DA15863AA3EBC25307EE43
:10D07000903ABDEEE77ADFED536AB8EEC77A77EE05
:10D08000C77A8DED057A67EEA67ABDEEE77AB8EE3F
:10D09000C77A77EEC77A8DED067A67EEA67AF5EE57
:10D0A000407AF1EE10FACDED077A5DD1B5EE407A17
:10D0B000F1EE10FA56D1012343480190022000906E
:10D0C00005A8039100F00AF9002C039982DA91ED8A
:10D0D000007AD1ED017AB1EE477AF1EE677A81ED0F
:10D0E000007AC1ED017A404274E717EE102AC2F3CC
:10D0F000C752C2EBD352082A97DD9FED2D7ADFEDA0
:10D100002E5AB0EE406AA6EEC76A70EE467AE6EE98
:10D11000C77AD6EEA57A36EE677A17EE102AC2F3F2
:10D12000C752C2EBE353192B17DD9FED287ADFEDD1
:10D13000285AB0EE460AA6EEC70A76EE407AE6EE28
:10D14000C77AD6EEA57A30EE677A6EE730EE400AFF
:10D1500080ED010A80ED000A7FE7B0EE460A81ED1E
:10D16000007A64E70223A7E70323A5E7934230EEA2
:10D17000270A09BF9FED0E7ADFED0E7ADFED0E7AFA
:10D1800030EE070A30EE277A30EE470A80ED007A5B
:10D1900070EE277AC0ED017A4FF0FF301AE700BF3A
:10D1A000D80F493FE3CB1640800FC93FD00FC93F8E
:10D1B000004435374344353708A3852E800F494353
:10D1C00084F9223F0000804398380C0000A3852E8C
:10D1D00032318D2418380C0010EE103A23F0004341
:10D1E000B3F1485F2CD2FDEEC07A17EE903A002BD7
:10D1F00060D060EE007A9FED317A9FED315ADFED1D
:10D20000315A9FED316ADFED316AA7EE875A9FED03
:10D21000307AE7EE855AA7EEA56AA7EE867AE7EEA2
:10D22000876A66EEA76A60EEC00AB6EE007AE7EE9D
:10D23000A60AB7EE000AD7EE870A30EE600A7047FA
:10D2400060EE007A9FED1D7A9FED1D5ADFED1D5AAD
:10D250009FED1D6ADFED1D6A1E4AA7EE875A9342B5
:10D260009FED1B7AE5EE275AA5EEA76AA6EE277A70
:10D27000E7EE276A66EEA76AD5D9174A934214D813
:10D2800003F17F4307EE103AB7EE006A36EE476AC5
:10D2900060EEC00AF6EE005A97EEA57AE7EEA60A0F
:10D2A00037EE607A36EE470A7047B6EE076AB5EE9B
:10D2B000027AEDE7B7EE000A704700BF4ED747ADE0
:10D2C000F6740F317CF293B4010DD037ABAA2A3D2E
:10D2D000610BB6BA9999993E0000483F2DE9F04F8D
:10D2E0002DED048BDBB01C4603938B46C64B68992F
:10D2F000069253F82150111D814604F1FF38C0F207
:10D300005082D31E48BF131DDB1004930133D90094
:10D31000069B15EB0804A3EB010218D4049B9FEDB8
:10D32000BE7A699E0134A3EB08031C441EA8002B9F
:10D33000A4BFF75C07EE907A03F10103ACBFF8EEEF
:10D34000677AF0EE477AA342E0EC017AEFD1002D44
:10D35000C0F2E680039BB8F1000F0DF58C7C4646C9
:10D3600005EB030EB8BF0020C0F2CD80039B1EAFBB
:10D3700007EB83079C0009EB8300DFEDA77ABA4631
:10D380004B46F3EC016A3AED017A8342E6EE877A86
:10D39000F7D101367645ECEC017A07F10407ECD1C0
:10D3A00009ABCDE907B10DF1280A03EB85039FED29
:10D3B000979ADFED978A05934C440AEB850746AEB2
:10D3C000019510460DEB8503002D93ED460A4FEABB
:10D3D000850B16DD06EB0B03524660EE097AB0EEC4
:10D3E000407AFDEEE77A73ED016AF8EEE77AB34230
:10D3F000A7EEE87A37EEA60ABDEEC77AA2EC017A6C
:10D40000EBD1029064F078F8B0EE408AB4EE000AF6
:10D4100028EE000A2EF006FDF2EE007AA0EE678AF2
:10D4200002980028FDEEC89AF8EEE97A38EE678A8D
:10D4300079DD691EC0F108035AF821E04EFA03FCB9
:10D440000CFA03F3AEEB030EC0F1070219EE903AAB
:10D450004EFA02F26344002A09EE903A4AF821E0BB
:10D4600000F3F280B5EE408AF1EE10FA6CD1019B28
:10D470009D420CDD0AEB0B030021944653F8042D6A
:10D48000BB4241EA0201F9D1002940F03981019BF8
:10D49000013B05F1010C5AF82330002B40F02E819E
:10D4A000059B012153F8042D0131002AFAD02944AB
:10D4B000699B049A03EB020E039BAE441D441EAB12
:10D4C00003EB850547AB9B441EF8013F07EE903AFE
:10D4D000F8EE677AB8F1000FE5EC017ADFED4E7AED
:10D4E00009DB2A464B46F3EC016A32ED017AA3428E
:10D4F000E6EE877AF7D10CF1010C8C45EBEC017A62
:10D50000E2DD0D465EE7731C7345CCF8000006F1C2
:10D51000020605D0B645CCF804000CF1080CF2D197
:10D52000039B9C003CE700F0D280F6EE007AB4EE5C
:10D53000E78AF1EE10FA80F22381B5EE408AF1EE2F
:10D5400010FA4FF0000292D0DDE907B1069B029578
:10D55000B0EE480A019D0190C81A914663F0CCFFD5
:10D560009FED2B7AB4EEC70AF1EE10FADDE9012344
:10D57000C0F28B81DFED257A60EE277A5C1CFDEE30
:10D58000E77A0832F8EEE77AA7EEC70AFDEEE77A07
:10D59000BDEEC00A10EE101A4AF8231017EE903AAA
:10D5A0004AF824301046B7EE000A63F0A5FF002CBD
:10D5B000B0EE407AC0F294810AF1040347A9DFED8E
:10D5C000136A03EB840301EB8401A20046AF73ED01
:10D5D000017AF8EEE77A534567EE877A27EE267AE6
:10D5E00061ED017AF3D1002D0DF1C80CC0F29581E7
:10D5F0001744E646264600209046064ADFED067AA6
:10D600003946002312E000BF0C380C000000803BBC
:10D6100000008043E0370C0000000000F2EC016ADB
:10D62000B1EC017A9D42E6EE877A03DB834203F197
:10D630000103F3DD013E731CCEED007A77D00EF1CD
:10D64000040E0130043FD8E70133002D09EE903A73
:10D6500040F33C8151464FF0000E51F8043B2BBB88
:10D660000EF1010E7545F8DC9E4600280ADD012802
:10D670007ED0022806D1691E5AF8213003F03F0CF3
:10D680004AF821C0022A7FF4EDAEB7EE000A30EE70
:10D69000488ABEF1000F3FF4E5AE0992029063F0B4
:10D6A0002BFF0298099A38EE408ADBE6C3F58073B7
:10D6B00041F8043C04E00B68C3F1FF0341F8043B6C
:10D6C0000EF1010E7545F6DC4FF0010ECDE76B1E35
:10D6D0005AF823201212002A7FF7C4AE19EE903AAE
:10D6E000002D03F1010309EE903AB3DC022A7FF426
:10D6F000B9AEF7EE007A37EEC88AB3E66146D7E6F0
:10D700006C1E59465AF82430019DDDF81CB0E146E4
:10D71000A0F10802002B7FF445AF0B4609A90B448A
:10D7200053F8041D013C083A0029F9D03AE7424673
:10D73000689B022B5EDC002B37DC10D10CF104035C
:10D740005FED4B7A134433ED017A634577EE877AC8
:10D75000F9D1B9F1000F40F0A980CBED007A19EEB4
:10D76000903A03F007005BB0BDEC048BBDE8F08F8E
:10D77000691E5AF8213003F07F0C4AF821C081E776
:10D7800019EE903A002D03F1010309EE903AC8BF5B
:10D7900002223FF75FAFF7EE007A37EEC88A022227
:10D7A00060E6002308210493B2E50CF10401DDEDED
:10D7B000327A1FED677A0A4472ED016A624537EEEC
:10D7C000267AF9D1B9F1000F67D177EEC77A8BEDE0
:10D7D000007A64B10123B1EC017A01339C4277EE07
:10D7E000877AF8DAB9F1000F01D0F1EE677ACBED64
:10D7F000017AB4E7689B032BB1D1002C00F08A803A
:10D800000CEB020090ED007A0346014671ED017ABF
:10D81000F0EE476A37EE277A614577EEC77A81EDF9
:10D82000007A77EEA67AC1ED017AEFD1012C71D0A2
:10D8300090ED007A0CF1040173ED017AF0EE476A85
:10D8400037EE277A994277EEC77A83ED007A77EE42
:10D85000A67AC3ED017AEFD15FED917A8B180CF1C6
:10D86000080C33ED017A9C4577EE877AF9D1DDED2E
:10D87000326A9DED337AB9F1000F1AD1CBED006A0F
:10D880008BED017ACBED027A69E7BDEEC00A1C464A
:10D8900010EE101A4AF8231084E6F1EE476A77EE8C
:10D8A000C77ACBED006A002C94D19EE7F1EE677A3F
:10D8B00053E7F1EE666AB1EE477AF1EE677ACBEDA7
:10D8C000006A8BED017ACBED027A48E7012815D08A
:10D8D00002287FF40BAF0EF03F034AF8213005E732
:10D8E000689B022B12DC002B25DC7FF438AF5FED48
:10D8F000B67AB9F1000F3FF430AFD7E70EF07F03EF
:10D90000022A4AF821307FF4ADADF2E6689B032B82
:10D910007FF425AF5FEDC07AA9E70020614623467A
:10D920000860002B3FF404AF023B5D1C486001F12E
:10D930000801F5D1FCE6DDED327AB9F1000F04D033
:10D940004FF00043CBF800304FE70023CBF8003016
:10D950004DE700BF10EE103A23F00043B3F1485FEB
:10D9600004D2FDEEC07A17EE903A5BB360EE007A17
:10D970009FED157ADFED155A9FED156ADFED156AFB
:10D98000E7EE875A9FED147AA5EEA76A20EE275A94
:10D99000E6EE276AA6EEA77A30B9DFED106AE7EE69
:10D9A000876AA6EE850A704727EE457AF6EE006A8A
:10D9B000A0EEA67ADFED0A6AD7EE270AE5EE260A80
:10D9C00030EE600A704700BFD3C92E2F342FD7B274
:10D9D0001BEF3836010D50B98988083CABAA2ABE26
:10D9E000ABAA2A3E10EE103A23F00042B2F1465F95
:10D9F000F0EE407A10D2BDEEC07A17EE101A01BBDD
:10DA0000431C134300F0A080012800F09C80BFEE6F
:10DA1000007A87EE270A70474F498A4211D39FED5B
:10DA20004F7ADFED4F6A002BBCBFF1EE600AF1EEDA
:10DA3000407A77EE677A36EEE07ADFED4A0A77EEE3
:10DA4000277A67EEA76ADFED484ADFED485A9FED77
:10DA5000485A9FED486A404926EEA67A8A42E7EE88
:10DA6000245AA7EE056ADFED444A9FED445AE5EEDD
:10DA7000874AA6EE075ADFED425A9FED426AE4EE6E
:10DA8000875AA5EE076ADFED404A9FED405AE5EE62
:10DA9000874AA6EE075A9FED3E6ADFED3E5AA4EE96
:10DAA000876AE5EE075AB0EE467AA5EEA67A27EE2B
:10DAB000A65AB0EE606AA7EE056ADFED374AE6EED9
:10DAC000260AE5EE240A37EEA00A1ED201283AD033
:10DAD000BFEE007AC7EE006A10EE103A6FF30B0348
:10DAE00006EE103A16EE903A76EE677A6FF30B0375
:10DAF00000EE103A70EEE70AF7EE007AE6EE007AF2
:10DB0000E0EE807AA7EEA60A704707EE100AF8EE5C
:10DB1000C76A20EE007A30EE260A9B1787EE006A6D
:10DB200003F00203C3F10103F0EE005A36EE606A1F
:10DB300007EE103A77EEC67AB8EEC77AE7EEE56AF6
:10DB400026EE870A70477047F0EEC07AB7EE007A8B
:10DB500087EE270A704700BF40A12C3FDA0F493FEC
:10DB600068212233000000005FAE9BB745F4A33864
:10DB70008453D9377AC09538C8261A3AB9378139CB
:10DB800016696B3B48DEBE3AA427B33C1F37113CF5
:10DB90008988083ED10D5D3DABAAAA3E42084B08DC
:10DBA00002F0553203F05533801AC91A8A088308E7
:10DBB00001F0333100F0333002F0333203F033330D
:10DBC0000344881803EB131300EB101003F00F331A
:10DBD00000F00F30184400EB002000EB0040000E76
:10DBE000704700BF2DE9F04782B00646DDF828E017
:10DBF0000846B4460D46002B4ED18A4214466DD9D4
:10DC0000B2FA82F242B1C2F12003954026FA03F340
:10DC100094401D4306FA02FC260CA7B2B5FBF6F1B0
:10DC20004FEA1C4306FB115543EA054301FB07F08D
:10DC3000984209D9E31801F1FF3580F00381984239
:10DC400040F20081023923441B1A1FFA8CFCB3FBFB
:10DC5000F6F006FB10334CEA034C00FB07F3634578
:10DC60000AD914EB0C0C00F1FF3580F0ED80634510
:10DC700040F2EA80A444023840EA0140ACEB030CD5
:10DC80000021BEF1000F04D02CFA02F30022CEE9ED
:10DC9000003202B0BDE8F0878B4209D9BEF1000F17
:10DCA00001D0CEE900610021084602B0BDE8F0874E
:10DCB000B3FA83F1174600294DD1834202D3B24211
:10DCC00000F20F81B6EB070C60EB030301201D4649
:10DCD000BEF1000FDDD0CEE900C5DAE7002A00F082
:10DCE00098801A46B4FA84F3002B40F0AF800B1BE7
:10DCF000270CA6B20121B3FBF7F54FEA1C4007FB46
:10DD0000153340EA034306FB05F8984507D9E318A5
:10DD100005F1FF3002D2984500F2E8800546A3EBFA
:10DD200008031FFA8CFCB3FBF7F007FB10334CEA37
:10DD3000034C06FB00F3634508D914EB0C0C00F10F
:10DD4000FF3602D2634500F2CE803046ACEB030CC6
:10DD500040EA054095E7C1F120058B4022FA05FC19
:10DD60004CEA030C00FA01F426FA05F3E84002FA43
:10DD700001F943EA04084FEA1C4206FA01FAB0FB33
:10DD8000F2F71FFA8CF602FB17004FEA184444EA38
:10DD9000004407FB06F0A0420AD91CEB040407F17B
:10DDA000FF3380F09C80A04240F29980023F64449F
:10DDB000241A1FFA88F3B4FBF2F002FB104443EA82
:10DDC000044300FB06F69E4209D91CEB030300F155
:10DDD000FF3480F082809E427FD90238634440EA5B
:10DDE0000740A0FB09749B1BA3423E46A04664D398
:10DDF00061D0BEF1000F0AD0BAEB060263EB080354
:10DE000003FA05F5CA401543CB40CEE90053002183
:10DE10003FE7730843EAC1734A08190C41EA02411B
:10DE20004FEAC67C9BB2B2FBF4F02646A0462746DA
:10DE30001F2243EA0143B1FBF4F1A3EB080341EADB
:10DE4000004158E72946FFE6284615E71A46C3F180
:10DE500020019C4026FA01F320FA01F1904003438F
:10DE6000270C06FA02FCB1FBF7F0A6B207FB10156F
:10DE7000190C41EA054100FB06F58D423BD96118BA
:10DE800001D28D4220D8491B0138B1FBF7F501952D
:10DE900005FB06F8019D9BB207FB151143EA014300
:10DEA000434526D2E31805F1FF31C6D24345C4D21B
:10DEB000A91E2344C1E7BA459BD2B7EB090664EB20
:10DEC0000C040138A04694E7651B29440238B1FBD5
:10DED000F7F5019505FB06F8DCE720467FE71F46CE
:10DEE00066E70846F4E6A44402382FE7023D2344DF
:10DEF00015E70199A1E7491BB1FBF7F5019505FB72
:10DF000006F8C7E770B590F82A30DC0657D4054606
:10DF100040F21A500E4647F03BFF044688B1436872
:10DF200030469847A36801219B6906469847002818
:10DF300047D1A36805F1080130469B68BDE87040F1
:10DF400018472349304640F029FF0446C0B190F8F5
:10DF50005030D90635D443F0100305F1080180F89C
:10DF6000503029F0AFFE95F82A3013F00C0F204600
:10DF700018BF0121BDE8704008BF002129F092BE02
:10DF80001449304640F00AFF0446E8B190F82A30C0
:10DF90009A0716D443F0020305F1080180F82A30ED
:10DFA00028F0AEFE95F82A3013F00C0F204618BF6B
:10DFB0000121BDE8704008BF002128F051BE0EF0DD
:10DFC00017FD054874F0CEFB044874F0CBFB00BF8E
:10DFD00040FD0B000CFB0B00A4A30B0094A30B0053
:10DFE00010B5144684B01A6030B1104600215EF0BE
:10DFF000DFFE98B104B010BD084603A9019365F097
:10E0000063F8019B20B90398002801DD1860EDE753
:10E01000186800215EF0CCFE0028EBD101462046B6
:10E020005EF0C6FE0028E5D1092062F065FB00BF66
:10E0300012F0ACBD2DE9F84F834608462A4940F05E
:10E04000ADFED0F808A0BAF1020F4AD9D0F80C8082
:10E05000DBF8040001224FEA8A012FF06FFC002454
:10E060000746CBF80440ABF80840254658F8250091
:10E070001E4940F2055238F0CBFF58F8256040F2B7
:10E0800005527068022138F041FFB0684FF4D46146
:10E0900039F012F84FF4D46347F6FF721449814601
:10E0A00038F024FFF06840F2A66139F005F8013439
:10E0B00040F2A6630E4947F6FF720646A4B238F056
:10E0C00015FF07EB8503544527F825905E8025460C
:10E0D000CCD34FEA4A0ACBF80470ABF808A0BDE8ED
:10E0E000F88F044874F02AFB64720B00547E0B0016
:10E0F0000080FFFF34A10B002DE9F0472DED028BCE
:10E100001C4696B0C368BDF88470BDF88C600546A7
:10E11000B0EE408A8A46002B00F0D18041688B42E5
:10E1200000F014818E4B18784FF00008FF2885F816
:10E13000458013D0019263F00BFC29468146894843
:10E140000AF0D4F939F00803019AC5F80C8085F873
:10E150004480484602D00EF0A1FB019A1F2F66D9D9
:10E16000BAF1000F40F0A480002E40F0D680259632
:10E170004FF00A09002A00F08F8040F20123ADF829
:10E180003830002C00F09980631C0DF13808ADF890
:10E190003A30404600230F9363F0FCFB0346002B0C
:10E1A0003FD1DFED717A9FED716A259A099228EED1
:10E1B000277A229A0D93C7EE067A9E4208BF1A4626
:10E1C00022920692209A0492694A089302FB04F470
:10E1D000684A0B93A2FB04240122640BF6EE006A4A
:10E1E00077EEA67A8DF83520FCEEE77A08224146D4
:10E1F0001846ADF81470ADF81C608DF820900C93A3
:10E20000CDED0A7AADF82C4001930CF0C9F8002846
:10E210005BD1534808AA04A963F096FB0346002883
:10E2200061D0184616B0BDEC028BBDE8F0871F2EFA
:10E230003BD8BAF1000F75D0259B002B00F08C80E5
:10E240001B799DF80810F0EE0C7A03F07F03B4EE12
:10E25000E78A63F34701F1EE10FA259B8DF8081069
:10E2600066D807EE904A9FED447AF8EE677AF4EEAE
:10E27000C77AF1EE10FA5BD8D3F80530CDF8093043
:10E28000259BB3F80930ADF80D3002AB25934FF064
:10E290000209002A7FF471AF0DF138084046CDE93C
:10E2A0000E2263F077FB034679E7BAF1000F34D012
:10E2B000002325934FF006095CE7234665E71F2FEF
:10E2C00080F845303FF64CAFB1E7C2B20199404605
:10E2D00063F04EFB034600289BD0184616B0BDECF9
:10E2E000028BBDE8F0871E4C1E492A4605F1280026
:10E2F0000AF0D2F821789DF99020012063F054FBB8
:10E30000034600288DD12078012163F01FFB0346CE
:10E31000002886D1209AEA6083E7CDF894A04FF0D8
:10E32000080927E7A6B1CDF894A04FF0040921E72A
:10E33000D3F80530CDF80930259BB3F80930ADF896
:10E340000D3002AB25934FF0030913E7112368E763
:10E3500025964FF005090DE74FF001090AE700BFC8
:10E36000A70601206D0A03000024744900401C44E4
:10E3700040420F005917B7D16666A63F38B5DFEDAA
:10E38000117A416020EE270A0446BCEEC00A049DC3
:10E3900080ED020A11461A469DF8143084F82030A8
:10E3A0000C3062F065FC35B1224628460649BDE8CE
:10E3B00038400AF071B821460348BDE838400AF0F9
:10E3C00037B800BF00007A4415C70300F0B583B02A
:10E3D000416017464A68044690790A9A84F82C00EE
:10E3E00022858D7D05F0300605F0060500283DD11B
:10E3F0004FF6FF72E284002E44D1089BE36194F84B
:10E400002C20099B2362002384F82D3084F82A30C5
:10E41000A3840B9BDAB1002B3BD02349224618463C
:10E420000AF03AF85EB116F0040118BF01216068E5
:10E430001ABF84F82B100022012213F05BF925B1DA
:10E44000AA060ED5022384F82B3003B0F0BD2BB3FF
:10E450001649224618460AF01FF8002DF5D06B0722
:10E46000F0D5012384F82B3003B0F0BD4A68019346
:10E47000D0680AF0BDFE32462E46019BE084154668
:10E48000002EBAD01A46394604F1080062F0F0FBBB
:10E49000B3E70548214609F0CBFFC3E7034821460F
:10E4A00009F0C6FFD9E700BF9DB3080015B4080006
:10E4B0002DE9F0414FF6FF7682B003610023154647
:10E4C00081608371C360C27104468680084601A9D9
:10E4D0000BF04AFB681C221D01A9C0B263F082FA4E
:10E4E000074618B1384602B0BDE8F0810F4AA5884A
:10E4F0001388DFF84080AB4228BF2B4613800C4ABC
:10E500001388AB4238BF2B461380044638F81400FA
:10E51000B0422A46294601D063F068FA4434B4F583
:10E52000AA7FF3D1384602B0BDE8F081A4060120ED
:10E53000FC780120A00A01202DE9F04F89B0814626
:10E540001D4640689DF848808A46164658F0B8FD3A
:10E55000002D4FD088F00108DFF8ACB04FEA481822
:10E56000002701E02D1B45D0B5F5806F2C464246B3
:10E5700028BF4FF4806403A94846CDE90667CDE97A
:10E5800004478DF80C708DF80DA001F03DFE584544
:10E590002644E7D00190D9F8040058F073FD184ADA
:10E5A000019B934219D00BD9164A934210D0013ADD
:10E5B00023F00203934218D0002009B0BDE8F08F89
:10E5C000043A93420ED16FF0730009B0BDE8F08FAA
:10E5D0006FF0120009B0BDE8F08F6FF00F0009B0C6
:10E5E000BDE8F08F03329342E6D16FF0040009B02A
:10E5F000BDE8F08FD9F8040058F044FDDCE700BF17
:10E600000B00AD0B0100AE0B0000AD0B2DE9F04F80
:10E6100085B0804601920C46002A40F03D8201F10F
:10E620000C06D4F800A03BF00BF898F80020404608
:10E63000002A77D04FF000095746CB46292A5BD0F5
:10E640005E2A00F2EB81232A3FD9243A3A2A3CD8A9
:10E65000DFE812F0A6013B003B003B005B013B0002
:10E660001C01FA003B003B00DB013B003B003B0090
:10E670003B003B003B003B003B003B003B003B00C2
:10E680003B003B003B003B003B00B0013B003B003C
:10E690003B003B003B003B003B003B003B003B00A2
:10E6A0003B003B003B003B003B003B003B003B0092
:10E6B0003B003B003B003B003B003B003B003B0082
:10E6C0003B00B10074003B006B002768002E00F097
:10E6D00091827A1C22600122F2552268511C21602D
:10E6E00098F80010B15445466268013262606A7859
:10E6F00005F10108002AA1D14046BBF1000F0DD061
:10E700002268A2EB0B02013A51B2914218BF49F0C4
:10E7100001095FFA89F90EB106F80B20B9F1000F73
:10E7200040F0B68105B0BDE8F08F2268571C276025
:10E73000002ED8D05021B1542768D4E798F8012092
:10E74000002A00F0A581276842F02001642908F121
:10E75000010507F1010000F0FD8142F02402772A53
:10E7600000F0F881002E00F0488201222060F2556E
:10E77000226898F80110531CA1F161002360324413
:10E78000152800F2F481DFE810F076027302F2013E
:10E79000F201F2016D02F201F201F201F201F20165
:10E7A000F201F2017002F201F201F2016702F201DC
:10E7B0006A02F201F10198F8012027685E2A07F148
:10E7C000010300F0F28108F10105002E00F01B8228
:10E7D00003222360F255226801322260626801320E
:10E7E000626098F801205D2A00F048824FF0000E28
:10E7F0005C2A00F06581002A00F04A8129464878A9
:10E800002D2800F0BC812068002E00F0C181451C3D
:10E81000256032542268501C20600878B0544A7831
:10E820005D2A01F101050EF1010EE1D14FFA8EF2E0
:10E83000724518BF49F001095FFA89F9002E3FF4CB
:10E8400056AF06F803E052E72268BA4200F0208192
:10E8500098F801103F2900F0C881002E00F0DE81F9
:10E8600045466221B1542268BF1A0132023FB754B3
:10E8700079B2B94218BF49F0010922685FFA89F9F3
:10E88000971C626827600132626030E72268BA42F2
:10E8900000F0FE8008F10105002E00F04181B81C57
:10E8A000D21BF119304437F0E9F9226802326021B5
:10E8B0002260B15420683A1A3044023A427020680B
:10E8C0000230206098F801004FFA82FC944518BF8E
:10E8D00049F001093F280CBF62226122F2552268EB
:10E8E00007F10101A2EB0702A2F10202725450B239
:10E8F00018BF45462768904218BF49F001095FFAE2
:10E9000089F9626802326260F1E698F801202768AE
:10E910003F2A00F06081A268531C5A0051B2914214
:10E9200018BF49F00109A3605FFA89F9002E00F0D1
:10E930006781791C21607E21F1552168481C206087
:10E94000725462680132626001220292019A03935A
:10E9500008F101002146FFF759FE0546002800F0A6
:10E9600097800278292A40F09380029B002B3FF485
:10E97000BEAE039B5A00013251B2914218BF49F01A
:10E9800001095FFA89F92168002E00F05681481CC0
:10E9900020607E2070542168481C20607254A3E6D9
:10E9A0002268571C2760002E3FF49DAE5121B154C0
:10E9B000276898E62268BA426AD008F10105002E5D
:10E9C00000F09C80B81CD21BF119304437F056F986
:10E9D00022680232226098F801203F2A0CBF62228E
:10E9E0006122F255226807F10101A2EB0702A2F1B0
:10E9F0000202725450B218BF4546904218BF49F007
:10EA0000010927685FFA89F96EE627687A1C226097
:10EA1000002E3FF468AE0222F25564E67C2A7FF4B1
:10EA200054AE2268BBF1000F38D0A2EB0B010139C4
:10EA300048B2884218BF49F001098EB306F80B109E
:10EA4000226806EB0A050AF102002946A2EB0A0237
:10EA5000304437F013F92368F11860200333236042
:10EA60008870D4F800B061220BF10101216006F832
:10EA70000A202268A2EB0A02023A51B26A7091425D
:10EA800018BF49F0010927685FFA89F9454638E758
:10EA9000002005B0BDE8F08F0026C2E5002ED0D1E1
:10EAA000171D02F1030BA7EB0A02023A51B2914281
:10EAB00018BF49F0010927605FFA89F9454620E748
:10EAC0006A7842F02000642805F101016BD042F021
:10EAD0002400772867D0A2F1610015280CD8DFE860
:10EAE00000F0AAA80B0B0B5E0B0B0B0B0B0B0B5CBC
:10EAF0000B0B0B5A0B480B600D467CE60232226072
:10EB0000D11B174698F8012002393F2A18BF454605
:10EB10004AB28A4218BF49F001095FFA89F9E3E570
:10EB2000111DC81BBA1A043A023821600F464FFA69
:10EB300080FC51B2844508BF914214BF01220022DB
:10EB400049EA02025FFA82F998F801203F2A18BFC9
:10EB50004546D6E6002E50D005222060F2552268A8
:10EB6000511C216098F80110B154BDE50B211170C2
:10EB7000BAE548782D284FF009027FF444AE887832
:10EB80005D283FF440AE20680231002E7FF43FAE96
:10EB90000230206043E60D2231E60A222FE60C22E5
:10EBA0002DE60B222BE600222DE6002E48D0042273
:10EBB0002360F2552268013222606268013262608D
:10EBC00098F802205D2A08F1020508BF4FF0000EF8
:10EBD0007FF40CAE32E698F802203A2A7FF49BAE1E
:10EBE000002308F102080293B0E608F101054EB3D4
:10EBF000612137E6BA1C226075E5BA1C226073E514
:10EC0000BA1C22609DE6626801326260BA1C226012
:10EC100098F801205D2A7FF4E9AD68E5BF1A023F4C
:10EC200079B2B94218BF49F0010945465FFA89F93E
:10EC300026E60822E3E50722E1E50231216053E5FB
:10EC40001A46B8E7B91A023948B2884218BF49F0E3
:10EC500001095FFA89F913E60D21117044E50921D4
:10EC6000117041E50C2111703EE50A2111703BE560
:10EC70000821117038E50721117035E54FF0000EBD
:10EC8000DFE500BF08B502F0C3F908B1012008BDF7
:10EC900002F0B6FB70B902F0E7FB68B9074B1868E1
:10ECA000C20705D4C303F1D4800C00F0040008BDF2
:10ECB000052008BD022008BD032008BDEC7401201A
:10ECC000034B53F8203013B19A6801329A607047B1
:10ECD0000C260120114B53F82000F0B10179427944
:10ECE0001F298ABF0E4B4FF0A04301F01F01D3F83C
:10ECF00010351F2A23FA01F38ABF09494FF0A041BA
:10ED000002F01F02D1F8101503F00103D1405B009F
:10ED100001F00101194366F0D1BB7047343C01207A
:10ED2000000300502DE9F04FABB0044603910020E2
:10ED3000214647F02DF8002800F0308301212046BD
:10ED40003DF0ACFC4268CDE90C4200230E938DF8F7
:10ED50006030082104A878F045FA0023CDE90A3391
:10ED6000DDE90C040EAB012218A9A0470E9B002B75
:10ED700040F02C83002800F06C819DF86090DFF853
:10ED8000F082DFF8F0B200263446B2464D46002D40
:10ED900000F066810EAB0C980D9F012218A9B847B0
:10EDA0000E9B002B40F0128308B98DF860007D2D7A
:10EDB00000F256815A2D40F25F815B3D222D00F218
:10EDC0004F81DFE815F036004D0123004D014D0164
:10EDD0004D014D014D014D014D014D01F6004D011B
:10EDE0004D014D014D014D014D014D01B2004D014F
:10EDF0004D014D014D014D016B004D014D014D0186
:10EE00004D014D014D0154004D012300002C00F037
:10EE100027810A9B002B00F0DC82013B0B9A0A93AE
:10EE200052F82340204641F079FB82469DF860501D
:10EE3000ADE70021084643F089F9054694B18A4BB5
:10EE40009A451DD0002E00F00B8131462A462046FF
:10EE500040F098FA0B9B0026CBB1214608A842F05F
:10EE600005FD284641F05AFB2C468246DEE700208D
:10EE700042F036FF0546002CF4D07B4B9A45E1D199
:10EE80002946204642F0F2FC0B9B002BE5D10121E4
:10EE900008A842F02FFD0B9B1C60E2E79DF8603054
:10EEA000722B40F0DD800EAB0D9D0C98012218A94D
:10EEB000A8470E9B002B40F08982002800F0CD80EF
:10EEC0009DF86030752B40F0CB800EAB0D9D0C98FB
:10EED000012218A9A8470E9B002B40F0778200283A
:10EEE00000F0BB809DF86030652B40F0B9800EAB20
:10EEF0000D9D0C98012218A9A8470E9B002B40F0ED
:10EF0000658208B98DF86000002C00F01C82564B19
:10EF10009A4500F02D82002E00F005823E223146F7
:10EF2000204640F02FFA002680E79DF86030752BD0
:10EF300040F096800EAB0D9D0C98012218A9A847B1
:10EF40000E9B002B40F04282002800F086809DF846
:10EF500060306C2B40F084800EAB0D9D0C9801222C
:10EF600018A9A8470E9B002B40F03082002874D0CF
:10EF70009DF860306C2B73D10EAB0D9D0C98012267
:10EF800018A9A8470E9B002B40F0208208B98DF8E5
:10EF90006000002C00F0CF81334B9A4500F0E381F4
:10EFA000002E00F0C2810E223146204640F0EAF9E0
:10EFB000B9E79DF86030612B52D10EAB0D9D0C98D6
:10EFC000012218A9A8470E9B002B40F0FF810028C2
:10EFD00043D09DF860306C2B42D10EAB0D9D0C9848
:10EFE000012218A9A8470E9B002B40F0EF810028B2
:10EFF00033D09DF86030732B32D10EAB0D9D0C9841
:10F00000012218A9A8470E9B002B40F0DF8120B3F6
:10F010009DF86030652B23D10EAB0D9D0C9801221D
:10F0200018A9A8470E9B002B40F0D08108B98DF895
:10F030006000002C00F08F810B4B9A4500F09D8101
:10F04000002E00F06E811E223146204640F09AF9D3
:10F0500069E78DF86000814691E600238DF8603005
:10F06000024873F07FFB00BF64720B00C08D0B0081
:10F070000020FF03011000043A2DF1D81F2D40F2AB
:10F080004A81A5F12002D2B20123934013EA080F6E
:10F0900040F0AB8013EA0B037FF4C8AE222DDFD122
:10F0A0009DF86010059335460029D9D022297BD0E0
:10F0B0005C2913D004A877F023FF0EAB0D9E0C98AB
:10F0C000012218A9B0470E9B002B40F07F8110B1A0
:10F0D0009DF86010E8E78DF86000C1E70EAB0D9E6B
:10F0E0000C98012218A9B0470E9B002B40F06E81AE
:10F0F00018B98DF860000146DCE79DF86010A1F1B9
:10F100006203132BD6D801A252F823F06DF102004E
:10F11000B5F00200B5F00200B5F0020069F102009E
:10F12000B5F00200B5F00200B5F00200B5F0020043
:10F13000B5F00200B5F00200B5F0020065F1020082
:10F14000B5F00200B5F00200B5F0020061F1020076
:10F15000B5F002005DF1020071F102000921A9E79A
:10F160000D21A7E70A21A5E70C21A3E70821A1E7C4
:10F170004FF0000904260EAB0C980D9F012218A930
:10F18000B8470E9B002B40F02181002840F0A3805F
:10F190008DF86000C923013E43EA0919EBD14946C5
:10F1A00004A877F0D7FE88E70EAB0C982E46012214
:10F1B0000D9D18A9A8470E9B002B40F0078108B9A8
:10F1C0008DF86000DDE9051043F06CF80246002C74
:10F1D00051D0834B9A4500F09780002E00F0878035
:10F1E0003146204640F0CEF89DE60023059399462F
:10F1F000294604A877F084FE9DF86050452D15D867
:10F200002A2D15D9A5F12B031A2B11D8DFE803F00D
:10F2100014101423101010101010101010101010D3
:10F22000101010101010101010102300652D12D0A7
:10F23000284673F04BF988B10EAB0C980D9F012254
:10F2400018A9B8470E9B002B40F0C0800028CFD1F2
:10F250008DF86000CCE74FF00109EDE70346DDE9EA
:10F260000510B9F1000F44D01A46009346F028F972
:10F270000246002CADD1914641F050F9039BDBB919
:10F280009DF8600073F04AF988B10EABDDE90C041B
:10F29000012218A9A0470E9B002B40F09780002860
:10F2A000EED18DF8600073F039F90028EDD19DF8AA
:10F2B0006030002B7FF4D4AEB9F1000F3FF4D0AE34
:10F2C0000A9B002B7FF4CCAE04A877F00BFF4846D6
:10F2D0002BB0BDE8F08F9DF8602042F02002A2F133
:10F2E0003003DBB2092B84BF573AD3B253E716463B
:10F2F0009CE50A224B4646F015FA0246002CBAD08D
:10F30000374B9A457FF469AF1146204642F0AEFA7A
:10F31000DFF8CCA08AE50A2D09D8082D3FF686AD86
:10F320009EE61E2682E53E2680E50E267EE50D2D14
:10F330003FF47CAD94E60E2041F0F0F8039B4BBB0C
:10F340004FF00E099CE73E2041F0E8F8039BCBB953
:10F350004FF03E0994E71E2041F0E0F8039BABB963
:10F360004FF01E098CE70E21204642F07FFACFE7CE
:10F370003E21204642F07AFACAE71E21204642F09A
:10F3800075FAC5E70A9B4FF03E099AE70A9B4FF0D2
:10F390001E0996E70A9B4FF00E0992E70FAA204636
:10F3A0007E2100260027CDE916673EF017FC0D4AA6
:10F3B0000D4B129201214022CDE913120CAC1AA977
:10F3C00012AACDE90C4315911192C2E4184673F0CC
:10F3D00071F9039BA146002B7FF476AF50E700BF85
:10F3E00064720B00F0650B00F51406000288112A08
:10F3F0000B4608D0362A0BD119B181889A899142DF
:10F4000008D0012070474FF6FF71012299811A74CC
:10F410000020704700B5C28883B0DA81C2890093AA
:10F4200000F110015868824228BF02461868019214
:10F4300036F0F0FBDDE90032012101209A601974F9
:10F4400003B000BDC207034620D400B510F003028C
:10F4500083B00BD1114A016891421AD0184641F08D
:10F460005DF85E22C1880E4873F070F9022AF5D16A
:10F470000C4A0240062AF1D040F05CFFFCEEC07A54
:10F48000CDED017A9DF8040003B000BDC0F3470044
:10F49000704741F01DF8C0B2F6E700BF3C710B00A9
:10F4A000D0990B00070080FF70B588B014460DF1AD
:10F4B0001E030DF11F02CDE900320E460DF11D03B2
:10F4C00007AA214604460EF031F99DF81C209DF84C
:10F4D0001D300B490592204604939DF81E409DF86F
:10F4E0001F503FF05BFC03903FF056FBCDE9004519
:10F4F000DDE90432039831465CF060FD08B070BD70
:10F500003CD80B002DE9F04F0446E3B0674812F0F9
:10F510003DFDB0F1000A21DB654E7388B3F57F7FB6
:10F5200080F0B2801A1DA2421CD85A1E341D6148B8
:10F53000A15C614D2F290BBF00230022A354E2548C
:10F5400005A92BF0CFFC286010B12BF0FFFD68B9A6
:10F5500040F251335046338062F0A0FF002063B088
:10F56000BDE8F08F012063B0BDE8F08F2868059AF0
:10F57000803006A97DF0A5FA0023C6E90133F360C7
:10F5800040F25113054644F8043C002840F08280C4
:10F590001AA906A87DF085FB044620B180E07DF025
:10F5A00080FB013428B99DF882301AA906A8002BE7
:10F5B000F5D1002106A802947DF073FB029BB36095
:10F5C000002B54D04FF0000B0DF18207D846CDF838
:10F5D0000CA01AA906A87DF064FBBDF87230BDF836
:10F5E0007010C6F804B003F01F0252000192480ADE
:10F5F000C3F344120092DB0A01F01F0200F2BC7058
:10F60000C1F343116EF0FAFA9DF874302B4A13F0EF
:10F610001003A0FB0202C6E9040214BF01231A9AD8
:10F62000F36018BF00223846B26169F083FA0546DC
:10F630007080039862F032FF95B10024A5EB040AB4
:10F64000BAF1040F28BF4FF0040A39191748CDF852
:10F65000008000235246544412F076FDA542EDD8B6
:10F66000029B0BF1010B9B45B3D1DDF80CA006A862
:10F670007CF04CFD0023B268738050467260F360EA
:10F68000B36162F00BFF69E740F25123338062F00F
:10F6900005FF63E703235046737062F0FFFE5DE7EA
:10F6A000294606A87DF0FDFAB560E0E72045012077
:10F6B00010480120144801209846012000CA9A3BB6
:10F6C00038B52B4A2B4B0446012110681D6857F0B2
:10F6D000C9FB294A02F1200C52F8043F13B11979F1
:10F6E000A14202D06245F7D138BDDA791ABB5A6916
:10F6F0009969AA1A411AC2EB02420A444FF6FF71F5
:10F700008A4228BF0A46D9891C8AA4B214FA81F118
:10F710009C89B1FBF4FC04FB1C119C6824F81120AB
:10F720001A8A998992B28A4218D21A8A01321A82A6
:10F730005D61986138BD1F2C88BF104A597994BF0C
:10F740004FF0A04204F01F04D2F81025E24002F06E
:10F7500001029142ECD00022DA71E9E7DA8992B233
:10F760000132B2FBF1F401FB1422DA81E0E700BFC1
:10F7700084760120BC7401200C0A01200003005093
:10F780002DE9F04110F8017C0578A7F10306B6FADF
:10F7900086F67609CDB18846841C06E000F01CF898
:10F7A00080B9013D04F102040FD014F8013C414638
:10F7B0002046002BF2D098F800209342F1D823780D
:10F7C0009342EED33046BDE8F081FE1E18BF0126FD
:10F7D0003046BDE8F08100BF03780A7843F020018D
:10F7E0006429C3F340101DD0732910D022F02001EA
:10F7F000413919290AD9A2F13001092906D96FEA3C
:10F80000531303F001035F2A18BF18467047202ADC
:10F81000FCD06FEA5313093A03F00103042A88BFAE
:10F82000184670476FEA5313303A03F00103092A70
:10F8300088BF1846704700BF2DE9F04F95B081464C
:10F8400000F15804D0E9140300AF5B6821469847E3
:10F85000D9F8583033B109F1080318463B6226F055
:10F8600035FE18B95437BD46BDE8F08F99F84810F9
:10F87000002940F0A381D9F80800002800F01C817D
:10F8800026F082FF8346002800F01681B9F8383050
:10F890005A2B6D4600F08F81B3F5877F00F08B8186
:10F8A000B9F836200732D210D31D23F00703ADEB91
:10F8B000030D0021684636F091FBD9F85430D9F891
:10F8C00050005B6821469847EA464FF001087D608A
:10F8D000C7F82C90386AC7F80CD007F1380259469F
:10F8E00026F0FEFC002800F0D680FB6A93F83A1060
:10F8F000072915D893F8443093B1B7F93C20082371
:10F90000B3FBF1F31A44013A92FBF3F212FB03F258
:10F91000BA87B7F9382092FBF3F202FB03F33B8777
:10F9200007F1380025F0E4FCFB6A786307F1380042
:10F9300093F83A402023B3FBF4F425F0FBFC054692
:10F9400007F1380025F0F6FCB0EBC41F4FEAC416EF
:10F9500000F2B980C5F34A1301339B007B61073382
:10F96000ADF5007D23F00703C7F828D007F1380074
:10F97000ADEB030DC7F810D025F0BAFC4FF40072C0
:10F980000123C7E90623844600253D63C7F808B074
:10F99000C7F824C07A6A786B398F3E69A7F844109B
:10F9A0000023521B92B2FB647B8F904203EB050154
:10F9B00088BF7A6AA7F8461098BF1B18B7F93C10A1
:10F9C000A7F848108CBF9B185B197A69A7F84A30D2
:10F9D0000021304636F002FBBC6ABA69002120469D
:10F9E00036F0FCFA23463246386A07F1440126F025
:10F9F000BBFCB7F94620B7F94A3094B29C423CDAD6
:10FA0000F96AB7F9440091F83A30B1F87660B1F884
:10FA10007410D7F828B006FB021113FB00F2002A7D
:10FA2000B8BF073201EBE201B7F94820121A03FB15
:10FA300002F2FB6A002A9B6DB8BF073201340B4407
:10FA40004FEAE209A4B2601EC0F3CC0200F0070046
:10FA50001AF8021008FA00F008430AF802005946A2
:10FA600018464A4636F0D6F8B7F94A10A14200EBDC
:10FA70000603CB4404F10104E5DC05F0A9FC73F0B6
:10FA80006BFF7A6B3B6B1544FA6901339A423B6317
:10FA900080D1D7F808B0DBF808B0D7F80CD0BBF1AC
:10FAA000000F7FF417AFD7F82C907D68D9E91403C5
:10FAB00051469B689847AD46386A26F065FC543736
:10FAC000BD46BDE8F08F07F1380025F0EDFCFA6A7D
:10FAD000B6FBF0F692F83A30002E57D0B1B2072BB1
:10FAE00079630CD892F844204AB9796B0822B2FBAA
:10FAF000F3F2B1FBF2F302FB03F39BB27B6307F17A
:10FB0000380025F0F5FB7D6BB0FBF5F307F138000D
:10FB10009EB225F0EDFB721CB0FBF5F303FB150361
:10FB200092B29BB2002B14BF11463146F96107F126
:10FB3000380025F0B9FC7B6B10FB03F39BB2B3FBE1
:10FB4000F4F204FB12340CB1013292B292005B0960
:10FB5000BA6101339A00BB697A61073323F0070366
:10FB6000ADEB030DD31DDB086A46A2EBC303C7F858
:10FB700028D007F138009D46C7F810D025F0B8FB13
:10FB8000FB698446002B7FF4FFAE84E7072B06D881
:10FB9000FA6A92F8442012B901227A63A5E707F1C4
:10FBA000380025F0A5FBF86107F1380025F0A0FB2F
:10FBB00001237B63BBE7B9F8342073E60023C9F85F
:10FBC000303009F1280B61E62DE9F04F00F1080B08
:10FBD00093B0814602AF584626F078FC18B94437F6
:10FBE000BD46BDE8F08F99F84810002940F04C81DF
:10FBF000D9F80800002800F0D68026F0C5FD84461C
:10FC0000002800F0D08009F1B2037B60C7F81CB077
:10FC1000C7F808C0B968F86907F128026D4626F0F0
:10FC20005FFB002800F0B68007F1280025F060FB9C
:10FC3000044607F1280099F83A8025F07BFB99F8F3
:10FC4000822083B2002A00F0B780C4F3CF027A6129
:10FC50004FF40072BA6108245B0901339A00BB6952
:10FC60003A61073323F00703ADEB030DD31D23F0F7
:10FC7000070302AEADEB030D02AB07F12800FB60FA
:10FC800025F036FB7B698646002B00F003814FF0A0
:10FC9000000A3D60D04609F1500B3546C7F820E018
:10FCA00049E025F047FB99F83A60F60816FB00F6A4
:10FCB000B3B27B62D7E903620021304636F08EF999
:10FCC000BA690021284636F089F93246FE692B468A
:10FCD00007F13401304626F047FB584607F134025D
:10FCE000314626F08DF9584626F0E0F8002861D01C
:10FCF00099F8801041B90123D9F8500000931A46B1
:10FD0000D9F860607B68B0477B6AD9F850000093EF
:10FD100000222B460121D9F86060B047584626F0F2
:10FD20005DF905F055FB73F017FE7B6908F10108DA
:10FD30004345A2442AD0798D3B8DBB860AEB010254
:10FD4000FA863A6AB7F92C603E87A2EB0A020023D2
:10FD500092B2A242FB6301EB0403534499F83A20A8
:10FD60003CBF3B6ACB18072A07F134007B8798D841
:10FD700007F1340025F0DEFA99F83A300822B2FB98
:10FD8000F3F3B0FBF3F6B3B27B6293E73D685846FA
:10FD900026F028F9BB689B68BB60AD46002B7FF45A
:10FDA00039AFD7F81CB0584626F0EEFA4437BD46B6
:10FDB000BDE8F08F3D68EDE707F128007B6225F094
:10FDC000B9FA2026B6FBF8F6B0EBC61F7B6A4FEAFD
:10FDD000C61818D85B0901339B003B610733ADF5AA
:10FDE000007D23F0070302AEADEB030D02AB07F17C
:10FDF0002800FB6025F07CFA01234FF40072C7E96C
:10FE00000532864643E707F1280025F04DFB99F8B7
:10FE10003A20B8FBF0F000283FD0072A84B20AD875
:10FE200099F844303BB90823B3FBF2F2B4FBF2F388
:10FE300002FB03F39CB207F1280025F059FAB0FB4E
:10FE4000F4F307F1280099B2796125F051FA796944
:10FE5000B0FBF4F34A1C03FB140392B29BB2002BD9
:10FE600018BF1146796107F1280025F01DFB10FB32
:10FE700004F39BB2B3FBF6F206FB12360EB101326D
:10FE800092B29200BA61E7E60023C9F8303009F176
:10FE9000280CB8E609F1500B79E7072A02D899F83F
:10FEA000443053B107F1280025F022FA786107F1B8
:10FEB000280025F01DFA0124D5E70124B3E700BF8F
:10FEC0002DE9F043884690F82A1011F0100785B00C
:10FED0006BD14368DB68044653F8281040F21A508F
:10FEE00045F056FF064600285DD06368DB6853F88E
:10FEF000280073689847B36801A95B6881469847F2
:10FF0000B36839469B68054648469847B368394602
:10FF10009B694846984763682549DB6853F8280081
:10FF20003EF03CFF064668B190F8503023F01003D5
:10FF300001A980F8503027F003FB00210546304628
:10FF400027F0C0FE63681B49DB6853F828003EF0C9
:10FF500025FF064668B190F82A3023F0020301A974
:10FF600080F82A3026F0BAFB00210546304626F0FC
:10FF7000C7FE7DB194F82A30DB070ED504F11802D4
:10FF800001A9104625F042FA94F82A3043F0010303
:10FF900084F82A3005B0BDE8F08304F1180101A807
:10FFA00025F068F9F0E70546B5E70CF021FD00BF44
:10FFB00040FD0B000CFB0B0070B586B005460191AF
:10FFC000164619F0C7FA90B9019840F02DFA0622AA
:10FFD000044603A930463CF0EBFA03AA2146284622
:10FFE00019F0CEFA002804DB0E2006B070BD5FF0D9
:10FFF00067F8404272F05EFB70B586B0054601912D
:020000023000CC
:10000000164619F0A7FA90B9019840F00DFA0522AA
:10001000044603A930463CF0CBFA03AA2146284601
:1000200019F00AFB002804DB0E2006B070BD5FF05B
:1000300047F8404272F03EFB242B2DE9F0478846FA
:1000400001D8012B06D1FCF7AFFB1623036000207B
:10005000BDE8F087344E0D46294615F8014B375D53
:1000600017F00807F8D12D2C10D12C7801278D1C02
:1000700033F0100115D1302C0DD1297801F0DF01BA
:10008000582908D16C78023510230AE02B2C04BFC4
:100090002C788D1CECE7002BF6D1302C14BF0A23F2
:1000A000082307F1004E0EF1FF3E0021BEFBF3F9DD
:1000B0000E4603FB19EAA4F1300CBCF1090F10D86D
:1000C0006446A3421EDDB1F1FF3F07D0B14516D310
:1000D00001D1A24513DB06FB0346012115F8014BB4
:1000E000E9E7A4F1410CBCF1190F01D8373CE8E76E
:1000F000A4F1610CBCF1190F04D8573CE1E74FF0B3
:10010000FF31EBE74B1C05D122230360764632B961
:1001100030469DE707B17642002AF9D009B105F1D2
:10012000FF38C2F80080F3E76D860C002DE9F0433C
:10013000344E86460D46284615F8014B375D17F0BC
:100140000807F8D12D2C10D12C780127851C33F00D
:10015000100015D1302C0DD1287800F0DF00582880
:1001600008D16C78023510230AE02B2C04BF2C78C0
:10017000851CECE7002BF6D1302C14BF0A23082392
:100180004FF0FF380026B8FBF3F803FB08F96FEADD
:1001900009093046A4F1300CBCF1090F10D86446AF
:1001A000A3421EDDB6F1FF3F07D0804516D301D133
:1001B000A14513DB00FB0340012615F8014BE9E7DD
:1001C000A4F1410CBCF1190F01D8373CE8E7A4F1C8
:1001D000610CBCF1190F04D8573CE1E74FF0FF3632
:1001E000EBE7731C06D12223CEF80030304632B93B
:1001F000BDE8F08307B14042002AF9D006B1691E7C
:100200001160F5E76D860C00F0B583B004460D462D
:1002100001926AF03DFF6368019A07460120587217
:1002200060680E46294657F04DF8134B984204D0AB
:10023000636800225A7203B0F0BD17F57A7546F173
:10024000000605E06AF024FF854276EB01010CD33D
:1002500063685A7A002AF5D19B7A042B96BF074A25
:10026000074852F8230003B0F0BD63680548002238
:100270005A7203B0F0BD00BF0000AD0B48C80B00C0
:100280000100AD0B0700AD0BF8B543689A6852B397
:10029000054600240BE073689847B36805F1080130
:1002A0009B6898476B689A68013494421BD2DB685C
:1002B00040F21A5053F8241045F06AFD6B68DB6871
:1002C0000646A70053F82400002EE4D10D493EF065
:1002D00065FD48B105F1080127F0F4FC6B689A68E8
:1002E00001349442E3D3F8BD6B680749DB68D85901
:1002F0003EF054FD0028D5D005F1080126F000FDA0
:10030000D0E700BF40FD0B000CFB0B0090F9503014
:100310002149B0F90C2000B5002B836AB4BFB0F8B6
:1003200012C0B0F810C0002B08BF0B469444997B54
:1003300092B2C1B193F9051011FB02F259880A4437
:1003400012B2A0F8462093F90510B3F802E011FBB1
:100350000CE31BB29A42D2BFA0F84A30A0F84A2060
:10036000A0F8463000BD93F9041011FB02F2198881
:100370000A4412B2A0F8442093F90410B3F800E044
:1003800011FB0CE31BB29A42D2BFA0F84830A0F890
:100390004820A0F8443000BD1C03012090F95030E3
:1003A0002149B0F90E2000B5002B836AB4BFB0F824
:1003B00010C0B0F812C0002B08BF0B469444997BC4
:1003C00092B2C1B193F9041011FB02F219880A44E8
:1003D00012B2A0F8442093F90410B3F800E011FB26
:1003E0000CE31BB29A42D2BFA0F84830A0F84820D4
:1003F000A0F8443000BD93F9051011FB02F25988B2
:100400000A4412B2A0F8462093F90510B3F802E0AE
:1004100011FB0CE31BB29A42D2BFA0F84A30A0F8FD
:100420004A20A0F8463000BD1C03012010EE102A1F
:1004300022F00043B3F17E5F05D34BD1002A71DB7C
:100440009FED5C0A7047B3F17C5F05D2B3F14A5F60
:1004500047D89FED590A704700B5002A83B0F7EEE0
:10046000007A62DB77EEC07AB6EE007A67EE877AC2
:10047000F5EE407AF1EE10FA00F18580B1EEE76A10
:10048000DFED4E6A9FED4E5A9FED4E7A9FED4E4A3C
:10049000A7EEA65A16EE103A6FF30B03A7EE857A75
:1004A00006EE903AF0EE674AF7EE005AE7EE845A0D
:1004B000E6EEE64A36EE865A67EE277A84EE850A3D
:1004C00087EEA57AA7EE060A30EE260A30EE000A7D
:1004D00003B000BD70EE407A9FED367A87EE270AB2
:1004E000704760EE006A9FED356ADFED357A9FED6B
:1004F000357AE6EE867A9FED346AA6EEA77AF7EEB5
:10050000005AE6EE865A27EE267ADFED2B7AC7EE02
:10051000256A9FED2E7AA0EE667A30EE470A37EE16
:10052000C00A70479FED2A0A704730EE270AF6EEA0
:10053000007A60EE277AF5EE407AF1EE10FA2DD4CB
:10054000F1EEE75A9FED1D6A9FED1D7ADFED1D6A02
:100550009FED1D5A9FED180AA7EE867AB7EE006A46
:10056000E7EE876AA7EE856A66EEA77AC7EE866A27
:10057000DFED187AE6EEA57A77EEA57A30EE670A17
:1005800030EE000AA4E7B0EE670ACDED017A66F01E
:1005900071F9DDED017AB0EE406A71E7B0EE670AFD
:1005A000CDED017A66F066F9DDED017AF0EE405AA4
:1005B000C8E700BF00000000DA0FC93F6BD30DBCD5
:1005C000BA132FBD75AA2A3EAEE534BF6821A23307
:1005D000DA0F49406821A2B300B510EE103A5A0074
:1005E00083B0F0EE407A26D523F00043B3F18B4F71
:1005F00007D333F0FDFBDFED267A30EE270A03B098
:1006000000BDBFEE000AA7EEA70A77EEA76AB5EE17
:10061000400AF1EE10FA24D4B1EEC07A77EE877A70
:10062000B7EE007A87EE270A36EEC00A03B05DF80F
:1006300004EB33F0DDBBB7EE007A70EE477A37EEAD
:10064000A77AA7EEA77AB5EE407AF1EE10FA15D4A4
:10065000B1EEC70A37EE800A03B05DF804EB33F061
:1006600011BBCDED017ACDED006A66F003F9DDED49
:10067000017ADDED006AB0EE407ACFE7B0EE470ACE
:10068000CDED007A66F0F6F8DDED007AE2E700BF26
:100690001872313F30B5084687B011461A460F4BE5
:1006A0000DF10C0CCDE9003C032336F0C3FB0C49E3
:1006B000039C0C2041F018FA9DF8102021460546B5
:1006C0000CF0E4FD9DF8143013B9284607B030BD96
:1006D00028460CF0FDFD284607B030BD80D60B0043
:1006E000F8D60B0000B583B001900CF0D3FD019853
:1006F00003B000BD08B508680CF016FE0E2008BD5A
:1007000010B58EB003AB51F8044B0193184B009316
:100710000138032336F0E6FA606840F23B5106AA3E
:100720003DF05CFA227A049B039C0994520042F04B
:1007300001020892059A6FF000415B0040F6261016
:1007400043F001038A420A900B930ED0520040F20C
:10075000E64342F00102CDE90C32022106AA022052
:1007600038F062FA0E200EB010BD0121F6E700BF8E
:1007700098D60B0010B58EB003AB51F8044B019323
:10078000184B00930138032336F0ACFA606840F24E
:100790009E6106AA3DF022FA227A049B039C0994EA
:1007A000520042F001020892059A6FF000415B008E
:1007B00040F6261043F001038A420A900B930ED0B4
:1007C000520040F2E64342F00102CDE90C32022130
:1007D00006AA022038F028FA0E200EB010BD012122
:1007E000F6E700BFE0D60B0030B597B002AB51F88A
:1007F000044B01932F4B00930138062336F072FA15
:10080000606840F29F6108AA3DF0E8F9049B227AF3
:10081000029C0B945B0043F0010352000E93059B76
:1008200042F001026FF0004144F6F6500A928B420A
:10083000039A0D900C9234D05B0044F6C65143F0FD
:1008400001030922CDE90F134FF00B0E4FF00A0CF4
:1008500014460321069B0DEB82000DEB8C0C5B0014
:1008600043F00103079A44F296250562CCF8203044
:100870006FF000439A420DD00DEB8E0E0DEB840409
:10088000520042F00102013144F26623CEF82030DA
:10089000C9B2E26208AA032038F0C6F90E2017B0E8
:1008A00030BD07224FF0090E4FF0080C144602210C
:1008B000D0E700BFB0D60B0010B508468EB0114689
:1008C0001A46174B0DF11C0CCDE9003C072336F0FE
:1008D000B1FADDE90740134940F2173236F002FC65
:1008E00008980E2803D00022012113F047FA0E4980
:1008F000182041F0F9F89DF834209DF8303005902B
:10090000CDE902329DF82C200A9B2146CDE9003228
:100910009DF82430089A0CF017FD05980EB010BD14
:1009200084D70B00D0F60B00BCD70B000CF01EBD1B
:1009300008B508680CF06AFD0E2008BDF0B5054644
:1009400085B001F134000E4604F0A6FC2B88102B74
:100950002FD0112B2AD10022A888424C134634F8FC
:100960001210814202F1440203D00133052BF6D16B
:10097000042303EB031304EBC3013B4801930091F1
:1009800007F0B4FD019B00994FF6FF7224F8332065
:10099000CB6D00220E2B81F85A2002D05A602A7AA1
:1009A0001A720023B361012005B0F0BD002005B02C
:1009B000F0BD00222B4C13464FF6FF7034F8121096
:1009C000814202F1440203D00133052BF6D1042306
:1009D00003EB0312D700A888E05304EBC202002007
:1009E00082F85A00A2F876000E20D065E87B0092CB
:1009F00019010B44022804EBC30314BF96F8450009
:100A00000120D87007F108004FF000024FF6FF7187
:100A1000204483F87820A3F8581083F8792009F04F
:100A200063FC07F16000009A0F49204407F034FD91
:100A30000023B3612869696907F16C03234403C388
:100A400002A860F0A3FFBDF808302A8A9A4202D8B3
:100A50006A8A9A4203D2A88802A960F07FFF002325
:100A6000F360A0E7A00A01203513050038B503881C
:100A7000102B0C4618D0262B2ED11A4B1878FF2895
:100A800010D060F065FF21460546174807F02EFD9F
:100A90000023E36084F8443035F00803284601D091
:100AA0000BF0FCFE012038BD81880022032060F09D
:100AB0007BFF0C4B1878FF280ED060F049FF2146D1
:100AC0000546094807F012FD0023E36084F844302E
:100AD00035F00803284601D1002038BD0BF0DEFEBA
:100AE000FAE700BFA70601206D0A030030B587B002
:100AF000044615460846052269463BF059FD03A900
:100B0000062228463BF054FD0199049A204674F0D1
:100B1000CBFEDDE90012039835F07CF82046DDE9D4
:100B200003120CF0F1FF0E2007B030BD30B587B0D6
:100B3000044615460846052269463BF039FD03A9DF
:100B4000062228463BF034FD0199049A204674F0B1
:100B5000ABFEDDE90012039835F05CF82046DDE9D4
:100B600003120CF0E3FF0E2007B030BD90F80C012B
:100B7000400040F0010070472DE9F04108468CB07C
:100B800011461A46254B07ACCDE90034052336F053
:100B900051F90522079804A93BF00AFD059EA6F12C
:100BA0001002102A37D81E4BD340DB0733D5089DDF
:100BB000022D20DD062D20D10998049F20B104A923
:100BC00001223BF0F5FCE8B980460A98C0B13FF03D
:100BD0007FFC044613494FF48A7040F085FFCDE94D
:100BE000005443463246394603900CF06BFF03989D
:100BF0000CB0BDE8F081002DDEDC0B4871F046FD45
:100C00000446E7E705984FF4B772102136F07EF9F5
:100C1000DDF81080D9E7054871F0A4FD70D90B000C
:100C200001010100A8D90B0068A00B00C0A30B00B4
:100C300070B551F8043B88B01D4603AB0193184BC7
:100C400000930138022336F04DF80522039805A9D8
:100C50003BF0AEFC069CA4F11002102A1CD8114BEC
:100C6000D340DB0718D5DDE9040620B105A9012230
:100C70003BF09EFC40B903462846224631460CF024
:100C800067FF0E2008B070BD06984FF4B7721021B0
:100C900036F03CF9059BEFE7034871F063FD00BFB8
:100CA00098D90B0001010100C0A30B0010B5044648
:100CB00008463FF0B9FB022807DD062807D10146A8
:100CC00020460CF061FF0E2010BD0028F7DC014823
:100CD00071F0DCFC68A00B0030B5114B87B005AD9E
:100CE000CDE900350446012300200D4635F0FAFF1A
:100CF0002946204674F028FF059840F071FD421007
:100D000004D0084840F20F5171F0C8FC2946204633
:100D100004AB03920CF0EEFF039903487DF007F853
:100D200058DA0B00ECAB0B00D4690B0010B90E23A2
:100D30001846704730B50D4683B0044674F004FF82
:100D4000294620460CF042FF0022019046F656014B
:100D500004483DF0D5F8019B00B14360184603B04C
:100D600030BD00BF6C000120E0B130B50F4BDFF8A3
:100D700040C01C780439002201E090420FD051F8A5
:100D8000043F9D0702F10102F7D11D686545F4D1CA
:100D90005D6895F804E0A645EFD1184630BD0E23F6
:100DA000184630BD0E231846704700BFBC7B01209B
:100DB00018DB0B0010B5084688B011461A46104BD8
:100DC0000DF1100CCDE9003C042336F033F8049803
:100DD00040F2FB4174F074FE0A4904460C2040F0D6
:100DE00083FE9DF81C2000929DF818309DF8142079
:100DF000039021460CF038FF039808B010BD00BFE7
:100E0000F8DA0B0018DB0B0008B50CF041FF0028E6
:100E100008BF0E2008BD00BF08B50CF03BFF00283E
:100E20000CBF1E203E2008BD08B5054B1A7802B144
:100E300008BD20F0A7F9024B01221A7008BD00BFBF
:100E4000837B01200E4A0F49506810B50E4C0023D9
:100E5000C008C4E9001310D00C49D26891F800E032
:100E600002F1040C01E0834207D05CF833201179D1
:100E7000714503F10103F6D16260034810BD00BF64
:100E800068C90B0018DB0B00A0460120BC7B0120C9
:100E90002DE9F041184F194E00240125D6E9000133
:100EA000D7E90032A4F1200CC4F1200805FA0CFCAB
:100EB00025FA08F803430A434CEA080C05FA04F142
:100EC0000B4002EA0C021343E0B207D05FF028FCAB
:100ED000204654F081FE204654F0B6FF0134402CE9
:100EE000DCD1074900220023C7E90023C6E900231B
:100EF000C1E90023BDE8F0815011012060110120FB
:100F0000E8110120002975D02DE9F04F3A4B1C68FB
:100F10005E683A4B87B0D3E90098394B00940025BE
:100F20001C680194043ACDE90255CDE904505F688C
:100F3000344C02EB81014FF0FF3C4FF0010E01E019
:100F400091422CD052F8043F9807F9D11868A0427A
:100F5000F6D1586893F808B090F804C0ACF12000BE
:100F6000CCF1200A2EFA0AFA0EFA00F040EA0A0042
:100F70000EFA0CFABBF1000F2FD049EA0A0948EA31
:100F80000008CDF808B05B7A002BD9D0019D0493FE
:100F900045EA0A059142019547EA0007D2D1DDE909
:100FA00004501DB1164B019AC3E90027039B1BB1E6
:100FB000114B009AC3E90026029B13B10F4BC3E902
:100FC0000098BCF1FF3F05D078B10F490F4A0023CC
:100FD0000B60137007B0BDE8F08F009D45EA0A056D
:100FE0000095012506430395CDE707B0BDE8F04F16
:100FF00020F0C8B8704700BF6011012050110120D7
:10100000E811012018DB0B00EC740120837B012028
:10101000054B1B78012B01D000207047034B18783B
:10102000FF3818BF01207047BD7B0120BC7B012029
:1010300008B500F009F8FFF72BFF00F0D5F9BDE87F
:10104000084000F00DBA00BF10B5124C124A2368D8
:101050006FF3172393421CD04FF4807200210F4886
:1010600034F0BCFF0E490F4B00220A701A704FF08B
:1010700080404FF44031130103F180430132082ACC
:10108000C3F80419F7D1044B4FF47C12C0F884293B
:10109000236010BDB87B0120AF0000ADC07B0120F4
:1010A000BD7B0120BC7B0120002A75D070B51446A1
:1010B0008A0788B005460B4603D1464A0968914223
:1010C00030D028462E6801930CF042FE019A01466A
:1010D000002330463BF0A6FA042C064615D02046E5
:1010E0003FF0A2F94223FF220021044635F0FEFE24
:1010F000012305AA314628468DF814400CF02CFE39
:10110000002846D00E2008B070BD014601232846B5
:1011100005AA0CF00DFE9DF81400400040F00100FF
:1011200008B070BD01930CF013FE019902AA45F0BE
:10113000C9FD002844D0DDE90232042CA2EB0306ED
:101140002FD0A3072AD12368234A934208D0234AE9
:10115000934205D0224A934202D0224A93421DD1A3
:10116000052205A920463BF023FA069BB3422DD168
:101170009DF81C10059C0022402035F0E9FF012855
:1011800021D102993346224628460CF0E5FD00287D
:10119000B8D1154871F0B2FA10467047134871F093
:1011A00075FA304632F018FF02990446024633467B
:1011B00028460CF0BDFD2146304640F0CFFCA2E7AA
:1011C0000B4871F063FA0B4871F0CCFA0A4871F0E1
:1011D000C9FA00BFC4790B0074650B00F0650B0001
:1011E000A8650B00907C0B00C09D0B002C9B0B0096
:1011F00060900B00DCA80B0010A00B0010B504469B
:1012000008460CF0A5FD042C09D0052C01D00020C7
:1012100010BD064B03EA400040F0010010BD80B253
:1012200000280CBF1E203E2010BD00BFFEFF0100A5
:10123000F0B1DFF84CC00439002351F8042F12F04C
:10124000030F03F1010311D110B4146864450AD0EF
:10125000984210D051F8042F940703F10103F7D1FD
:1012600014686445F4D1104610BC70479842E4D12C
:101270000E22104670470E22104610BC704700BF69
:1012800074DB0B0038B5084BD3E9004554EA05037D
:1012900005D019F04DFF201A65EB010138BD4FF064
:1012A000FF30014638BD00BF1012012010B52DEDF2
:1012B000028B08468AB011461A46334B05ACCDE97D
:1012C0000034022335F0B6FDDDE90504B0F10E026D
:1012D00018BF0122B4F10E0318BF01239A424DD06A
:1012E0000E2848D03FF026F8B0EE408A19F020FFD3
:1012F000F6F716FE9FED257A06EE900A0E2CC6EE46
:10130000877A25D040F2AD310698CDED037A35F0DD
:10131000D3FE04465FF0E4FD07A967F023FD9DF8C6
:1013200022009DF821109DF820309DF81F20CDE966
:1013300000109DF81E10BDF81C006CF035FD231A3E
:1013400008EE103ADDED037AB8EEC88A38EE278A47
:10135000B4EEE78AF1EE10FA13D40D49082040F0FC
:10136000C3FBB0EE480A04460CF008FD20460AB064
:10137000BDEC028B10BD9FED078AB7E7064871F000
:10138000F1F9064871F0EEF964DB0B0000007A44D5
:1013900074DB0B0000000000A89F0B00CC9E0B002C
:1013A00008B50CF0EFFCB4EE400AF1EE10FA08D6E6
:1013B00010EE103A23F0030040F00200A0F1FF40CD
:1013C00008BD014808BD00BF02004000704700BFD3
:1013D0000349044A0A6000234B600846704700BF77
:1013E000A046012074DB0B0008B501205BF0E4FB94
:1013F000024B00200021C3E9000108BD10120120AA
:10140000034B1878A0F10200B0FA80F04009704751
:10141000BD7B012010B5084686B011461A460C4B1C
:101420000DF1140CCDE9003C012335F003FD0598C6
:1014300040F2FB4174F044FB06490446082040F0AA
:1014400053FB214603900CF0A1FC039806B010BD9D
:10145000B0DB0B00B8DB0B00406870470E20704714
:10146000704700BF704700BF0020704710B5094BA0
:10147000094C1B680BB1A34208D1C02200210748C8
:1014800034F0ACFD40F8044C043810BD044871F051
:1014900035F900BFB84C012038770B00BC4C012057
:1014A000989E0B0010B5094B094C1B68A34203D052
:1014B00013B1084871F022F9B4220021064834F033
:1014C0008DFD054B43F8044C181F10BDC80D0120BD
:1014D00038770B00909E0B00CC0D0120164B01229B
:1014E000002186B0C3F80025C3F81011D3F81011FD
:1014F00001910199DA60D3F81021002AFBD0002273
:10150000C3F81021D3F8101105910599C3F80421EF
:10151000D3F8041104910499C3F80821D3F80811F1
:1015200003910399C3F80C21D3F80C11029102998D
:10153000C3F8002506B070470070004008B50CF0F5
:1015400061FC0E2008BD00BF10B582B008461146F0
:101550004FF00212019335F08BFB019B18680CF0E1
:1015600005FD06490446082040F0BEFA21460190D8
:101570000CF028FC019802B010BD00BFF4DB0B009A
:1015800010B504460CF05EFCC8B920460CF060FCB7
:10159000B5EEC00AF1EE10FA0DD9B4EE400AF1EE44
:1015A00010FA0AD610EE103A23F0030040F00200C1
:1015B000A0F1FF4010BD0E2010BD024810BD5DF02F
:1015C0007FFD00BF0200400010B504460CF03AFC5D
:1015D00030B920460CF042FC400040F0010010BD44
:1015E0005DF06EFD08B50CF0CDFC0E2008BD00BF0F
:1015F00010B582B0084611464FF00212019335F043
:1016000037FB019B40F2FB41186874F059FA064918
:101610000446042040F068FA214601900CF0AAFC30
:10162000019802B010BD00BF60DC0B0030B583B084
:1016300004460D460CF0A8FC80B9019028463EF007
:10164000F3FE0199A2234FF6FF7235F04FFC81B2F1
:1016500020460CF09BFC0E2003B030BD5DF030FD49
:101660002DE9F04F2DED088B804B8FB009ACCDE903
:101670000034052335F036FB0021099850F0E6FDD3
:10168000002107460A9850F0E1FD054600210B981D
:1016900050F0DCFDEB790290012B40F0E380C37940
:1016A000012B40F0DF80AA68012A40F2DB808368CA
:1016B000012B40F2D7809A4240F0D4806621B8686E
:1016C00053F008F9EC6929798146204650F004FF6F
:1016D000AB68A8692979013B00FB0340F0EE408A22
:1016E00050F0FAFE0C98029B0E28DC69B0EE40AA7E
:1016F00000F0A2803EF01EFE0D980E28B0EE409A3B
:1017000000F0A4803EF016FEF0EE409ABB68C3B332
:10171000EB690493029BD7F81CA0DB69D9F81C6025
:1017200003934FF00008BB46CDF81C900EE0B4EEDA
:10173000C0AAF1EE10FA2AD5F0EE697AE6EC017A49
:10174000DBF8082008F10108424518D950469BF8FB
:10175000041050F0C1FEDBF81820F4EEC08AF1EE60
:1017600010FAB0EE408A9244E1DDF0EE497AE6EC00
:10177000017ADBF8082008F101084245E6D8DDF8D7
:101780001C9048460FB0BDEC088BBDE8F08FAC68EC
:10179000013C012C27464FF000091ED9CDE90586F2
:1017A0002E46049D04E0A7EB0804012CC14610D985
:1017B000B0693179640804EB090800FB085050F067
:1017C0008BFEB4EEC80AF1EE10FAECDB012C4746B2
:1017D000EED83546DDF81480069E049CA869297968
:1017E00000FB094050F078FEA869297900FB07400A
:1017F000F0EE40BA50F070FE029C039BA069217984
:1018000000FB0930F0EE40AA50F066FEA069039A92
:10181000217900FB0720B0EE40BA50F05DFE38EEB3
:101820006B8A30EE4B0A7AEEEBAA28EE008AC8EEFD
:101830002A7A77EE8B7A81E72046197950F04CFEB0
:101840000D980E28B0EE409A7FF45CAF029A906833
:1018500093691179013803FB004050F03DFEF0EE32
:10186000409A53E7024870F07DFF00BF8C480C009F
:10187000E4930B002DE9F0472DED068B5D4B88B00E
:1018800005ACCDE90034032335F02CFA059800218E
:1018900050F0DCFC8368012B75D9C579012D044615
:1018A00040F0A580007950F0B5FD07460698E6693E
:1018B0000E286ED0002150F0C9FCC579012D81465B
:1018C00040F09280A26883689A4240F08D8000794F
:1018D00050F0A0FD80463046D9F81CA0B847A36957
:1018E00003935046B0EE408AC047A368012BF0EE48
:1018F000408A74D9039B9FED40AA1E44D9F8183042
:101900009A443046B847A3695046B0EE489A1E4400
:10191000B0EE408AC047F0EE689A38EE099A70EE51
:10192000699AF0EE4A6A07EE905AD9EE896AA3687E
:10193000D9F81820B8EE677A0135C6EE877AAB423F
:101940009244F0EE408A3AEE27AADAD8F6EE007A10
:101950002AEE27AA013B07EE903AF8EE677A67EE87
:101960008A7AF4EE677AF1EE10FA3BD617EE903AE7
:1019700023F0030040F00200A0F1FF4008B0BDECEE
:10198000068BBDE8F0871D4808B0BDEC068BBDE8AE
:10199000F0870798DFED188A3EF0CCFC3046B0EEB9
:1019A00040AAB847A368012B16D92A462179E069D5
:1019B000B0EE408A50F04CFD07EE905A30EE088AA7
:1019C000B8EE677A38EE688AA368C8EE077A013500
:1019D000AB4278EEA78AE8D82AEE28AAB6E79FEDB0
:1019E00006AAB7E70648C9E7064870F0BBFE0648F6
:1019F00070F0B8FE74480C00000000000200808007
:101A000002004000248D0B00188D0B001E280ED004
:101A10003E280CD010F001030AD110F0030209D1C6
:101A20000168094A914208BF012318467047012303
:101A300018467047022AFBD16FF3D600831F18BFE8
:101A400001231846704700BF3C710B0010B5426877
:101A5000FF2A82B004460B460ED9D4E90221207930
:101A600036F02AF9D4E901320E200132A3F5807351
:101A7000C4E9013202B010BD019100220179402079
:101A800035F066FB0246D4E90210083102FB01F191
:101A9000009232F0E7FA009AA168D4F804C0E0603E
:101AA00001FB02210844082161F31F2CC2EBC20292
:101AB000C4F804C0002134F091FA019BCDE700BFC7
:101AC0002DE9F04313468BB005460C46242820D858
:101AD000DFE800F024242424241F1F1F1F1F1F1FC2
:101AE0001F1FA61F131F1F1F1F1F1F1F1F1F1F6743
:101AF0001F131F1F1F1F1F1FB30013F0010240F011
:101B0000B18013F0030104D1B24A1868904200F08A
:101B1000A980002420460BB0BDE8F0830979039327
:101B2000002201F07F01402035F012FBE368AA4A51
:101B300021681E46A3689946237991429846074634
:101B4000039B00F0F3801846012207A93AF030FD0C
:101B5000002800F0828008F07F03012B099A00F032
:101B6000EB805A2B94BF20330020012A00F0C18063
:101B70005A2A00F317812032934240F0B08023F0BC
:101B80000203642B00F0AB80089B009309FB07F273
:101B9000079B3146284644F0BFFF00285DD03E2415
:101BA000B8E78D4D0A68AA42B3D0097903930022A1
:101BB00001F07F01402035F0CBFAA268E36802FB18
:101BC00000F8227902F07F062268AA421F46039B92
:101BD00000F0BB80184607A905223AF0E9FC002274
:101BE0003146402035F0B4FAA168089B05463046DE
:101BF000B3FBF5F31944039300F02AFA044639467F
:101C00004246C06834F006F8E068039B079903FB7E
:101C100005F2404433F0FEFF20460BB0BDE8F083F0
:101C20006D4A096891423FF474AF1946204600F0AE
:101C300047F920460BB0BDE8F0831846012204A9FD
:101C400003933AF0B5FC039B00283FD014F0030245
:101C500003D1624B216899424FD01E2420460BB01D
:101C6000BDE8F08318463EF0DFFB2179002201F049
:101C70007F018146402035F06BFAE3682668A16851
:101C800022799846544B9E4201FB00F700F0848075
:101C9000102D60D009FB01F102F07F0000F0D8F9AF
:101CA000C3680446002F3FF435AFB9F1000F3FF48D
:101CB00031AF09F1FF35414618463A4633F0AAFFE5
:101CC000013D691C00EB0703F5D123E7DA0706D4D1
:101CD00013F0030206D13F4A1B689342BDD1002096
:101CE00070F0D4FC022AB8D16FF3D603062BF6D1DC
:101CF000B3E7622B3FF448AFF1E72179364D01F0AD
:101D00007F01402035F024FA0246D4E9023003FB7B
:101D100002F12368AB4256D00124DDE9042300948C
:101D200029F0A6FC00287FF43AAF96E76268C2F378
:101D3000172200FB026606E7012A3FF425AF5A2A64
:101D40003DDC422A3FF420AFC9E76268C2F31722A4
:101D500000FB02773EE711464020002235F0F8F9FB
:101D6000A36809FB03F300FB03F1E06832F07AF9A2
:101D7000A368E06009FB03F3A360636803F0FF035B
:101D80006360B9F1000F3FF4C5AE09F1FF39C31923
:101D9000002F3FF4BFAE88E76368C3F3172300FB4F
:101DA000038875E793429AD123F00203642B96D0FF
:101DB000022D3FF4E9AE00287FF4E6AE8FE7622AF9
:101DC0003FF4E2AE8BE76368C3F3172302FB030023
:101DD000A2E700BF3C710B00A8650B00F0650B008B
:101DE000F0B5012885B007460E463FD08B0736D0A8
:101DF00030463FF005FD002857D0451029463846AB
:101E000000F026F90021044630463AF067FC064609
:101E10003AF02CFF68B17DB100252A460346E168FF
:101E2000384635F049FF304601353AF01FFF0028AB
:101E3000F3D1204605B0F0BD01462046FFF706FE6F
:101E400030463AF013FF0028F3D001462046FFF752
:101E5000FDFD30463AF00AFF0028EDD1E9E70B68B6
:101E6000144A934202D0144A9342C1D1012201A9DB
:101E700030463AF09DFB0028BAD039460022402077
:101E800035F066F9029BB3FBF0F100FB01F5AB42C4
:101E90000DD1384600F0DCF8019904462A46C068A6
:101EA00033F0B8FE204605B0F0BD0546A6E703486E
:101EB00070F058FC907C0B00F0650B00249A0B002E
:101EC00070B50E4686B00446012203A930463AF0AA
:101ED0006FFB00283AD021790022402035F038F9F4
:101EE0006268049BB3FBF0F3B3EB122F0546C2F319
:101EF0001721E06813D8C91A61F31F226260A26833
:101F00000399019302FB050003FB05F233F082FE07
:101F1000A268019B0E201A44A26006B070BDA168A1
:101F20000193194405FB01F132F09CF86268E0600E
:101F300002F0FF026260B442019BE0D1052203A9D6
:101F400020463AF035FBE068019BD8E70146304671
:101F50003AF0C4FB054601E0FFF778FD28463AF069
:101F600085FE014620460029F6D10E2006B070BD40
:101F700070B50D460179044601F07F0116464020F8
:101F8000002235F0E5F8E2682A60A36800FB03F35D
:101F90006B60237903F07F03AB602168094B9942A2
:101FA00001D0002070BD94F90430002B03DBB3078F
:101FB00001D5012070BD6368C3F3172300FB032222
:101FC0002A60EEE7A8650B004268C36891688B42FF
:101FD00084460BD21079D168DCF808201A4401330A
:101FE00000F07F00CCF80C3035F006BB00207047C5
:101FF000084A0023C1E90233C1E90020064B026808
:102000009A4201D0084670474368C3F317238B6098
:10201000084670473C650B00A8650B0038B50C46B8
:102020001D4611462046094A34F022FE286841F038
:1020300051FE012C007804D06968BDE83840FFF7F4
:10204000CFBEBDE83840002100F002B80400020015
:102050007828F8B51CD005460E46002201464020DF
:1020600035F076F8012D0CBF0B490C4907461020BE
:102070003FF03AFD05714368866003F0FF030446B4
:10208000436006FB07F031F0E1FFE0602046F8BD59
:10209000034870F067FB00BFF0650B0074650B0030
:1020A000949A0B0070B50D79012D0C4606462FD081
:1020B0001F492A4643F05EFEA3682BB930461D49EE
:1020C000BDE8704043F0B4BD1B49304643F0B0FD5D
:1020D000A3689BB1002501E043F0AAFD2A46E16810
:1020E000207935F089FA01220146304640F0C8FADD
:1020F000A36812490135AB423046EDD8104930464D
:1021000043F096FD30460B49BDE8704043F090BD6A
:102110000C4943F08DFDD4E9022130462B4645F0B1
:10212000A5FA30460349BDE8704043F081BD00BFC9
:1021300090270B00B0280B009C270B00A0270B005A
:10214000A4270B0084270B002DE9F04788B0002A54
:1021500035D011F0030304468C46806815461E46B0
:1021600003D1904B0A689A422ED062460146002362
:1021700020683AF057FA8C4B216894F804C09942D1
:10218000024609D0042D0FD1E1680CF07F0008B0A1
:10219000BDE8F04735F030BA6368042D00EB132238
:1021A000F2D01CF0800F0AD02B46E1680CF07F00C3
:1021B00035F082FD0E25284608B0BDE8F0870025E1
:1021C000284608B0BDE8F08702AA44F07BFD00284D
:1021D00000F0E2802179042D01F07F0132464FF0BA
:1021E000400078D034F0B4FF15F0030280464BD1A4
:1021F0002968887B30B101EB800003696B4883421A
:1022000000F0AD806A4A91423ED1B8F1010F40F032
:10221000C680052205A928463AF0CAF9DDE90597E6
:1022200061484FF0000ADDE902212668E3688D1A53
:102230008642A7EB05052AD0002D34DD6068B5EB9A
:10224000102F65D8D019A26801932A44121A08FBEE
:10225000013108FB02F208FB003033F00FFDDDE92D
:10226000013009EB0A0108FB07F200FB083033F0EC
:1022700005FD6368C5EB132262F31F23A268636048
:102280002A44A2600E2596E74A4870F0FFF994F9B7
:102290000410002993DA002D40F081806168C1F3B9
:1022A000172108FB013308FB023009EB0A0108FB88
:1022B00007F2019333F0E2FC0399A2680298019BB4
:1022C000521A384408FB02F208FB013108FB0030C7
:1022D00033F0D4FCCDE734F03BFF334B2168029A56
:1022E0009942064629D1B2F1807F51DA10203FF0A1
:1022F000FBFB054694E80F0085E80F00029A02EB0D
:10230000112363F31F216960039B9B1AAB6052E7A3
:10231000A26801932A4408FB02F1184631F0A2FE9C
:102320006268E06065F31F226260019B9945DDE908
:102330000221034608BF814684E703992079891A60
:10234000FFF786FEDDE902130546E0685B1A06FB2F
:1023500003F206FB0101E86833F05CFC2BE7297906
:10236000402001F07F0134F0F3FE404517D1AB6807
:102370000D482A681F46EB688242994602D04FF00A
:10238000000A50E76A68C2F3172208FB02FA4AE71C
:1023900009490A487BF0CBFC094870F077F90948F5
:1023A00070F0E0F9C4790B00A8650B004921030027
:1023B000907C0B002C9B0B0048920B00EC6C0B00EC
:1023C00060900B00F8920B00042808D0052801D07B
:1023D000002070478868400040F0010070478B681B
:1023E000002B0CBF1E203E20704700BF10EE102AAD
:1023F00022F00043B3F17E5FF0EE407A07D30FD0B6
:1024000070EE407A9FED3B7A87EE270A7047B3F172
:102410007C5F27D2A3F50003B3F1645F07D2704756
:102420009FED357A9FED350AA7EE870A704760EE7B
:10243000006A9FED336ADFED335A9FED337A9FEDEB
:10244000335AE6EE865AB7EE006AA6EEA57AA6EEF5
:10245000856A27EE267AC7EE066AE0EE267AB0EEA7
:10246000670A7047B7EE007AF0EEC07A77EE677AC7
:1024700000B5B6EE007A67EE877A83B0F5EE407A63
:10248000F1EE10FA28D4F1EEE76A002ADFED1C5ACB
:102490009FED1C6A9FED1C7A9FED1C5A9FED160A5A
:1024A000A7EEA56AF7EE005AA7EE867AE7EE855A00
:1024B00067EE277AB0EE005A87EEA57ADFED147A40
:1024C000E7EE266AE6EE857A30EE670A01DB03B0B6
:1024D00000BDB1EE400AFAE78DED010AB0EE670AE1
:1024E000CDED007A64F0C6F9019ADDED007AF0EEE8
:1024F000406ACAE700000000DA0FC93F000080030D
:102500006BD30DBCBA132FBD75AA2A3EAEE534BFFE
:102510006821A2B300B585B08DED010A019B23F0BF
:102520000042B2F18B4F00EE102A4FEAD37127D24E
:102530005B000ED4B2F1665F2BD2DFED1F7A70EE36
:10254000277ACDED037A039B09B1B1EE400A05B0BD
:1025500000BDB7EE007AF0EE476AE0EE006A019146
:10256000B0EE006AF1EEE67A77EE807AC7EE276A7F
:10257000E0EE066AB0EE660A31F03AFC0199E3E754
:10258000019131F035FCDFED0D7A019930EE270A2B
:10259000DAE720EE007AF7EE006A37EE266A01915C
:1025A000F1EEC67A77EEA67AC7EE276A36EE800A93
:1025B00031F068FB0199C7E70000807B1872313F5A
:1025C00008B55AF01DFC044B02689A4200D108BDC0
:1025D0000D205EF091F800BFEF29780100B585B0BD
:1025E00040F2FF1C01A903AB02AACDF80CC02BF0EE
:1025F000ADFC0248039970F0BDF800BFB0AB0B0012
:10260000F4EE400AF1EE10FAF0EE407A53D610EEF6
:10261000901AB1F17E5F49D010EE102A8B0F03F0B3
:10262000020343EAD27332F0004208D1022B3FD0BA
:102630009FED397A032B08BFB0EE470A704731F09F
:1026400000412ED0B1F1FF4F21D001F150609042F6
:1026500027D3B2F1FF4F24D000B5980783B030D50F
:1026600002F150628A4251D387EEA00A0193B0EE84
:10267000C00A00F063F8019B022B3ED19FED277A40
:10268000DFED277A30EE070A37EEC00A25E0B2F117
:10269000FF4F03F1FF3328D0022B20D99FED210AF1
:1026A0007047DB070AD49FED200A704700F046B858
:1026B0009FED1B0A704730EE800A70479FED1B0AA2
:1026C000704787EEA00A0193B0EEC00A00F036F81A
:1026D000019B012B01D1B1EE400A03B000BD144AA9
:1026E00002EB830393ED000A7047022B11D8114AC5
:1026F00002EB830393ED000A70479FED087ADFED4C
:10270000087A30EE070A30EE670AE6E79FED050A21
:10271000B2E79FED090A7047DB0F49C02EBDBB33FE
:10272000DB0F494000000000DB0FC93FDB0FC9BFD2
:1027300060390C006C390C00DB0F493F10EE102A99
:1027400022F00043B3F1994F4FEAD27109D3B4EEAE
:10275000400AF1EE10FA0ED6002943D09FED4A0A46
:1027600070474A48834207D8B3F1665F3DD212F002
:10277000FF4F00F081807047454A9342B0EEC00A97
:102780004ED9444A93426ED8F7EE087AF7EE006AC3
:10279000E0EE276A70EE677A9FED3F7A9FED3F0A81
:1027A00087EEA66A26EE065ADFED3D7ADFED3D4A5A
:1027B0009FED3D4ADFED3D5A65EE056AE6EEA74A1C
:1027C000DFED3B7AE6EE847AE6EEA45A67EEA67A6F
:1027D000E5EE257A97EE867A77EE467A30EE670A4E
:1027E00089BB70479FED330A704720EE006ADFED2A
:1027F0002C7ADFED2C5A9FED2C5ADFED2C6A26EE59
:10280000067AE7EE275ADFED2A7AE7EE057AE7EE59
:10281000256A67EE877AE6EE267AA7EEC00A704749
:10282000A2F5D002934211D8F0EE007AFFEE006AD2
:10283000E0EE276A70EE277A9FED1F7A9FED1F0A60
:1028400086EEA76AAEE7B1EE400A7047F7EE007A6F
:1028500070EE676A30EE270A9FED197A86EE806A7D
:102860009FED180A9EE7FFEE007A87EE806A9FEDE3
:10287000167A9FED100A95E760EE007A82B0CDEDF2
:10288000017A019B02B07047DA0FC9BFFFFFDF3E3C
:10289000FFFF973FFFFF1B40B40F14335E987B3F51
:1028A00025AC7C3D0DF5113E4712DABDA9AAAA3E22
:1028B00098CA4CBEDA0FC93F6937AC313863ED3E78
:1028C00068212233DA0F493F6821A23300B585B071
:1028D0008DED010A019B23F00042B2F17C5F00EE16
:1028E000102A4FEAD37124D2B2F13E5F0CD213F01A
:1028F000FF4F04D160EE007ACDED037A039B09B15E
:10290000B1EE400A05B000BD30EE007AF7EE007A75
:1029100077EEC07A67EE006A019186EEA70A30EE84
:10292000070A31F0AFF9F6EE007A20EE270A019996
:10293000E5E7F7EE007A77EEC07A019180EE277A2C
:1029400037EE070A31F09EF9F6EE007A20EE270AFC
:102950000199D4E7014B18682AF0C4BCB84601209D
:1029600010B5D1F800C001280C46134600F1FF3124
:1029700088BF221D604698BF002260F0F3FE2068E9
:1029800010BD00BF10B5044C206831F023FB034A92
:1029900000231360236010BDB8460120C04601200B
:1029A00000B583B0019001A860F048FF0E2003B08D
:1029B00000BD00BF08B50BF067FB0E2008BD00BFCF
:1029C00070B508468EB011461A461F4B08ACCDE9CB
:1029D0000034062334F02EFA9DF83440089840F273
:1029E000DD213CB373F0A4F840F2926106460998E9
:1029F00073F09EF802460A98079240F2533173F042
:102A00005FF84FF48F6106900B9873F071F80F49DF
:102A1000054628203FF070F802949DF8304000955C
:102A2000DDE906323146019405900BF0B1FA0598C4
:102A30000EB070BD73F044F840F2926106460998FA
:102A400073F03EF80246D6E730DD0B0070DD0B0078
:102A500010B504460BF066FB38B920460BF06AFB54
:102A600000280CBF1E203E2010BD5CF029FB00BFDB
:102A700010B504460BF056FB38B920460BF060FB4E
:102A800000280CBF1E203E2010BD5CF019FB00BFCB
:102A900010B504460BF046FB40B920460BF050FB46
:102AA00030B120460BF060FB0E2010BD5CF008FB3F
:102AB00001486FF023FE00BFFCA10B0030B50C688D
:102AC00087B005462046CDE902210BF02BFBDDE95E
:102AD000022188B904AB0193084B0093681E0223BE
:102AE000043134F0FFF820469DF8142004990BF0CF
:102AF00043FB0E2007B030BD5CF0E2FA60DD0B0056
:102B000010B504460BF00EFB50B920460BF012FB3B
:102B100008B90E2010BD20460BF034FC0E2010BD6D
:102B20005CF0CEFA10B504460BF0FCFA20B9204652
:102B30000BF030FC0E2010BD5CF0C2FA08B50BF0B3
:102B400081FC0E2008BD00BF2DE9F0472DED028B62
:102B500008468CB011461A46304B05ACCDE900341E
:102B6000072334F067F940F21E31059872F0A8FF90
:102B700040F256318046069872F0A2FF4FF4B262DE
:102B800081460121079834F0A5F9089D082D824659
:102B900001D0102D3DD10A9CA4F10801F72933D8AA
:102BA000630731D10B989DF82460EDB2E4B240B3D5
:102BB0003DF0C0FBB0EE408A40F2F252B0EE480A5F
:102BC0000121002034F04CF9154908203EF094FF13
:102BD00053464A464146CDE90164009507460BF04D
:102BE000E9FBDFED107A28EE278AFCEEC87A17EEB3
:102BF000900A39F0C5FD38460CB0BDEC028BBDE83B
:102C0000F0879FED098AD7E7084840F2E4416FF06A
:102C1000B1FD064840F2DE216FF0ACFD28DE0B006E
:102C200060DE0B0000007A44AE47E13D1CAB0B00B8
:102C300010B504460BF01AFC30B920460BF020FC0E
:102C4000400040F0010010BD5CF03AFAF0B585B0EC
:102C500006460C4617460BF009FC00283CD10546F9
:102C600040F26141384634F027FA294640F2614289
:102C7000074634F063F9A30703D11D4B22689A423B
:102C800032D0062201A9204639F092FC9DF80C10A2
:102C9000029C0022402034F05BFAB4FBF0F4BC420A
:102CA0001CD330460BF0EAFB039B482B0FD01028B7
:102CB00017D0422B01D0012B09D101993A46304659
:102CC0000BF0E2FB400040F0010005B0F0BD082829
:102CD000F3D108486FF046FD5CF0F2F906486FF05A
:102CE00041FD06486FF03EFD05486FF0CFFC00BF88
:102CF0000CB20B007C970B003CA60B0064970B00FA
:102D00006CA70B0090F82C20012A5CD190F82D3094
:102D1000002B58D090F82E30002B54D090F82B3048
:102D2000002B50D0036A002B4DD030B5044683B041
:102D300000926EF0B5F994F82B30009A591E8A4033
:102D4000D2B2216A002818BF134603FB01F1CDE976
:102D500000136EF0A5F9236A0099002814BF4FF400
:102D6000FA524FF47A721D46B1FBF2F200926EF005
:102D700097F994F82D10009A019B002894F82E00E2
:102D800002F1010201FB00F012FB00F2218A92B273
:102D900014BF4FF4FA5E4FF47A7E914214D303FBD2
:102DA00005F1A2EB000CB1FBFEF30EFB13111FFAB1
:102DB0008CFC89B100216CF30F016CF31F4161623F
:102DC000228503B030BD70474FF0E023D3F8F03DCB
:102DD000DB07F6D500BEF4E7ACEB0000A084A4F856
:102DE00026C02285EDE700BF2DE9F04F01298BB009
:102DF0000546164605D0022918D001200BB0BDE8C3
:102E0000F08F127812F060010F4637D173780A2BD9
:102E100053D00B2B7FD0012BEFD04FF0E023D3F812
:102E2000F03DDB0700D500BE0020E7E7137803F094
:102E3000E002202AE1D103F01F03012B00F0F28011
:102E4000022BEAD1B3880DF12701D8B2DFB200F02E
:102E500067FB0028E8D09DF827303BB9984B1C460B
:102E60005B681BB1DB79002B00F09F8171F078FF6C
:102E70003146024628466DF023FBBFE72029CCD11E
:102E8000B38802F01F010129D8B200F0F2800229B4
:102E9000C3D10DF1270100F043FB0028C4D096F9FF
:102EA0000030002BC0F2AD8171F05AFF4023024682
:102EB000314628466DF030FCA0E7814AB18853685E
:102EC0001446C9B2002BAFD09089002896D0184480
:102ED00004E01A781344C21A002AA5DD5A78042A9D
:102EE000F7D19A788A42F4D100238DF82730A37C59
:102EF0008B4202D1E37C8DF82730A37E8B4204BF46
:102F0000E37E8DF827300DF1270201233146284654
:102F10006DF002FC72E76A49B3884A680C46DBB27E
:102F2000002A81D0888900283FF47EAF104405E054
:102F300011780A44811A00297FF776AF5178042965
:102F4000F6D191789942F3D1A27C71889A42884651
:102F500000F0E480A27E9A4200F0F780A2896168C6
:102F600001EB020CA268ACEB0201002952DD5FFA12
:102F700088FE05E011780A44ACEB0201002949DD26
:102F800051780429F6D191789942F3D1D1787145DD
:102F9000F0D111798946B1B34FF0000163F3070115
:102FA0006EF30F21CDE9043E03919046E24693462D
:102FB00004E098F80030B945984421D9AAEB0803F9
:102FC000002B1DDD98F80130052BF2D14146284633
:102FD00071F03CFE00283FF420AF636898F80210BF
:102FE0001BB1DB79002B00F0FB8098F80330D8068A
:102FF00040F1C080284671F0F5FD7B1CDFB2D8E7B8
:10300000B9457FF411AF314628466DF0DFF900284D
:103010003FF40AAF2A48FFF775FE314628466DF0A7
:1030200065FBEAE6B388D8B21B0A4BD1244B1C4699
:103030005B68002B3FF4F8AEA18900293FF4F4AEA1
:10304000194405E01A781344CA1A002A7FF7ECAE37
:103050005A78042AF6D19A788242F3D100238DF867
:10306000273071F07DFE3146024628466DF02AFA7F
:10307000C4E6190A41D1124B1C465B68002B3FF491
:10308000D3AEA18900293FF4CFAE03EB010C06E0DB
:1030900019780B44ACEB030100297FF7C5AE5978D2
:1030A0000429F5D199788142F2D1002312068DF8D6
:1030B00027307FF5F9AE314628466DF019F99DE6C7
:1030C00020120120D9B20DF1270200F0FFF90028EB
:1030D0003FF4AAAE9DF827303BB9864B1C465B688F
:1030E0001BB1DB79202B00F0918071F039FE314665
:1030F000024628466DF0BAF980E60DF1270200F08D
:10310000E5F900283FF490AE96F90030002BBFF6A9
:10311000CBAE314628466DF06BF86FE6A17B03938A
:1031200000222846628271F079FD73486CF07EFEC1
:10313000314628466DF078F900283FF475AE00223C
:10314000039BA2736262228504E7A17D03930022A0
:103150002846628371F062FD68486CF067FE314674
:1031600028466DF061F900283FF45EAE0022039B13
:10317000A275F3E62846069171F034FD0699CB0955
:1031800061D1049BA376059BA175E376B8F8043062
:1031900000200090C3F30A03A26C2383284671F039
:1031A000A5FD00287FF429AF3EE6A37BBB427FF458
:1031B0005DAE73881B0A012B7FF458AE7378012B28
:1031C0007FF454AE71F0CCFD9DF827300268502199
:1031D00001FB034022F07F420262FFF793FD45E6C8
:1031E00098F80330284603F00C03CDE9061371F07C
:1031F000F9FC0699079BCA0922D1002B3FF4FDAECA
:10320000BFE7314628466DF071F8F7E594F82A30AB
:103210008B427FF46AAF73881B0A012B7FF465AF82
:103220007378012B7FF461AF71F09AFD9DF8273020
:103230000268502101FB03400262FFF763FD54E77F
:10324000002B3FF4DAAEBDF80C30A1736382B8F8FE
:103250000430C3F30A032382B4F840305B08A3822E
:103260009BF80030069300200BEB03026DF088F80A
:103270000128069B25D05078242809D000230093EC
:10328000E26C284671F032FD00287FF4B6AECBE543
:1032900090780128F2D1907A84F82D00507984F842
:1032A0002C001BF803301A445378242BE6D1937872
:1032B000022BE3D1D378012B04BF137984F82E308D
:1032C000DCE71BF8033013445A78242AD6D19A78C5
:1032D000022AD3D1DA7884F82C20012ACED11A79A7
:1032E00084F82D205A7984F82E209B6823F07F43A0
:1032F0002362C3E7201201205C120120501201203A
:103300000020704710B50D4C0C485022002132F0BF
:1033100065FE0B4901234FF4446204F13C006CF05C
:1033200089FD0848E064012307494FF4446204F131
:1033300030006CF07FFD054BA36410BD201201200E
:10334000904D0120906B0120D0590120546C012038
:103350004B79012B02D18B79012B01D000207047D2
:10336000CB7913F0DF0FF9D10B7801EB020C0B4492
:103370006345F3D210B593F800E09E44F44507D3BB
:103380005C78042C04D0E6457346F4D3002010BDCD
:10339000ACEB030EBEF1080FF8DD93F805E0BEF1CB
:1033A000010FF3D19B79022BF0D10B79012B2BD894
:1033B0002AD0CB78002BE9D1384B5B6823BB374B45
:1033C000596018700B78D21A002A60DD0B4409206E
:1033D0000AE00B2A20D01A781344ACEB030E024407
:1033E000BEF1000F90B217DD5A78042AF1D15A7954
:1033F000012A11D19A79022A0ED1284A9268002A0C
:10340000E9D1264A9360E6E74FF0E023D3F8F03D98
:10341000D907BBD500BEB9E7204B988198B301EB23
:10342000000C0B460AE091F807E0BEF1200F1AD01D
:103430001A781344ACEB0302002A24DD5A78052ADB
:10344000F1D1DA7802F0030EBEF1010FF0D193F85A
:1034500002E05FEADE1EEBD0D206E9D40F4C9A7987
:1034600084F82B20E4E7242AE2D19A78032ADFD1DA
:10347000B3F804E040F201129645D9D1074C1A7A0C
:1034800084F82A20D4E7054A0123137710BD034BA3
:103490000920988101EB000CC3E700BF2012012036
:1034A00010B530220021054832F098FD04486CF038
:1034B000BDFCBDE8104003486CF0B8BC20120120F0
:1034C0005C12012050120120704700BF10B5134C50
:1034D0006368FBB193F802C08646F4454FF00000E4
:1034E00000D010BD1878D4F808C01C5C03442344F5
:1034F000ACEB0300002806DC0EE018780344ACEBCC
:103500000300002808DDD8788842F6D10023137024
:10351000012010BD184610BD002010BD2012012052
:103520000E4B5A68C2B1B3F80CC09B689444ACEB24
:103530000302002A06DC0FE01A781344ACEB030206
:10354000002A09DD5A78052AF6D19A788242F3D109
:1035500000230B70012070470020704720120120CB
:10356000002070472DE9F04F514CA27B8A4283B076
:1035700080461F4625D0A37D8B420BD1A16C002332
:10358000BAB204F130006CF01FFD38B9012003B06D
:10359000BDE8F08F002003B0BDE8F08F0122238B3F
:1035A0000092A26CA17D404671F0A0FB0028EDD0F6
:1035B000E27EA37D0092B9B2002240466CF004FF87
:1035C000E4E7E37C002BE1D0B4F84430B4F84620C3
:1035D000B4F84010208A92B29BB29342B6BFC2EBBD
:1035E00041029A1AD21892B2E38C8A4228BF0A4644
:1035F000002B38D0B3EB810F35DCA18C8A4236D357
:10360000258DA68ADFF8B0E0A5EB030C1FFA8CFC31
:10361000AA46B346DEF80050A6EB0C06B242A94615
:1036200027DA002D33D1884228BF08460A230246F4
:10363000CEF80030E16C1F48002315466CF0A0FC6A
:1036400001230093E26CA17B2B46404671F04EFBB8
:1036500000289BD0E27CA37B0092B9B200224046B6
:103660006CF032FF92E7824228BF0246E2E7002276
:10367000E0E7DC44624513DD4DB98245524628BF80
:1036800002468B42D6D00A23CEF80030D2E79842C9
:1036900028BF184609F1FF330246CEF80030C9E7CB
:1036A000002DF4D1984228BF18460246C2E700BF59
:1036B000201201205C1201200C48012008B50AF0FC
:1036C00039FF0E2008BD00BF70B590F80FE0D0F8AC
:1036D00008C0BEF1000F13D0049CC4F800C0D0F89D
:1036E00010C081B390F80DE0007BB2FBFEF10EFB41
:1036F0001121C008C9B201FB00C11960002070BDD2
:10370000049C4FEA5C0CC4F800C0856890F814E093
:1037100004694FEA550C0EFB0CFC41B904EB0C029A
:103720001A60037DC3F101030375002070BD457B62
:10373000017BB2FBF5F605FB1622C908D2B212FBDB
:1037400001C2A218ECE7C3F800C0002070BD00BFA2
:1037500010B508468EB011461A462B4B0AACCDE97F
:103760000034042333F066FB0A98052207A938F0D9
:103770001FFF099B622B2FD0682B2AD0422B2ED003
:1037800030DC012B08BF002430D19DF834204AB929
:103790000B9A089903FB02F25200B1FBF2F002FB14
:1037A000101159BB1949059318203EF09DF99DF859
:1037B000342003920C9A02929DF82C200192059BD2
:1037C000089A0799009404900AF0A0FE04980EB09D
:1037D00010BD01240223D8E701242346D5E70024A5
:1037E0000123D2E723F02003482B04D0084840F2FD
:1037F000FD216EF0BFFF00240223C6E7054840F21A
:10380000FD216EF0B7FF00BF04DF0B0024DF0B00CB
:1038100038AB0B007CA30B00704700BF08B50AF063
:103820006FFF0E2008BD00BFF0B50446856B85B064
:103830001F46E9B1012A164672D0A26A636BE2B94B
:10384000AB426FD0E18C01350D44ED1AEB0755D535
:1038500023693B600A9A63691360002E55D1A36BFC
:103860000133A363A06A003818BF012005B0F0BD82
:10387000A26A636B0E46002AE2D0AB42E18CE2D131
:10388000E36A9A4228BF1A46C9074CBFA169216959
:103890003960206B0192083003AB79F051F90028B0
:1038A00046D1039B019A934242D1A16A891AA1622F
:1038B00091B912F003000FD0C0F104001318227B5D
:1038C0000393082A37D0102A06D13A6823F001035F
:1038D0001A4422F8021C039B0A9A1360E18CCA075F
:1038E0004CBFE36163610131636B89B20135013320
:1038F0000D44ED1A6363EB07E184A9D4A3693B602F
:103900000A9AE3691360002EA9D0012EAAD1E36BB5
:10391000227B0133E3633B6803EBD2033B60A1E707
:10392000C56B8AE70A9B3A6010461A6005B0F0BD85
:10393000022005B0F0BD4FF0800C3A685B1A1A44C3
:10394000013102F801CC8842039BF6D1C4E700BFE5
:1039500070B51E460D4686B011462846224A33F001
:1039600087F93468214B2340062B05D0A00731D1BD
:1039700023681F4A934209D121461E4845F2663208
:1039800035F022F98107044624D103681A4A93428C
:1039900020D1012D21D97068062203A938F008FE34
:1039A00040F2FD234FF480620498039E082133F017
:1039B000D1FA4207034613D11049019340203EF04B
:1039C00093F8019B3246214605460AF0B7FD28468A
:1039D00006B070BD0A486EF0B1FE00231E46EBE74C
:1039E000084808216EF0C6FE040002000F0080FFA8
:1039F000E07C0B0078B00B000CB20B0098DF0B00E2
:103A000070960B0044A80B0009B1012A12D010B522
:103A10000146006B0C6A8A8C82B000238C620830ED
:103A2000019178F019FD01990023C1E90D33CB63B1
:103A300002B010BD704700BF08B50AF097FE0E2017
:103A400008BD00BF2DE9F04F2DED068B824693B0E7
:103A50001E462298DAF82430E1B1012A154600F01A
:103A60004E84DAF818200260DAF820109AF81C2048
:103A7000994229D082B9DAF8103033608DB9DAF87A
:103A800024300133CAF82430012013B0BDEC068B7A
:103A9000BDE8F08F0D46E4E7DAF814303360002D0E
:103AA000EDD0012DF0D1DAF828309AF80C2001334E
:103AB000CAF828303368012003EBD203336013B017
:103AC000BDEC068BBDE8F08FDAE90437002A18BF99
:103AD0001F4637609AF81C3083F001038AF81C30C7
:103AE000DAF818304FEA930B9AF82C30002B00F0DC
:103AF0000A8400249FED96AADFED969A9FED969A90
:103B0000DFED968A0D971095119605945F460AF1A0
:103B10003005564655F804BFDBF808200392002A0A
:103B200000F0DC80002F00F0D7800D9B04930BF198
:103B30001003CDE90737CDE90945DBF814200297DA
:103B400042BB9BF80D304BB99BF80C30002B00F0BA
:103B5000D083DBF80800114601F0FAFADBF8080020
:103B6000002800F053810BF114030022009311464A
:103B7000079B01F04DFA022800F0A683DBF8142021
:103B8000A0F10100B0FA80F0400992088BF80D0016
:103B9000CBF81420039B717B587BDBF810A0884284
:103BA0004FEA012340F037810298834228BF034641
:103BB000934228BF134698467068B8FBF1F189B26A
:103BC0005FF074FDF7EE000A0BF11800B0EE4A0A40
:103BD00067F0C8FCF0EE690AB0EE408A0BF11C00F9
:103BE000B0EE490A67F0E0FC28EE288A727BBCEE52
:103BF000C88A022A18EE103A9FB240F00A810304E4
:103C000000F1FD80C0F5FF407F3080B24FF40043EB
:103C100007FB00F007FB03F3C013DF13039B597B83
:103C2000059BDBE90845002B40F09A80337B102B85
:103C300040F07E81B37B002B00F0D7818A4240F0B8
:103C4000D382B8F1000F00F00481049BAAF10402B2
:103C5000DDF814A0CDF818A0A3F1040E4FEA880CEB
:103C600002EB8809A04252F8041F63D1AF4261D130
:103C7000230433FB01F34FEA054A3AFB11F123F326
:103C8000CF3321F3CF31C3EA01434A454EF8043F15
:103C9000E8D1039B727B5B7B9A4240F0C880029B19
:103CA000DBF81420A3EB08030293049B6344049302
:103CB000DBF81030A2EB08026344CBF81030029B13
:103CC000CBF81420CBE90807002B7FF439AFDDE9EE
:103CD00008740A9D96F82C30012205920134A34203
:103CE0003FF718AF059B109DBB46B2460D9F119E36
:103CF000002B00F008839AF80E30ABB99AF80C301C
:103D0000102B00F04785BBF1000F0DD00BF1FF33F6
:103D100007EB83034FF08031043F57F8042F82FAFA
:103D200041F29F423A60F8D1DAF820300133CAF804
:103D30002030A3E6B1F5803F5ED38BB2002B5BD081
:103D4000069B1BB14B4013F0802F55D106918FE796
:103D50000000000000FE7F3F00FE7FBF0000004724
:103D6000337B102B77D196F80EC0BCF1000F00F01A
:103D70007E818A4240F0C481B8F1000F69D0AAF177
:103D80000402049B4FF0000AA04202EB8809A3F151
:103D9000040E52F8041FCDF818A04FEA880C1BD16E
:103DA000AF4219D1230433FB01F34FEA054A3AFB32
:103DB00011F123F3CF3321F3CF31C3EA01435EF88E
:103DC000041F93FA11F34A45CEF800303FF461AF77
:103DD000A04252F8041FE3D0B1F5803F09D38BB263
:103DE0003BB1069B1BB14B4013F0802F01D10691D4
:103DF000D8E73D460446D5E73D46044638E700F59A
:103E0000FF407F3083B24FF4004001E7DBF814201D
:103E1000C0E6384602E74FEA4208029A934228BFBA
:103E20001346984528BF9846C6E64FEA880C049B7F
:103E3000DBF8141063440493029BA3EB0803029382
:103E4000DBF810304FEA580803EB8803A1EB0802B7
:103E500033E7C44623E78A424FEA480340F003832E
:103E6000002B00F02E82049A0693AAF1020C002186
:103E7000A2F1020A0B918E46624632F802CF96F802
:103E80000E904FEA0C414FEA0C2C01F07F411FFAD3
:103E90008CFC41EA0C01B9F1000F03D14FF08023F3
:103EA00091FA43F1A0422FD1AF422DD14FEA044CF9
:103EB0003CFB01FC4FEA054939FB11F92CF3CF31EA
:103EC00029F3CF39C1EA09413AF8029F4FEA094C78
:103ED0004FEA09291FFA89F90CF07F4C4CEA090CCA
:103EE00091FA1CF14FEA114C069B0EF1010E0CF4F5
:103EF0007F4CC1F307214CEA01017345AAF8001079
:103F0000BBD14FEA880CC4E6B1F5803F0BD31FFA52
:103F100081FCBCF1000F06D00B9B3BB181EA030C86
:103F20001CF0802F02D03D460446BFE70B91BDE751
:103F30008A4240F00B825FEA480300F0C281049994
:103F40000693A1F1020905990B91AAF102028A4692
:103F500032F802CF96F80EE04FEA0C414FEA0C2CF3
:103F600001F07F411FFA8CFC41EA0C01BEF1000F09
:103F700003D14FF0802391FA43F1A04221D1AF4207
:103F80001FD14FEA044C3CFB01FC4FEA054E3EFBBF
:103F900011FE2CF3CF312EF3CF3CC1EA0C414FEA96
:103FA000114C069B0AF1010A0CF47F4CC1F3072166
:103FB0004CEA01019A4529F8021FC9D14FEA880C41
:103FC00067E6B1F5803F0BD31FFA81FCBCF1000F0F
:103FD00006D00B9B3BB181EA030C1CF0802F02D072
:103FE0003D460446CDE70B91CBE78A4240F054832F
:103FF000B8F1000F3FF42DAF049ACDF818B0AAF134
:104000000403A2F1040E059A0B924FEA880C03EB0D
:10401000880A4FF0802953F8042F92FA49F2A042FF
:1040200015D1AF4213D1210431FB02F14FEA054B08
:104030003BFB12F221F3CF3122F3CF32C1EA02412E
:1040400053454EF8041FE6D1DDF818B021E6B2F56D
:10405000803F07D391B229B10B9931B1514011F092
:10406000802F02D03D460446DDE70B92DBE78A4213
:1040700040F09682B8F1000F3FF4EBAEAAF10403D2
:10408000049ACDF82CC003EB880AA2F1040E53F871
:10409000041FCDF818B04FEA880C4FF0802991FA30
:1040A00049F1A0421CD1AF421AD1220432FB01F2E5
:1040B0004FEA054B3BFB11F122F3CF3221F3CF3115
:1040C000C2EA01425EF8041F92FA11F25345CEF89B
:1040D0000020B9D053F8041F91FA49F1A042E2D070
:1040E000B1F5803F07D38AB22AB10B9A32B14A4068
:1040F00012F0802F02D03D460446D6E70B91D4E75C
:10410000B8F1010F7FF691AE04994FEA5803AAF176
:10411000040C01EBC30E8A4600210C91CDE90EB6CA
:104120000104069139040B915CF8042FA04293B26C
:1041300043EA024348D1AF4246D121044FEA054940
:1041400031FB03FB39FB13F32BF3CF3B23F3CF33CB
:10415000CBEA0343DAF8006093FA16F3CAF80030AA
:10416000130C1B04A04243EA12431AD1AF4218D1E8
:1041700031FB03F139FB13F321F3CF3123F3CF33B9
:10418000C1EA0342DAF8043092FA13F2CAF80420C2
:104190000AF1080AF245C7D1DDE90EB64FEA880CEC
:1041A00077E5B3F5803F07D39AB22AB10C9A4AB1AA
:1041B0005A4012F0802F05D00699DDF82C903D462C
:1041C0000446D5E70C93D3E7B3F5803F07D399B204
:1041D00029B10C9931B1594011F0802F02D03D46E0
:1041E0000446AAE70C93A8E7B8F1010F7FF61DAECD
:1041F0000499CDF838B04FEA580301EBC303AAF194
:1042000004098A4605990C910104069139040B9121
:104210009B4659F8042FA04293B243EA024340D18F
:10422000AF423ED121044FEA054E31FB03FC3EFB79
:1042300013F32CF3CF3C23F3CF33CCEA0343CAF878
:104240000030130C1B04A04243EA124316D1AF42C4
:1042500014D131FB03F13EFB13F321F3CF3123F3F0
:10426000CF33C1EA0341CAF804100AF1080ADA455B
:10427000CFD1DDF838B04FEA880C0AE5B3F5803FBE
:1042800007D39AB22AB10C9A4AB15A4012F0802F41
:1042900005D00699DDF82CE03D460446D9E70C939D
:1042A000D7E7B3F5803F07D399B229B10C9931B163
:1042B000594011F0802F02D03D460446B2E70C93DE
:1042C000B0E74FEA880CEAE4DDE9087400230A9DB0
:1042D000CBF80830CBF814308BF80D30059B2BB998
:1042E000029BDDE904019A0031F078FE96F82C304B
:1042F000F2E4DDE908740A9DCBF80820EEE7DAF86D
:104300002830FFF7AEBBBBF1000F3FF40DAD4FEA15
:104310008B020021384631F061FE9AF80E30002BF6
:104320007FF402AD9AF80C30102B7FF4EFAC0BF158
:10433000FF3107EB81013B1F4FF0802053F8042F22
:1043400092FA40F28B421A60F8D1EDE44FEA48034A
:10435000012B7FF66AAD049ACDF83880010408F18C
:10436000FF3306913904AAF102090AEB430ECDE9A5
:104370000B1B02F1020A059A904639F8023FB27B04
:1043800019041B0201F07F419BB219431AB94FF087
:10439000802391FA43F18BB2A04243EA014350D10A
:1043A000AF424ED122044FEA054C32FB03FB3CFBEB
:1043B00013F32BF3CF3B23F3CF33CBEA03434FEA83
:1043C000134B0BF47F4BC3F307234BEA030B0B0C8C
:1043D0001B04A0422AF802BC43EA11431CD1AF429D
:1043E0001AD132FB03F23CFB13FC22F3CF332CF344
:1043F000CF32C3EA02431A0C02F47F42C3F307230D
:104400001343F1452AF8043BB7D1DDF83880DDF8D5
:1044100030B04FEA880C3CE4B3F5803F0BD399B23F
:1044200049B1B8F1000F00F0AD8183EA080111F045
:10443000802F00F0A781069ADDF82CC03D46044687
:10444000CFE7B3F5803F0BD39AB24AB1B8F1000F72
:1044500000F09A8183EA080212F0802F00F0948124
:104460003D4604469EE7012B7FF6DFAC049A08F137
:10447000FF330AEB4303AAF1020E02F1020A002203
:10448000069202040B923A04CDE90EB80C929B46B8
:104490003EF8023FB27B19041B0201F07F419BB240
:1044A00019431AB94FF0802391FA43F18AB2A0421E
:1044B00042EA014264D1AF4262D123044FEA054C83
:1044C00033FB02F83CFB12F228F3CF3822F3CF3251
:1044D000C8EA02493AF8028C4FEA08424FEA082833
:1044E0001FFA88F802F07F4242EA080299FA12F2B3
:1044F0004FEA124808F47F48C2F3072248EA02084C
:104500000A0C1204A0422AF8028C42EA114225D178
:10451000AF4223D133FB02F33CFB12F223F3CF3340
:1045200022F3CF32C3EA0243BAF800100A040902A8
:1045300089B202F07F420A4393FA12F31A0C02F492
:104540007F42C3F307231343F3452AF8043B9FD16B
:10455000DDE90EB84FEA880CFFF79BBBB2F5803F50
:1045600009D391B239B1069919B1514011F0802F98
:1045700001D10692CEE7DDE90B3C3D460446C9E792
:10458000B2F5803F09D393B23BB1069B1BB15340B8
:1045900013F0802F01D106928FE73D4604468CE749
:1045A000B8F1010F7FF641AC020404990B924FEA77
:1045B00058033A04CDE90EB8AAF1040A0C9201EBB3
:1045C000C30EB046CDF818C05AF8043F4FF0802211
:1045D00093FA42F91FFA89F3A04243EA09434BD107
:1045E000AF4249D122044FEA054C32FB03FB3CFBAE
:1045F00013F32BF3CF3B23F3CF33CBEA03430E6804
:1046000093FA16F30B604FEA19431B04A04243EAE6
:1046100019431BD1AF4219D132FB03F23CFB13FC0F
:1046200022F3CF332CF3CF32C3EA02424B6892FA23
:1046300013F34B6008318E45C6D14646DDF83C8009
:10464000DDF838B04FEA880CFFF723BBB3F5803FA5
:104650000DD31FFA83F9B9F1000F08D0069E26B1D9
:1046600083EA060919F0802F01D10693D4E7DDE92A
:104670000B2C3D460446CFE7B3F5803F09D39AB2F1
:104680003AB1069A1AB15A4012F0802F01D106931E
:10469000A8E73D460446A5E7B8F1010F7FF6C5AB94
:1046A000049ACDF838804FEA580302EBC3030104A3
:1046B0009146059A06913904CDE90B1BAAF1040A2B
:1046C000B346984616465AF8043F4FF0802293FAB4
:1046D00042FC1FFA8CF3A04243EA0C4344D1AF42A0
:1046E00042D12204290432FB03FE31FB13F32EF3E3
:1046F000CF3E23F3CF33CEEA0343C9F800304FEA6D
:104700001C431B04A04243EA1C431AD1AF4218D1F8
:1047100032FB03F231FB13F322F3CF3223F3CF3317
:10472000C2EA0343C9F8043009F10809C145CAD1F6
:10473000DDF838805E464FEA880CDDF830B0FFF7D0
:10474000A8BAB3F5803F0AD31FFA83FCBCF1000F6F
:1047500005D0EEB183EA060C1CF0802F18D0069A23
:104760000B993D460446D3E7B3F5803F07D39AB291
:104770002AB15EB183EA060212F0802F06D03D46D0
:104780000446AEE798462CE698460BE61E46A8E798
:104790001E46BDE7BBF1000F7FF4C9ADFFF7C4BAF9
:1047A0002DE9F04308468BB011461A462E4B04AC57
:1047B000CDE90034062332F03DFB40F28263FF2254
:1047C0000121049832F092FB40F2133302220121BE
:1047D0000746069832F08AFB4FF4B2620446012184
:1047E000099832F077FB079D082D804601D0102DE7
:1047F00037D107F10D001D4980003DF075F9E4B295
:104800009DF820300093059ACDF808800194EBB212
:10481000F9B2064609F07AFF002F17DDDFF8548061
:1048200098F8083008EB830306F13005D3F81090B0
:104830000024002319461A464046C847013445F86B
:10484000040F31460AF026F8A742F2D196F82C0060
:1048500006F134013DF008FE306330460BB0BDE890
:10486000F08303486DF07EFF5CE00B00ACE00B00D2
:10487000789A0B0080E10B0000B583B0019000F046
:10488000BBFB019809F07EFF00280CBF1E203E20D4
:1048900003B000BD00B583B0019000F0ADFB0198FE
:1048A000006B03B000BD00BF30B551F8044B89B0B8
:1048B00005462046CDE9022100F09EFB05AB0193A1
:1048C0000E4B0093DDE90221681E032332F00AFA41
:1048D00094F82C20069840F281630021013A32F0CE
:1048E00005FBC0B204EB80009DF81C200599406BCD
:1048F00009F08CFF204609B030BD00BF94E00B00EA
:1049000030B551F8044B87B005462046CDE9022169
:1049100000F072FB05AB01930C4B0093DDE9022123
:10492000681E012332F0DEF994F82C20059840F23D
:1049300081630021013A32F0D9FAC0B204EB80045D
:10494000606B09F0A9FF0E2007B030BD8CE00B00B2
:1049500090F82C307BB170B5064600F1300500248C
:1049600055F8040F09F064FF013496F82C20E3B2E7
:104970009A42F5D870BD704700B5084683B011461D
:10498000002232F075F9054928203DF0ADF801907C
:1049900009F012FF019803B000BD00BF80E10B00D9
:1049A00008B509F021FF0E2008BD00BF09F022BFA5
:1049B00008B509F021FF00280CBF1E203E2008BDCD
:1049C00009F01CBF08B509F01BFF00280CBF1E2012
:1049D0003E2008BD10B584B002AB51F8044B0193E2
:1049E000074B00930138022332F07CF920469DF8F2
:1049F0000C20029909F00AFF0E2004B010BD00BF80
:104A000070E10B0008B509F033FF0E2008BD00BFB0
:104A100010B5044608463CF0A3FE0146204609F0C6
:104A20002FFF0E2010BD00BF08B509F02BFF0E2090
:104A300008BD00BF10B584B003AB51F8044B01931F
:104A4000054B00930138012332F04CF9204609F060
:104A500023FF0E2004B010BD68E10B0008B509F07B
:104A60007FFF0E2008BD00BF70B5456A86B0002DDF
:104A700000F0A6800446002953D011460A98A56884
:104A8000056094F9540088426FD0C2F1010284F8A5
:104A9000542094F84420B2FA82F2520904EB8201C5
:104AA00084F8442084F855204A6B1A602046164644
:104AB00031F0A8FF0021204631F062FF01460028B6
:104AC0006ED0D4E90B239B1A0493636A13440593B5
:104AD000002300932069334604AA05A9F5F75CFD7D
:104AE000431C20D0226B0499521AE26230B3002199
:104AF00003902A46304631F071FA94F84510039B32
:104B0000002960D1023319D0A2680391304631F0F8
:104B100065FA0A9A03991160012384F8453002204E
:104B200021E00A46AAE703902A460021304631F0E8
:104B300055FA94F84520039B002A44D1A36D03EB5A
:104B400055032046A36531F05DFF0021204631F07A
:104B500017FF0546D4E90B01A26A091A521AB2F5E9
:104B6000007F16DC284606B070BD94F9551004EBA2
:104B700081010120496B01EB42021A60FF210A9B6F
:104B800084F854101A68A36D03EB5203A36506B0B2
:104B900070BD1749224604F1140000F079FBE1E7EB
:104BA000A2680391304631F019FA0A9B0399196003
:104BB00094F8450080F001004000C0B206B070BD1E
:104BC0000A9B1D60ABE7A26803930021304631F0D9
:104BD00005FA039B03330A9B4FF001024FF00001DB
:104BE0008CBF002001201960904084F84520BAE76E
:104BF000056C060070B51E460D4686B01146284667
:104C00001C4A32F035F834681B4B2340062B1ED06B
:104C1000A30718D00121204637F040FD037C13F094
:104C2000010324D1012D1AD81E46144901935C209A
:104C30003CF062FF019B32462146054609F030FEFA
:104C4000284606B070BD0E4B22689A42E2D121463A
:104C50000C4845F2663233F0B7FF0446DAE7706875
:104C6000062203A937F0A4FCDDE90363DDE706486B
:104C70006DF064FD040002000F0080FF64E20B0091
:104C8000E07C0B0078B00B0070960B0000B583B091
:104C9000019000F0B1F90198006C03B000BD00BFB5
:104CA00000B583B0019000F0A7F9019809F06AFE01
:104CB000B4EE400AF1EE10FA09D610EE103A23F0E5
:104CC000030040F00200A0F1FF4003B000BD014826
:104CD000FBE700BF0200400000B583B0019000F088
:104CE0008BF9019809F08EFE400040F0010003B0FE
:104CF00000BD00BF10B582B00446019100F07CF900
:104D00000199064845F2663233F05EFF01462046BF
:104D100009F07AFE0E2002B010BD00BF78B00B0083
:104D200038B50C46054600F067F90121204637F0FA
:104D3000B5FC037CDB0705D42846214609F064FE58
:104D40000E2038BD01486DF0F9FC00BF70960B00D5
:104D500009B1012A24D010B5044682B000F0ECFA63
:104D600094F8453023B902B0BDE8104000F0C0BA55
:104D70000022206C114663F0D1FA0028F3D1FF2302
:104D8000C4E90B0084F84500A065019084F8543014
:104D9000204631F037FE0199204631F0F1FDE2E77F
:104DA000704700BF08B509F003FF0E2008BD00BF23
:104DB00010B5084688B011461A46114B0DF1140C77
:104DC000CDE9003C032332F035F8059840F25E410E
:104DD00070F076FE40F26F510446069870F088FE3F
:104DE0000849039024203CF087FEBDF81C30039A4C
:104DF0000290214609F0A4FE029808B010BD00BF41
:104E000050E30B0078E30B0010B5044609F012FFE5
:104E100038B9204609F014FF00280CBF1E203E20A0
:104E200010BD5AF04DF900BF10B5044609F002FF5D
:104E300038B9204609F006FF00280CBF1E203E208E
:104E400010BD5AF03DF900BF10B5044609F0F2FE5E
:104E500040B9204609F0F6FE30B1204609F0FEFECA
:104E60000E2010BD5AF02CF901486DF047FC00BF30
:104E7000FCA10B0030B50C6887B005462046CDE993
:104E8000022109F0D7FEDDE9022188B904AB0193C4
:104E9000084B0093681E0223043131F023FF2046A3
:104EA0009DF81420049909F0E1FE0E2007B030BDF2
:104EB0005AF006F968E30B0010B5044609F0BAFE93
:104EC00050B9204609F0BCFE08B90E2010BD20469E
:104ED00009F080FF0E2010BD5AF0F2F810B504461C
:104EE00009F0A8FE20B9204609F084FF0E2010BD6D
:104EF0005AF0E6F83E4BD3F80021D00050D510B55B
:104F00003C4B84B003F1100453F8040BB8B1C27FDA
:104F100042B98168D1F804C1BCF1000F02D04277D8
:104F2000C1F80421427F52B1827F62B18268D2F817
:104F3000101141B3D2F8141169B3012151609C42A0
:104F4000E2D104B010BDC27F002AF8D190F822202F
:104F5000002AF4D18168D1F808C1BCF1000F38D122
:104F6000D1F80C214ABB90F91C20002AE7DB51093B
:104F7000DFF87CC002F01F026031012000FA02F26B
:104F80004CF82120DBE7D2F808110029D7D1D2F85C
:104F900014110029D1D1D2F80C110029CFD1CCE7BE
:104FA000D3F804219107AAD4D3F804215207A6D438
:104FB000D3F804319B04A2D47047002102930190DE
:104FC00026F046F90198029B82680021C2F80C1174
:104FD000C9E70121CDE90232019026F039F90198A3
:104FE000039A8168029BC1F808218168B8E700BF75
:104FF00000E100E0380A012008B5437B03B108BD99
:105000005AF05EF8407BB0FA80F04009704700BF6C
:10501000F0B583B004460E4601464FF4A360CDE9D7
:105020000032089D40F0C6FE07462046FFF7EAFF23
:10503000DDE9003240B90895BD6831462046AC46EE
:1050400003B0BDE8F0406047002202201A602A60E9
:1050500003B0F0BD00234373704700BF30B583B089
:105060000C4605464FF4A360019240F0A3FE204693
:10507000FFF7C2FF61686B68019A994211D16B7B9F
:1050800062B9627B9A421BD1227B2B7B9A4212D15E
:10509000A27BAB7B9A4209D103B030BD022BF0D189
:1050A000F2E70A484FF4B2616DF064FB074840F242
:1050B000C5516DF05FFB054840F2E6216DF05AFBEB
:1050C000024840F213316DF055FB00BF4C9F0B00BE
:1050D00008B5437B23B1007B400040F0010008BDD0
:1050E00059F0EEFF407B18B1400040F001007047DE
:1050F00008B559F0E5FF00BF00B5437B83B063B14D
:10510000014601904FF4A36040F054FE01994868B5
:10511000400040F0010003B000BD59F0D1FF00BFD6
:1051200038B5437B93B104460D4601464FF4A36066
:1051300040F040FE28463BF077F94FF4B26201217F
:1051400031F0C8FE034663600E2038BD59F0B8FF49
:105150002DE9F04104460F464FF4A3602146164660
:1051600040F028FE05462046FFF74CFF30B96B683B
:10517000324639462046BDE8F0411847BDE8F08187
:10518000704700BF014B00221A707047757B0120E9
:105190000349044B0120002208701A60704700BFC9
:1051A000757B01208C6B0120014B1878704700BF84
:1051B000757B0120024B1868003818BF012070472A
:1051C0008C6B012008B50D4B186818B10C4A126899
:1051D0000AB1002008BD65F03DFF084B1A681B6846
:1051E0008242A0EB030088BF00F1FF3040F2EE23C3
:1051F000984294BF0020012008BD00BF8C6B0120A5
:10520000AC460120014B00221A6070478C6B0120D4
:10521000024A136823EA000313607047AC4601207A
:10522000024A136803431360704700BFAC46012075
:10523000134B1B7813B1134B1B6803B1704700B5B8
:10524000114B83B01A68019265F004FF0E4B019A6E
:105250001860196811B132B103B000BD196801318D
:105260001960002AF8D1012065F092F9074B03F18B
:1052700078029A6203B05DF804EB57F0CBBD00BF33
:10528000757B0120AC4601208C6B0120A4700120AD
:10529000C0E9001200F000B800B583B0019012F030
:1052A000BFF80198C368BBB90F490A68824213D09E
:1052B0000E4A8360D2F800C01368C0F80CC00BB16E
:1052C000136898600B6863B1106012F0EFF803B0D8
:1052D0005DF804EB57F09EBD03B05DF804EB12F0EF
:1052E000E5B80860F0E700BFBC460120C4460120D5
:1052F00008B512F095F8044A1368013B1360BDE845
:10530000084012F0D3B800BFB046012010B5054BDD
:105310001C682CB1606827F0E5FFA468002CF9D167
:1053200010BD00BFBC460120024B1868003818BFF2
:1053300001207047BC46012008B512F071F8044AFC
:10534000136801331360BDE8084012F0AFB800BF26
:10535000B04601202DE9F043DFF8709083B00027BC
:10536000019712F05DF8D9F800504DB30DF1040823
:105370003E4602E00023E360ADB12C462846AD680E
:10538000A66028F0CBFA0028F4D1606828F0C6FAAD
:105390000028EFD13B46C8F80040274604F1080832
:1053A000E360002DE9D1019A0649074BC9F80020B6
:1053B00000220F601A6012F079F803B0BDE8F083A4
:1053C0002F46F0E7C4460120B0460120BC4601202C
:1053D0002DE9F041164E57F0E1FB336833B3DFF8A7
:1053E000588012F01DF8D8F80050DDB93468114B20
:1053F00035600122C8F800201D608CB12346D3E936
:105400000067A468C3E9025512F050F8384606B1A7
:10541000B04712F005F8002CF0D1D8F80050013D4B
:10542000C8F80050BDE8F04112F040B8BDE8F08186
:10543000BC460120C4460120B046012008B53BF01F
:105440006DF803460348D988972914BF9722422252
:105450006DF07CF9A8990B00014A042358F01ABAA0
:10546000E4220C0000B5084689B011461A460F4BDD
:105470000DF1100CCDE9003C042331F0DBFC40F2CF
:10548000E6320698012131F025FD094903901820E4
:105490003CF032FB07990091059A0290DDE9033157
:1054A0005EF0E8F9029809B000BD00BF58E40B00B7
:1054B000F0E40B0008B55EF023FA0E2008BD00BF33
:1054C00010B504465EF03AFA38B920465EF0CCFAE0
:1054D00000280CBF1E203E2010BD59F0F1FD00BF7A
:1054E00010B504465EF02AFA20B920465EF0CEFAE6
:1054F0000E2010BD59F0E4FD38B504460D465EF0AF
:105500001DFA78B920465EF01DFA68B128463AF0D7
:105510008BFFC1B220465EF017FA00280CBF1E2098
:105520003E2038BD59F0CCFD07F0B2F9F0B50C685B
:1055300087B0064620460D4617465EF0FFF9C0B913
:1055400020465EF0FFF9B0B102AB01930B4B009324
:105550000423E9183A46701E31F0C4FBDDE904303B
:10556000DDE90212009020465AF0A6FA0E2007B09C
:10557000F0BD59F0A5FD07F08BF900BFD0E40B009A
:1055800070B505465EF0DAF9F8B9044628465EF0D3
:10559000D9F9E0B1214620463CF0D8FD0824064662
:1055A00002E00134782C0ED0E1B228465EF0CCF94E
:1055B0000028F6D0610041F00101304601343CF092
:1055C00055F9782CF0D1304670BD59F079FD07F0CF
:1055D0005FF900BFF0B50C6887B0064620460D465F
:1055E00017465EF0ABF9D0B920465EF0ABF9C0B11A
:1055F00002AB01930C4B009304233A46E918701E4A
:1056000031F070FBDDE904310120CDE90010039A8F
:105610000299204672F01EFA0E2007B0F0BD59F034
:105620004FFD07F035F900BF78E40B002DE9F0419C
:105630000C688AB0074620460E4690465EF07EF91A
:1056400018BB054620465EF07DF900B3114B009370
:1056500003AB4246311D781E0193072331F042FB14
:10566000DDE90631049ACDE900152046039972F070
:10567000F1F9DDE90830059A0090039920465AF0C7
:105680001BFA0E200AB0BDE8F08159F019FD07F0B1
:10569000FFF800BF98E40B002DE9F0410C6886B0DC
:1056A000074620460E4690465EF0D8FA002839D1CB
:1056B000054620465EF0D6FA002835D01C4B0093F4
:1056C00002AB4246311D781E0193042331F00AFBE0
:1056D000029840F2D522012131F0FCFB2946074611
:1056E00040F207530398012231F000FC2946064698
:1056F00040F2F7430498012231F0F8FB4FF439737C
:10570000054609220598082131F0F0FBC0B200904F
:10571000EBB22046F2B239465EF0F4F90E2006B044
:10572000BDE8F08159F0CCFC02486CF0E7FF00BF07
:1057300038E60B00D0A40B0000B5084689B011462E
:105740001A460A4B0DF1140CCDE9003C032331F04D
:1057500071FB074918203CF0C7F9DDE906230599DC
:1057600003905EF0F7F9039809B000BDB8E50B00AF
:1057700058E60B0008B55EF043FA0E2008BD00BFE6
:1057800010B504465EF06AFA38B920465EF082FB36
:1057900000280CBF1E203E2010BD59F091FC00BF18
:1057A00010B504465EF05AFA20B920465EF088FB38
:1057B0000E2010BD59F084FC2DE9F0410D688CB02D
:1057C000074628460E4690465EF048FA002842D129
:1057D000044628465EF046FA002839D01F4B009355
:1057E00008AB4246311D781E0193042331F07AFA4A
:1057F000062205A9089836F0DBFE22469DF81C100B
:10580000402031F0A5FC0446DDE9090104AA03901B
:1058100003A8069BB3FBF4F3049350F067F8DDE9AB
:10582000031304FB01F103FB04F2CDE903121AB9DF
:105830000E200CB0BDE8F08105989DF82C30014495
:1058400028465EF013FA0028F2D105206CF032FFF2
:1058500003486CF053FF59F033FC00BF00E60B0027
:10586000D0A40B002DE9F0410D688AB00746284608
:105870000E4690465EF0F2F9002840D104462846D4
:105880005EF0F0F9002837D01E4B009304AB42467F
:10589000311D781E0193032331F024FA052207A954
:1058A000049836F085FE22469DF82410402031F001
:1058B0004FFC0446DDE9050103AA029002A8089BFB
:1058C000B3FBF4F3039350F011F8DDE9023204FB6B
:1058D00003F304FB02F2CDE902321AB90E200AB03A
:1058E000BDE8F0810799284619445EF0EFFA0028D8
:1058F000F4D105206CF0DEFE03486CF0FFFE59F099
:10590000DFFB00BF20E60B00D0A40B002DE9F04127
:105910000E6892B0074630460C4690465EF09EF9FF
:10592000002866D1054630465EF09CF900285DD01F
:10593000314B00930CAB211D4246781E0193062388
:1059400031F0D0F9052206A90C9836F031FE2A462E
:105950009DF82010402031F0FBFB0446DDE90E01EC
:1059600003AA029002A8079BB3FBF4F303934FF042
:10597000BDFF062209A90D9836F01AFE2A469DF8A9
:105980002C10402031F0E4FB0546DDE9100105AAAA
:10599000049004A80A9BB3FBF5F305934FF0A6FF10
:1059A000DDE90213049A059804FB03F305FB02F2F8
:1059B00000FB05F504FB01F1AB42CDE90332029196
:1059C000059510D11BB90E2012B0BDE8F0810998E1
:1059D000069C0244214430465EF0D2F90028F2D100
:1059E00005206CF067FE05486CF0BCFE04486CF0C6
:1059F00085FE59F065FB00BFD0E50B00409A0B0017
:105A0000D0A40B002DE9F843047B076E064604F092
:105A10001F044FF0FF33A3408C420068756888462E
:105A200027EA030728D24FF0000919E038B9B56812
:105A3000B36F4FF4007229463046984770B315F89B
:105A4000013B0138B9F1000F10D023B386F8643060
:105A50004FF00009FF230834A04543EA07270BD97C
:105A600096F86430002BE1D0FF23F4E7FF2BF2D14E
:105A7000A0454FF00109F3D8C6E900052346A3EB82
:105A80000803A4EB080404F01F043766337327FAF5
:105A900004F0BDE8F8839946FF23DCE76FF00100CE
:105AA000BDE8F8830EF072BA2DE9F04317885488E8
:105AB000B2F80480D68893B02422E41B05468946B8
:105AC00001340DEB0200002130F088FA04EBD472AF
:105AD0005210B5F94A3EADF830204FF48872A6EB6B
:105AE0000806A3EB0803ADF83220012201360D921F
:105AF000002B4FF6FF72CDF82C90ADF82840ADF892
:105B00002A60ADF844203BDDB5F9482ED21B002AAF
:105B100032DDB342B5F9460EB5F9441EA8BF33468F
:105B20009442A8BF1446B5F8402EB5F8426EA0EBDB
:105B30000800C91B4ABF521A09B200210028B6BF8B
:105B4000361A00B20020CDE900101BB224B2039334
:105B5000029495F8554ED5F83C0E0794D5F8504E62
:105B6000069495F8544E0594D5F84C4E049433B2EF
:105B700012B209A909F01CFD012013B0BDE8F083A1
:105B8000002013B0BDE8F083F0B50E2A83B06CD0CE
:105B9000154604460E460EF0B5F9002868D1B20746
:105BA0002CD0F30731D5A188E38801FB03F3B3EBD5
:105BB000660F4FEA660052D990FBF1F201FB12002A
:105BC000042D06B217B240D028463AF02DFC054607
:105BD00020460EF0D9F94FF0FF32C0F12003DA4031
:105BE0002846A223002131F081F93A460346314686
:105BF00020460EF02BFA0E2003B0F0BD214B326888
:105C00009A42CED120486CF041FD304601AA0221D3
:105C10003AF018FB019B18683AF006FC061EA388B0
:105C200028DB9E4226DA019B58683AF0FDFB021EF3
:105C3000E38803DB9A42B8BF3046C1DB1348013B1F
:105C4000002240F2A6616CF015FD3A46314620462E
:105C50000EF0BEF9400040F0010003B0F0BD0B486B
:105C6000013B00225C216CF005FD09486CF0EAFC68
:105C700059F026FA0548013B00224FF4D4616CF03C
:105C8000F9FC00BFC4790B0008A00B0068AB0B0047
:105C9000A0A70B00F0B52F4B8DB007ACCDE90034B9
:105CA000052331F01FF82C49079840F26E3231F08D
:105CB000AFF9294940F2EC52DDE9075031F0A8F97B
:105CC000DDE90860244940F2ED5231F0A1F9DDE947
:105CD000097420463BF01CFC10BB012204A920469D
:105CE00036F066FC40B3059BB3F5805F24D1049B7E
:105CF00013B30B980E2811D040F27E42164903933D
:105D000031F086F90B9A039B0093284613463146DF
:105D10003A465EF043F907980DB0F0BD0022F3E774
:105D200021460E4832F026FF0446012204A92046EF
:105D300036F03EFC0028D6D120463AF0EFFBC28870
:105D4000009207484FF40873432240F273416CF00D
:105D5000FDFC00BF44E70B0004F90B00A0E80B00BA
:105D600010AB0B0030B5174B87B003ACCDE9003456
:105D7000032330F0B7FF1449039840F2E12231F0D9
:105D800047F9124940F2EB42DDE9035031F040F9A6
:105D9000049C40F2EB42A0684FF4807131F0B6F8F9
:105DA00005980E280CD0084940F27E4231F030F9B7
:105DB0000599626828465EF02BFA039807B030BD5B
:105DC0000021F6E77CE70B0004F90B0078FC0B00E0
:105DD0002DE9F04F2DED028B5F4BA9B005ACCDE95D
:105DE0000034032330F07EFF5C49059840F2E12245
:105DF00031F00EF9DDE9053003933AF08FFBC37BF8
:105E0000002B40F08E80069D2E462F4628AB0DF1CC
:105E10002008B3EE0F8A0DF11F040DF13F09C3F105
:105E2000810A0AEB040307EE103AB8EEC77A284657
:105E3000C7EE087A17EE903AF4EE677AF1EE10FAB0
:105E400023F0030B4BF0020B6CBFDFF818B1ABF182
:105E5000FF4B594632F08EFE3AF06CFA20EE080AFB
:105E60005AF0FAFFFDEEC07AB54217EE902A594675
:105E700004F8012F30460BD032F07CFE3AF05AFA8B
:105E800020EE080A5AF0E8FFFDEEC07A17EE902ADD
:105E90004C4584F86020C4D16FF01E049FED308A19
:105EA000304D08F15F06A4EB080404EB090307EE8C
:105EB000103AB8EEC77A3846C7EE087A17EE903A2D
:105EC000F4EE677A23F00301F1EE10FA41F00201DB
:105ED00074BFA1F1FF41294632F04CFE3AF02AFA94
:105EE00020EE080A5AF0B8FFFDEEC07A17EE903A9D
:105EF00009F8013F4E45D8D107980E280FD0174911
:105F000040F27E4231F084F80799039842465EF0F1
:105F100007FA059829B0BDEC028BBDE8F08F00218F
:105F2000F3E706983AF0FAFA044606983AF0F6FAD9
:105F3000C27B0D4B04EB820422699A427FF463AF6B
:105F4000069C40F273426068032130F0DFFFD4E921
:105F5000025726695AE700BF94E70B0004F90B00CB
:105F600000007C4202004000754307002DE9F0412B
:105F70004F4B92B003ACCDE90034032330F0B2FEB6
:105F80004C49039840F2E12231F042F830220021DE
:105F900006A8039F30F022F8049E16F0030410D0E8
:105FA00030463AF0BBFAC288434840F21313CDE9B9
:105FB000003240F239214FF4897340F23A226CF0FA
:105FC000D9FB33683D4A93423FD03D4A93424ED07D
:105FD0003C4A934221D03C4A9342E1D106AD44F081
:105FE0000101042230463EF071F83AF0A3F9023480
:105FF000182CA5EC010AF2D105980E2823D02D49C2
:1060000040F27E4231F004F80599384606AA5EF067
:10601000D9F9039812B0BDE8F0812C4B610041F032
:10602000010104223046A3FB04353EF04FF83AF05C
:1060300081F904EB550501340DEB8505092C85ED3F
:10604000060AEAD1D8E70021DFE706AD44F00101F6
:10605000042230463EF03AF83AF06CF902342B460E
:10606000062C05F1140583ED000AEFD1C4E70DF10C
:10607000180845460224A11E41F0010104223046C1
:106080003EF024F83AF056F944F0010188ED000A98
:10609000042230463EF01AF83AF04CF904340E2C43
:1060A00085ED030A08F1140805F11005E3D1A3E713
:1060B000C4E70B0004F90B00D88B0B00F0E90B00D0
:1060C000A0E90B0044E90B00DCE80B00ABAAAAAA8C
:1060D0002DE9F04F2DED028B8FB04F4B04AF07F140
:1060E0000804CDE90034082330F0FCFD4B49B868C2
:1060F00040F2E12230F08CFF786ABB687B600E28AA
:106100006ED0464940F27E4230F082FF7B6A3B60AF
:1061100078693AF00FF9D7F80C804046B0EE408A23
:106120003BF05EFB002869D0C30767D5461007EE39
:10613000906AB8EE670AB5EE400AF1EE10FA58D44C
:10614000F1EEC07AFDEEE77A17EE909A19F0010FA2
:106150005FD009FB09F39E425BD1B300073323F004
:106160000703ADEB030D0DF1100A002E3BD0002408
:10617000AAF1040B25466100042241F001014046CA
:106180003DF0A4FF3AF050F90134A6424BF8040F59
:106190000544F0D138690E2818D03AF0CBF897F8BA
:1061A0002020FB69CDE901323B7E0093D7E9001046
:1061B000F0EE480A53464FEA59025EF0B7F9B86864
:1061C0002C37BD46BDEC028BBDE8F08F75B107EEF4
:1061D000905AF8EEE77AB7EE007A87EE270ADEE704
:1061E00000233B6094E738690E28D6D1B7EE000A49
:1061F000D5E760F03FFBF0EE407AA3E740463AF087
:106200008DF940F23F22C388054840F28E616CF060
:10621000B1FA04486CF0A6FADCE70B0004F90B00B5
:10622000FCAA0B00EC8B0B0000B52DED028B184B7C
:1062300089B00DF1140CCDE9003C032330F052FD80
:106240000698F8B13AF076F8B0EE408A1149059810
:1062500040F2E12230F0DCFE0798059B0E2814D0B6
:106260000C49039340F27E4230F0D2FE0799039B23
:106270001846B0EE480A5EF0A9FB059809B0BDECDF
:10628000028B00BDB6EE008AE0E70021F0E700BF18
:10629000ACE70B0004F90B002DE9F04F2DED028B5C
:1062A000624B93B008ACCDE900340A2330F01AFDFC
:1062B0005F49089840F26F3230F0AAFE5C4940F224
:1062C000DD520546099830F0A3FE5949064640F2D2
:1062D000DE520A9830F09CFE07460C980E2800F01B
:1062E00084803AF027F8B0EE408A0D980E2875D0D9
:1062F0003AF020F8F0EE408A0B994E4840F22A32EC
:106300001BF00CFB40F2EF220E9904464A481BF0AA
:1063100005FBAA88B3889342804677D1EA88F18842
:10632000914273D1A87BB27B82426FD1B8889842E8
:106330006CD1FB888B4269D1B97B914266D1E4B2C2
:10634000092C69DC0123A34013F0AA0F41D1092CC9
:1063500062D1082966D10F980E2852D03AF064F81D
:106360004FF0000A814610980E2841D03AF05CF8B0
:10637000034611980E284FF0000B40D02C4907938C
:1063800040F27E4230F044FEAA888188914240D19A
:10639000C188EA88079B91423BD1827B082A3ED183
:1063A000CDE902A35FFA88F3CDE904B00093284653
:1063B000CDF80490F0EE680AB0EE480A23463A465B
:1063C000314608F041FD0E2013B0BDEC028BBDE854
:1063D000F08F1029BFD019486CF0C4F9F7EE007A9D
:1063E00077EEC87AF0EE678A86E7B6EE008A7CE739
:1063F00011980E284FF0010B4FF00003BED1002082
:10640000CEE74FF0010A4FF00009ACE70C486CF002
:10641000A9F90C486CF0A6F90B486CF0A3F90B48ED
:106420006CF0A0F90A486CF09DF900BF10EC0B006D
:1064300004F90B0020FA0B0038EE0B00E4A40B006B
:106440007CA80B0054A30B00209D0B0068A30B003D
:1064500000A50B002DE9F0432E4B97B00FACCDE912
:106460000034072330F03EFC2B490F9840F2E12224
:1064700030F0CEFD054605220CA9109836F098F8AC
:10648000EC88264BAA8811A90AA800F0F3FB224643
:10649000234B12A90DF12A0000F0ECFBBDF9286096
:1064A000BDF92A70BDF92C80BDF92E909DF83810E9
:1064B000A9EB07030022A8EB0604402003FB04F429
:1064C00030F046FE15990D9BB3FBF0F30E29024602
:1064D0001BD0CDE908300846079139F0A5FFDDE96A
:1064E0000713099A9C4212D80E3918BF0121049053
:1064F00003912846CDE901890C990097334608F0AD
:10650000E9FF0E2017B0BDE8F0830020EAE7054858
:106510006CF0A8F810EB0B0004F90B00D0EC0B00AA
:10652000C8EC0B00C4940B0013460A46014640F227
:10653000E3201BF0E1B900BF70B52B4B86B002AC75
:10654000CDE90034042330F0CDFB2849039840F214
:10655000DC5230F05DFD2549054640F26F3202986D
:1065600030F056FD0599044640F2A72220481BF062
:10657000D5F940F2E152049906461E481BF0CEF9C7
:10658000AA88A3889A4223D1EA88E3889A421FD135
:10659000A37B102B01D0012B20D1C2B2092A1ADC17
:1065A0000123934013F0AA0F0CD1092A13D1AB7B1E
:1065B000082B16D12046F3B2294609F0DDF90E204A
:1065C00006B070BDAB7B102BF4D00B486CF0B6F866
:1065D0000A486CF0B3F80A486CF0B0F809486CF05F
:1065E000ADF809486CF0AAF8B8EA0B0004F90B0002
:1065F0008CED0B0020FA0B002C8E0B00809A0B0008
:106600005C8C0B00388E0B00248E0B0013460A4660
:10661000014640F2E3201BF06FB900BF2DE9F04FB7
:10662000394B97B00CACCDE900340A2330F05AFB5B
:1066300036490C9840F26F3230F0EAFC4FF4D463E4
:106640008288044600210E9830F050FC40F2A66388
:10665000E288002182460F9830F048FC2B4940F236
:10666000DC5283460D9830F0D3FCC6888288284BD4
:10667000054610A90AA800F0FDFA3246254B11A9DB
:106680000DF12A0000F0F6FAA27BAB7BBDF9286081
:10669000BDF92A70BDF92C80BDF92E909A422FD3F6
:1066A00014980E2822D039F0BFFE034615980E2804
:1066B0004FF0000221D0CDE9083239F0B5FEDDE916
:1066C00008320021CDE90601CDE904322046CDE9AA
:1066D0000289CDE900670FFA8BF30FFA8AF2294697
:1066E00008F066FF0E2017B0BDE8F08F15980E2851
:1066F0004FF001024FF00003DDD101210020E1E75E
:1067000005486CF02FF800BF40EA0B0004F90B00BD
:10671000D0EC0B00C8EC0B00488E0B0000B51E4BF4
:1067200089B00DF10C0CCDE9003C052330F0DAFA0C
:1067300040F26F321949039830F06AFC837BDDF830
:1067400018C001229A4094451FD2079B6FF0004168
:106750008B4201D09A421BD9BDF91010002911DBE0
:10676000828891420EDABDF91420002A0ADBB0F8C3
:1067700006E0724506DA0093634608F0E9FF0E2052
:1067800009B000BD06486BF0EDFF06486BF0EAFF6C
:1067900005486BF0E7FF00BFA0EB0B0004F90B000E
:1067A0009C8F0B00188C0B00B09A0B002DE9F04168
:1067B0001E4B88B003ACCDE90034052330F092FACB
:1067C00040F26F321A49039830F022FC827B079D19
:1067D000012393409D4225D2BDF91060BDF914708C
:1067E000BDF91880828804464FF4D46300213046F6
:1067F00030F07CFBE28840F2A6630021384630F09E
:1068000075FB40F22D520021404630F063FB2046DC
:10681000009543463A46314609F01CFA0E2008B06E
:10682000BDE8F08103486BF09DFF00BF90EA0B00CC
:1068300004F90B009C8F0B0000B5134B89B00DF1D0
:10684000080CCDE9003C062330F04CFA0F490298C1
:1068500040F26F3230F0DCFB827B079901239340DA
:1068600099420ED2BDF918C0BDF91430BDF91020FF
:10687000CDE900C1BDF90C1009F0AEFA0E2009B047
:1068800000BD03486BF06EFF70EB0B0004F90B00CA
:106890009C8F0B0030B5264B91B00BACCDE900348A
:1068A000052330F01FFA23490B9840F26F3230F085
:1068B000AFFB052205A905460C9835F079FE0522A7
:1068C00008A90D9835F074FE9DF81C100022402098
:1068D00030F03EFC9DF8281004460022402030F0A5
:1068E00037FC84421AD1069B099AB3FBF4F3B2FB3E
:1068F000F4F2934218D1A87B0E9901228240914272
:106900000FD29DF83C200292CDE900412846089A1A
:10691000059909F09BFA0E2011B030BD06486BF0C6
:1069200021FF06486BF01EFF05486BF01BFF00BF00
:1069300048EB0B0004F90B00B0A60B009C8F0B007A
:10694000C4A60B0070B51B4B8AB004ACCDE9003473
:10695000062330F0C7F940F26F321749049830F03F
:1069600057FB827B099D012393409D421FD2828861
:10697000124B0446C08805A9064602A800F07AF921
:10698000324606A90DF10A000D4B00F073F9BDF96E
:106990000E10BDF90C30BDF90A20CDE900152046D6
:1069A000BDF9081009F0E4FA0E200AB070BD0548E0
:1069B0006BF0D8FEC8EB0B0004F90B00D0EC0B0019
:1069C000C8EC0B009C8F0B0000B5114B87B00DF18C
:1069D0000C0CCDE9003C032330F084F90D490398F9
:1069E00040F2E12230F014FB827B049901239340B2
:1069F000994207D2059A9A4204D209F043FD0E202B
:106A000007B000BD044840F225316BF0B3FE00BF73
:106A1000F8EB0B0004F90B00DCAA0B002DE9F043A6
:106A20002DED028B5A4BA1B013ACCDE900340D23F0
:106A300030F058F95749139840F26F3230F0E8FAC5
:106A400040F2DC5204465349149830F0E1FAA27B3C
:106A5000837B9A42C0F09880054615980E2800F076
:106A60008F8039F0E1FC0FFA80F916980E2800F0BB
:106A7000838039F0D9FC0FFA80F819980E2878D065
:106A800039F0D2FC06B21A980E286FD039F0CCFC3F
:106A900007B2189B00930DF14203029310AB1799B4
:106AA00001930FAA0DF13E0320466EF053FE1C9B8E
:106AB00000930DF14A03029312AB019328461B99F0
:106AC0000DF1460311AA6EF045FE1D980E284AD01E
:106AD00039F030FCB0EE408A1E980E283BD039F0D9
:106AE00029FCB5EEC00AF1EE10FAF0EE400A32D4FD
:106AF0001F980E2834D0CDED0D0A39F095FCDDED50
:106B00000D0A0023CDE90A03BDF94230BDF940204A
:106B100005972046BDF94A400994BDF948400894BC
:106B2000CDE90235BDF94640BDF93E300794BDF9C7
:106B300044400496CDE90032B0EE480ABDF93C303D
:106B400006944246494609F0C9FC0E2021B0BDEC2E
:106B5000028BBDE8F0831F980E28F7EE000ACAD119
:106B600001230020CEE79FED0C8AB5E7EF887F0870
:106B70008FE7AE88760886E7E3884FEA53087CE71C
:106B8000A3884FEA530970E704486BF0EBFD00BFA0
:106B900060EC0B0004F90B0000000000488E0B00B5
:106BA00000B52E4B8DB00DF1140CCDE9003C072340
:106BB00030F098F82A49059840F2E12230F028FA9E
:106BC000DDF820C00CF1FF33012B20D9BCF1040FFC
:106BD00040D1079B022B2FDDA3F1040EBEF11C0F49
:106BE0002CD8204A012101FA0EF10A4052B39DF837
:106BF0002C109DF82820CDE901219DF82420009239
:106C00000699624609F0F4F90E200DB000BD079B0D
:106C1000022B11DD1A1F1C2A10D812494FF0010E49
:106C20000EFA02FE0EEA01010029E0D1142A05D174
:106C3000BCF1010FDBD008E0002BD8DC0A48194674
:106C40006BF098FDBEF1140FF8D108481822614688
:106C50006BF090FD064861466BF08CFDD8EA0B00A6
:106C600004F90B0011100010C0930B00B0930B003F
:106C7000A0930B00F8B50F461D461968064614464A
:106C8000386830F019FA2B680021224630F02EF9CE
:106C90003080B8680E2809D0696830F00DFA2246B5
:106CA0006B68B6F9001030F021F90446B480F8BDE5
:106CB00030B585B004461D4602A8094B0191FFF787
:106CC000D9FF0199074B0DF10A002A460431FFF75D
:106CD000D1FF02AB03CB20602046616005B030BD20
:106CE000D0EC0B00C8EC0B002DE9F0430D4685B04D
:106CF000002191464BF0AAFA0446002128464BF0A9
:106D0000A5FA2379662B68D00379662B054664D0F3
:106D1000002308208DF80F302DF05EF98046082002
:106D20002DF066F9074608202DF062F94346CDE9BB
:106D3000007006460DF10F02294620464BF006F87A
:106D400000284DD0B9F1040F56D8DFE809F01A2514
:106D5000303B03002046CDE900769DF80F20294600
:106D6000434601F0B7F8044640462DF033F9384663
:106D70002DF030F930462DF02DF9204605B0BDE854
:106D8000F0832046CDE900769DF80F202946434642
:106D900000F03CF80446E7E72046CDE900769DF890
:106DA0000F202946434600F017FA0446DCE7204648
:106DB000CDE900769DF80F202946434600F0F2FB0E
:106DC0000446D1E72046CDE900769DF80F202946FC
:106DD000434600F0CDFD0446C6E708486BF0C2FC10
:106DE00040462DF0F7F838462DF0F4F830462DF0F7
:106DF000F1F803486BF0B6FC0024B5E704910B00F2
:106E000040900B000022FFF76FBF00BF2DE9F04359
:106E1000074610463A7983B08C46622A19460A9D85
:106E20000B9EFB69DCF81C405ED019D8422A2CD09E
:106E3000482A11D19CF804E0BEF1480F00F00C8103
:106E4000BEF1680F00F02D81BEF1620F55D003D85E
:106E5000BEF1420F00F08280002003B0BDE8F08355
:106E6000682AF9D19CF80420682A00F04081622A3F
:106E700043D0F1D89946B046BE46422A23462E4614
:106E800067464C464546F446D2D19CF80420622A17
:106E900000F095806AD8422A3BD0482ADCD1019381
:106EA0004DF00EFD019BD0F81CC04FF0000E0021EC
:106EB00027881A783A402CF8022B0269D5F804800A
:106EC000776801318A4243443C44F1D8296802FB87
:106ED00018110B44316802FB1711C2680EF1010E44
:106EE00072450C44E3D8B8E7A046AE4662461C465D
:106EF0003546BC464346764617463A79622A00F044
:106F00001B81482A00F03D81682A7FD0622A8DD9F2
:106F1000A2E701934DF0D4FC019BD0F81CC04FF0C8
:106F2000000E002127781A783A400CF8012B0269EC
:106F3000D5F80480776801318A4243443C44F1D853
:106F4000296802FB18110B44316802FB1711C26853
:106F50000EF1010E72450C44E3D87EE7B6461A46A0
:106F60002E462346BC46754614468EE7682A7FF4B3
:106F700073AF01934DF0A4FC019BD0F81CE00027F7
:106F80000021B4F800C01A7802EA0C022EF8022B95
:106F90000269D5F80480D6F804C001318A4243441E
:106FA0006444EED8296802FB18110B44316802FBD7
:106FB0001C11C2680137BA420C44E1D84DE768227F
:106FC00001934DF07DFC019BD0F81CC04FF0000EEA
:106FD000002194F900701A783A402CF8022B0269CB
:106FE000D5F80480776801318A4243443C44F0D8A4
:106FF000296802FB18110B44316802FB1711C268A3
:107000000EF1010E72450C44E2D826E701934DF0D3
:1070100057FC019BD0F81CC04FF0000E00211F88C8
:1070200094F900203A402CF8022B0269D6F804802B
:107030006F6801318A4244443B44F0D8316802FB16
:1070400018110C44296802FB1711C2680EF1010ED9
:1070500072450B44E2D800E701934DF031FC019BEF
:10706000D0F81CC04FF0000E002127881A883A4043
:107070002CF8022B0269D5F80480776801318A4226
:1070800043443C44F1D8296802FB18110B44316891
:1070900002FB1711C2680EF1010E72450C44E3D8D1
:1070A000DBE6724601934DF00BFC019BD0F81CC04F
:1070B0004FF0000E002127881A883A402CF8022B46
:1070C0000269D5F80480776801318A4243443C4420
:1070D000F1D8296802FB18110B44316802FB171123
:1070E000C2680EF1010E72450C44E3D8B5E6019377
:1070F0004DF0E6FB019BD0F81CC04FF0000E0021C4
:1071000027881A883A402CF8022B0269D5F80480A7
:10711000776801318A4243443C44F1D8296802FB34
:1071200018110B44316802FB1711C2680EF1010EF1
:1071300072450C44E3D890E601934DF0C1FB019BEE
:10714000D0F81CC04FF0000E00211F7822783A4082
:107150000CF8012B0269D6F804806F6801318A426D
:1071600044443B44F1D8316802FB18110C442968AF
:1071700002FB1711C2680EF1010E72450B44E3D8F1
:107180006BE601934DF09CFB019BD0F81CC04FF0C7
:10719000000E00211F8894F900203A402CF8022BA1
:1071A0000269D6F804806F6801318A4244443B4446
:1071B000F0D8316802FB18110C44296802FB171142
:1071C000C2680EF1010E72450B44E2D845E600BFDD
:1071D0000122FFF789BD00BF2DE9F04307461046A5
:1071E0003A7983B08C46622A19460A9D0B9EFB6948
:1071F000DCF81C405ED019D8422A2CD0482A11D184
:107200009CF804E0BEF1480F00F00C81BEF1680F5D
:1072100000F02D81BEF1620F55D003D8BEF1420FB0
:1072200000F08280002003B0BDE8F083682AF9D125
:107230009CF80420682A00F04081622A43D0F1D8EB
:107240009946B046BE46422A23462E4667464C46DD
:107250004546F446D2D19CF80420622A00F095807D
:107260006AD8422A3BD0482ADCD101934DF028FB52
:10727000019BD0F81CC04FF0000E002127881A781F
:107280003A432CF8022B0269D5F804807768013163
:107290008A4243443C44F1D8296802FB18110B444C
:1072A000316802FB1711C2680EF1010E72450C44E1
:1072B000E3D8B8E7A046AE4662461C463546BC4613
:1072C0004346764617463A79622A00F01B81482ADF
:1072D00000F03D81682A7FD0622A8DD9A2E7019310
:1072E0004DF0EEFA019BD0F81CC04FF0000E0021CB
:1072F00027781A783A430CF8012B0269D5F80480F4
:10730000776801318A4243443C44F1D8296802FB42
:1073100018110B44316802FB1711C2680EF1010EFF
:1073200072450C44E3D87EE7B6461A462E462346FD
:10733000BC46754614468EE7682A7FF473AF019306
:107340004DF0BEFA019BD0F81CE000270021B4F8F4
:1073500000C01A7842EA0C022EF8022B0269D5F816
:107360000480D6F804C001318A4243446444EED814
:10737000296802FB18110B44316802FB1C11C2681A
:107380000137BA420C44E1D84DE7682201934DF031
:1073900097FA019BD0F81CC04FF0000E002194F921
:1073A00000701A783A432CF8022B0269D5F8048051
:1073B000776801318A4243443C44F0D8296802FB93
:1073C00018110B44316802FB1711C2680EF1010E4F
:1073D00072450C44E2D826E701934DF071FA019B07
:1073E000D0F81CC04FF0000E00211F8894F9002037
:1073F0003A432CF8022B0269D6F804806F680131F9
:107400008A4244443B44F0D8316802FB18110C44D2
:10741000296802FB1711C2680EF1010E72450B4478
:10742000E2D800E701934DF04BFA019BD0F81CC065
:107430004FF0000E002127881A883A432CF8022BBF
:107440000269D5F80480776801318A4243443C449C
:10745000F1D8296802FB18110B44316802FB17119F
:10746000C2680EF1010E72450C44E3D8DBE67246A9
:1074700001934DF025FA019BD0F81CC04FF0000E8F
:10748000002127881A883A432CF8022B0269D5F884
:107490000480776801318A4243443C44F1D829682A
:1074A00002FB18110B44316802FB1711C2680EF180
:1074B000010E72450C44E3D8B5E601934DF000FA95
:1074C000019BD0F81CC04FF0000E002127881A88BD
:1074D0003A432CF8022B0269D5F804807768013111
:1074E0008A4243443C44F1D8296802FB18110B44FA
:1074F000316802FB1711C2680EF1010E72450C448F
:10750000E3D890E601934DF0DBF9019BD0F81CC065
:107510004FF0000E00211F7822783A430CF8012B1F
:107520000269D6F804806F6801318A4244443B44C2
:10753000F1D8316802FB18110C44296802FB1711BD
:10754000C2680EF1010E72450B44E3D86BE601935D
:107550004DF0B6F9019BD0F81CC04FF0000E002191
:107560001F8894F900203A432CF8022B0269D6F8C0
:1075700004806F6801318A4244443B44F0D831684A
:1075800002FB18110C44296802FB1711C2680EF1A6
:10759000010E72450B44E2D845E600BF0222FFF718
:1075A000A3BB00BF2DE9F043074610463A7983B0EC
:1075B0008C46622A19460A9D0B9EFB69DCF81C402A
:1075C0005ED019D8422A2CD0482A11D19CF804E068
:1075D000BEF1480F00F00C81BEF1680F00F02D8164
:1075E000BEF1620F55D003D8BEF1420F00F0828089
:1075F000002003B0BDE8F083682AF9D19CF804208C
:10760000682A00F04081622A43D0F1D89946B046FA
:10761000BE46422A23462E4667464C464546F44619
:10762000D2D19CF80420622A00F095806AD8422AC0
:107630003BD0482ADCD101934DF042F9019BD0F8B0
:107640001CC04FF0000E002127881A787A402CF8D1
:10765000022B0269D5F80480776801318A424344DD
:107660003C44F1D8296802FB18110B44316802FB35
:107670001711C2680EF1010E72450C44E3D8B8E749
:10768000A046AE4662461C463546BC464346764654
:1076900017463A79622A00F01B81482A00F03D81A2
:1076A000682A7FD0622A8DD9A2E701934DF008F9AC
:1076B000019BD0F81CC04FF0000E002127781A78EB
:1076C0007A400CF8012B0269D5F804807768013103
:1076D0008A4243443C44F1D8296802FB18110B4408
:1076E000316802FB1711C2680EF1010E72450C449D
:1076F000E3D87EE7B6461A462E462346BC46754674
:1077000014468EE7682A7FF473AF01934DF0D8F8E2
:10771000019BD0F81CE000270021B4F800C01A78C3
:1077200082EA0C022EF8022B0269D5F80480D6F802
:1077300004C001318A4243446444EED8296802FB04
:1077400018110B44316802FB1C11C2680137BA42A0
:107750000C44E1D84DE7682201934DF0B1F8019B4C
:10776000D0F81CC04FF0000E002194F900701A7878
:107770007A402CF8022B0269D5F804807768013131
:107780008A4243443C44F0D8296802FB18110B4458
:10779000316802FB1711C2680EF1010E72450C44EC
:1077A000E2D826E701934DF08BF8019BD0F81CC07E
:1077B0004FF0000E00211F8894F900207A402CF829
:1077C000022B0269D6F804806F6801318A42444472
:1077D0003B44F0D8316802FB18110C44296802FBC5
:1077E0001711C2680EF1010E72450B44E2D800E792
:1077F00001934DF065F8019BD0F81CC04FF0000ECE
:10780000002127881A887A402CF8022B0269D5F8C3
:107810000480776801318A4243443C44F1D82968A6
:1078200002FB18110B44316802FB1711C2680EF1FC
:10783000010E72450C44E3D8DBE6724601934DF02D
:107840003FF8019BD0F81CC04FF0000E00212788A4
:107850001A887A402CF8022B0269D5F804807768E0
:1078600001318A4243443C44F1D8296802FB181193
:107870000B44316802FB1711C2680EF1010E72450C
:107880000C44E3D8B5E601934DF01AF8019BD0F80B
:107890001CC04FF0000E002127881A887A402CF86F
:1078A000022B0269D5F80480776801318A4243448B
:1078B0003C44F1D8296802FB18110B44316802FBE3
:1078C0001711C2680EF1010E72450C44E3D890E620
:1078D00001934CF0F5FF019BD0F81CC04FF0000E57
:1078E00000211F7822787A400CF8012B0269D6F823
:1078F00004806F6801318A4244443B44F1D83168C6
:1079000002FB18110C44296802FB1711C2680EF122
:10791000010E72450B44E3D86BE601934CF0D0FFA7
:10792000019BD0F81CC04FF0000E00211F8894F975
:1079300000207A402CF8022B0269D6F804806F6888
:1079400001318A4244443B44F0D8316802FB1811AB
:107950000C44296802FB1711C2680EF1010E724532
:107960000B44E2D845E600BF0322FFF7BDB900BFD4
:107970002DE9F04117460279CC6982B0622A9C4613
:10798000089DC369099E6ED038D8422A00F0A380B2
:10799000482A40F09C8009790193422900F03E81F9
:1079A000622900F04482482900F08381614638460C
:1079B00068224CF085FF019BD0F81CC04FF0000EF0
:1079C0000021B4F900701A88BA402CF8022B026921
:1079D000D5F80480776801318A4243443C44F0D8AA
:1079E000296802FB18110B44316802FB1711C268A9
:1079F0000EF1010E72450C44E2D869E0682A66D1A6
:107A000009790193422900F09880622900F0C18130
:107A100048293846614600F027814CF051FF019B10
:107A2000D0F81CE000270021B4F900C0B3F9002011
:107A300002FA0CF22EF8022B0269D5F80480D6F86F
:107A400004C001318A4243446444EDD8296802FBF2
:107A500018110B44316802FB1C11C2680137BA428D
:107A60000C44E0D834E00A790193422A6146384652
:107A700000F08A80622A00F0B481482A00F0408138
:107A800068224CF01DFF019BD0F81CC04FF0000E87
:107A90000021B4F9007093F90020BA402CF8022BB1
:107AA0000269D5F80480776801318A4243443C4436
:107AB000EFD8296802FB18110B44316802FB17113B
:107AC000C2680EF1010E72450C44E1D800E00020BE
:107AD00002B0BDE8F0810A790193422A6146384636
:107AE00078D0622A00F0CC81482A00F02E816822EA
:107AF0004CF0E6FE019BD0F81CC04FF0000E0021B8
:107B0000B4F900701A78BA402CF8022B0269D5F843
:107B10000480776801318A4243443C44F0D82968A4
:107B200002FB18110B44316802FB1711C2680EF1F9
:107B3000010E72450C44E2D8CAE7614638464CF063
:107B4000BFFE019BD0F81CC04FF0000E002127782B
:107B5000B3F90020BA402CF8022B0269D5F8048052
:107B6000776801318A4243443C44F0D8296802FBDB
:107B700018110B44316802FB1711C2680EF1010E97
:107B800072450C44E2D8A3E768224CF099FE019BB1
:107B9000D0F81CC04FF0000E0021277893F9002088
:107BA000BA402CF8022B0269D5F8048077680131BD
:107BB0008A4243443C44F0D8296802FB18110B4424
:107BC000316802FB1711C2680EF1010E72450C44B8
:107BD000E2D87DE74CF074FE019BD0F81CC04FF05A
:107BE000000E002127781A78BA400CF8012B0269A0
:107BF000D5F80480776801318A4243443C44F1D887
:107C0000296802FB18110B44316802FB1711C26886
:107C10000EF1010E72450C44E3D859E7614638462F
:107C20004CF04EFE019BD0F81CC04FF0000E00211E
:107C300027781A88BA402CF8022B0269D5F80480FC
:107C4000776801318A4243443C44F1D8296802FBF9
:107C500018110B44316802FB1711C2680EF1010EB6
:107C600072450C44E3D833E74CF02AFE019BD0F870
:107C70001CC04FF0000E0021B4F900701A88BA4001
:107C80002CF8022B0269D5F80480776801318A420A
:107C900043443C44F0D8296802FB18110B44316876
:107CA00002FB1711C2680EF1010E72450C44E2D8B6
:107CB0000EE70A46384661464CF002FE019BD0F8BA
:107CC0001CC04FF0000E002127881A88BA402CF8FB
:107CD000022B0269D5F80480776801318A42434457
:107CE0003C44F1D8296802FB18110B44316802FBAF
:107CF0001711C2680EF1010E72450C44E3D8E7E695
:107D00004CF0DEFD019BD0F81CC04FF0000E0021AE
:107D1000278893F90020BA402CF8022B0269D5F885
:107D20000480776801318A4243443C44F0D8296892
:107D300002FB18110B44316802FB1711C2680EF1E7
:107D4000010E72450C44E2D8C2E64CF0B9FD019B2D
:107D5000D0F81CC04FF0000E002127881A78BA40D6
:107D60002CF8022B0269D5F80480776801318A4229
:107D700043443C44F1D8296802FB18110B44316894
:107D800002FB1711C2680EF1010E72450C44E3D8D4
:107D90009EE6614638464CF093FD019BD0F81CC02E
:107DA0004FF0000E002194F90070B3F90020BA40A2
:107DB0002CF8022B0269D5F80480776801318A42D9
:107DC00043443C44EFD8296802FB18110B44316846
:107DD00002FB1711C2680EF1010E72450C44E1D886
:107DE00076E64CF06DFD019BD0F81CC04FF0000E04
:107DF000002194F9007093F90020BA400CF8012B8F
:107E00000269D5F80480776801318A4243443C44D2
:107E1000EFD8296802FB18110B44316802FB1711D7
:107E2000C2680EF1010E72450C44E1D850E60A46D4
:107E3000384661464CF044FD019BD0F81CC04FF021
:107E4000000E002194F9007093F90020BA400CF85C
:107E5000012B0269D5F80480776801318A424344D6
:107E60003C44EFD8296802FB18110B44316802FB2F
:107E70001711C2680EF1010E72450C44E1D827E6D5
:107E800068224CF01DFD019BD0F81CC04FF0000E85
:107E9000002194F900701A78BA402CF8022B02697C
:107EA000D5F80480776801318A4243443C44F0D8D5
:107EB000296802FB18110B44316802FB1711C268D4
:107EC0000EF1010E72450C44E2D801E60422FEF7E1
:107ED0000BBF00BF2DE9F04117460279CC6982B093
:107EE000622A9C46089DC369099E6ED038D8422AF2
:107EF00000F0A380482A40F09C8009790193422930
:107F000000F03E81622900F04482482900F083811C
:107F10006146384668224CF0D3FC019BD0F81CC067
:107F20004FF0000E0021B4F900701A883A412CF885
:107F3000022B0269D5F80480776801318A424344F4
:107F40003C44F0D8296802FB18110B44316802FB4D
:107F50001711C2680EF1010E72450C44E2D869E0B7
:107F6000682A66D109790193422900F09880622934
:107F700000F0C18148293846614600F027814CF065
:107F80009FFC019BD0F81CE000270021B4F900C041
:107F9000B3F9002042FA0CF22EF8022B0269D5F850
:107FA0000480D6F804C001318A4243446444EDD8C9
:107FB000296802FB18110B44316802FB1C11C268CE
:107FC0000137BA420C44E0D834E00A790193422ADE
:107FD0006146384600F08A80622A00F0B481482A5F
:107FE00000F0408168224CF06BFC019BD0F81CC073
:107FF0004FF0000E0021B4F9007093F900203A41CF
:108000002CF8022B0269D5F80480776801318A4286
:1080100043443C44EFD8296802FB18110B443168F3
:1080200002FB1711C2680EF1010E72450C44E1D833
:1080300000E0002002B0BDE8F0810A790193422AF5
:108040006146384678D0622A00F0CC81482A00F098
:108050002E8168224CF034FC019BD0F81CC04FF0FC
:10806000000E0021B4F900701A783A412CF8022B66
:108070000269D5F80480776801318A4243443C4460
:10808000F0D8296802FB18110B44316802FB171164
:10809000C2680EF1010E72450C44E2D8CAE761468F
:1080A00038464CF00DFC019BD0F81CC04FF0000E80
:1080B00000212778B3F900203A412CF8022B0269FD
:1080C000D5F80480776801318A4243443C44F0D8B3
:1080D000296802FB18110B44316802FB1711C268B2
:1080E0000EF1010E72450C44E2D8A3E768224CF071
:1080F000E7FB019BD0F81CC04FF0000E0021277851
:1081000093F900203A412CF8022B0269D5F804803B
:10811000776801318A4243443C44F0D8296802FB25
:1081200018110B44316802FB1711C2680EF1010EE1
:1081300072450C44E2D87DE74CF0C2FB019BD0F8BD
:108140001CC04FF0000E002127781A783A410CF835
:10815000012B0269D5F80480776801318A424344D3
:108160003C44F1D8296802FB18110B44316802FB2A
:108170001711C2680EF1010E72450C44E3D859E79D
:10818000614638464CF09CFB019BD0F81CC04FF078
:10819000000E002127781A883A412CF8022B026938
:1081A000D5F80480776801318A4243443C44F1D8D1
:1081B000296802FB18110B44316802FB1711C268D1
:1081C0000EF1010E72450C44E3D833E74CF078FB16
:1081D000019BD0F81CC04FF0000E0021B4F90070D4
:1081E0001A883A412CF8022B0269D5F80480776886
:1081F00001318A4243443C44F0D8296802FB1811FB
:108200000B44316802FB1711C2680EF1010E724572
:108210000C44E2D80EE70A46384661464CF050FB63
:10822000019BD0F81CC04FF0000E002127881A884F
:108230003A412CF8022B0269D5F8048077680131A5
:108240008A4243443C44F1D8296802FB18110B448C
:10825000316802FB1711C2680EF1010E72450C4421
:10826000E3D8E7E64CF02CFB019BD0F81CC04FF0A4
:10827000000E0021278893F900203A412CF8022BA8
:108280000269D5F80480776801318A4243443C444E
:10829000F0D8296802FB18110B44316802FB171152
:1082A000C2680EF1010E72450C44E2D8C2E64CF0F1
:1082B00007FB019BD0F81CC04FF0000E002127885F
:1082C0001A783A412CF8022B0269D5F804807768B5
:1082D00001318A4243443C44F1D8296802FB181119
:1082E0000B44316802FB1711C2680EF1010E724592
:1082F0000C44E3D89EE6614638464CF0E1FA019B17
:10830000D0F81CC04FF0000E002194F90070B3F9B2
:1083100000203A412CF8022B0269D5F804807768D6
:1083200001318A4243443C44EFD8296802FB1811CA
:108330000B44316802FB1711C2680EF1010E724541
:108340000C44E1D876E64CF0BBFA019BD0F81CC097
:108350004FF0000E002194F9007093F900203A418B
:108360000CF8012B0269D5F80480776801318A4244
:1083700043443C44EFD8296802FB18110B44316890
:1083800002FB1711C2680EF1010E72450C44E1D8D0
:1083900050E60A46384661464CF092FA019BD0F806
:1083A0001CC04FF0000E002194F9007093F90020DA
:1083B0003A410CF8012B0269D5F804807768013145
:1083C0008A4243443C44EFD8296802FB18110B440D
:1083D000316802FB1711C2680EF1010E72450C44A0
:1083E000E1D827E668224CF06BFA019BD0F81CC05C
:1083F0004FF0000E002194F900701A783A412CF8E1
:10840000022B0269D5F80480776801318A4243441F
:108410003C44F0D8296802FB18110B44316802FB78
:108420001711C2680EF1010E72450C44E2D801E644
:1084300030B5184CD4F8B43083B013B909E01B68D8
:108440003BB19A688242FAD15A688A42F7D103B0A6
:1084500030BDCDE900010C202BF0BEFDD4F8B4C036
:10846000DDE90021BCF1000F0CD0634601E01B6880
:1084700043B19D68AA42FAD15D68A942E7D01B6862
:10848000002BF6D1C0E900C18260C4F8B40003B08B
:1084900030BD00BFA470012010B5DFF830E0DEF879
:1084A000B4C0BCF1000F0AD0634601E01B6833B1D1
:1084B0009C688C42FAD15C689442F7D110BDC0E947
:1084C00000C28160CEF8B40010BD00BFA4700120CE
:1084D00010B5054BD3F8B4402CB1204624F002FF70
:1084E0002468002CF9D110BDA47001200B4AD2F8E9
:1084F000B4308BB102F1B40C02E09C461B685BB156
:108500009A688242F9D15A688A42F6D11968CCF841
:10851000001000221A607047704700BFA47001204D
:108520002DE9F843144CD4F8B4701FB34FF0000990
:108530003846B8463F6825F0F1F920B9D8F804006C
:1085400025F0ECF9A0B1D4F8B4308BB1D8E9012111
:1085500004F1B40002E018461B684BB19E68B142BA
:10856000F9D15E68B242F6D11A680260C3F8009091
:10857000002FDDD1BDE8F883A47001200349044A2F
:108580000023C1F8B4301370704700BFA4700120FD
:10859000887B012008B5074B1B780BB9002008BD6C
:1085A000054808F063FF0028F8D1BDE808400248FC
:1085B00008F0BCBF637B0120F8440120014809F0AA
:1085C00033BC00BF5045012000B50B4883B008F014
:1085D0004DFF68B9094A127852B1034601220DF1E4
:1085E0000701054808F048FF9DF8070003B000BDEB
:1085F000FF2003B000BD00BFF8440120637B0120D1
:108600002DE9F041074682B013480E4609F076FC8A
:10861000F0B9124B1B78DBB1D6B1044680460CE0B2
:10862000AAB239190C48CDF80080002309F08CFD5E
:10863000002804440CDBA6420AD9074809F0A6FC2E
:10864000351B8542ECD3044809F0A0FC82B2E8E770
:1086500002B0BDE8F08100BF50450120637B0120DE
:1086600008B509F0DFFB0348012108F0D3FA0E201A
:1086700008BD00BF700D012030B585B002AB51F8C8
:10868000044B01930C4B0093013802232EF02AFB7C
:1086900040F29E22094902982EF0BAFC40F22A616B
:1086A00005469FED070A03982EF064FC29462046F4
:1086B00008F04AF905B030BDDCCB0B004CCD0B0007
:1086C0000000000008B508F0EDF90E2008BD00BF5D
:1086D00008B5152124F040FEBDE808400148AA2154
:1086E00024F03ABEA00A012008F0DEB908B508F06F
:1086F000F7F900280CBF1E203E2008BD08B508F081
:10870000F5F900280CBF1E203E2008BD08F002BA73
:1087100008B508F02BFA00280CBF1E203E2008BD2B
:1087200030B585B000240546ADF8061020460DF1A1
:108730000E01ADF80E4059F01DF90DF10601284665
:1087400059F018F918B9BDF80E0005B030BD204633
:1087500005B030BD08B5014869F098FFA8A70B0027
:108760002DE9F041036905465BB159F017F9286915
:1087700001215CF03BFA27482969FFF7B7FE002387
:108780002B61EB688BB1244B1878FF280DD059F082
:10879000DFF8294604462148FFF7A8FE0023EB60D6
:1087A00085F8443034F0080330D11D4C0023AB6110
:1087B00004F52A7825464FF6FF770E262B88BB4214
:1087C000284601D009F09AF8EE6588354545F5D17F
:1087D00062F05EFC4FF6FF7506460F4600231A4610
:1087E00034F813104433A94218BF42F00102B3F524
:1087F000AA7FF5D142B162F04BFC801B61EB07010F
:10880000802871F10001E9D3BDE8F081204604F031
:1088100045F8CAE76D150900A70601206D0A030097
:10882000A00A012010B58EB0044620221D4806A9DA
:108830005AF0B6FC80B31C4B0FCB0DF1080CACE822
:1088400007002046ACF8003008F02EF9F0B1694678
:1088500008F00EFD9DF8010014499DF800204FEA34
:10886000101C00F00F0011F80CC0085C00236CF322
:10887000070360F30F23100902F00F02085C8A5C03
:1088800060F3174362F31F63CDF8113002A920464D
:1088900008F004FB0EB010BD06A9204608F0FEFA51
:1088A0000EB010BD542F0B00682F0B00C07C0B00C6
:1088B00008B508F095F908B10E2008BD01483DF053
:1088C0002BFB00BFA8A60B0010B50446084638F0E5
:1088D00047FF0146204608F09DF90E2010BD00BF5D
:1088E00010B5044608463BF0F5F90146204608F06D
:1088F000D5FA0E2010BD00BF70B52DED028B51F8DA
:10890000043B94B01D460CAB0193394B00930138E6
:1089100008232EF0E7F90C98052206A933F048FE4B
:108920000D9800230E28CDE909330B9303D00522BF
:1089300009A933F03DFE1198002847D040F23C4190
:108940002EF080FBDFED2B7AB4EEE70AF1EE10FAA1
:10895000B0EE408A43D4DFED287AB4EEE70AF1EEB8
:1089600010FA3CDC40F22A6210989DF838409DF8DD
:108970003C6000212EF0AEFA079A1F2A03461DD84C
:1089800013980E2820D03CB31C49059340F27E3248
:108990002EF03EFB059B039009AA0192214606AAF0
:1089A000129C00922846B0EE480A3246029408F023
:1089B00089FA0E2014B0BDEC028B70BD4CB10A9A3E
:1089C00092B913980E28DFD10020E4E70C481190EB
:1089D000B4E7139A0E2AF7D00A483DF09DFA0A4AE6
:1089E0000A490B4869F0C6FE0A483DF095FA00BFF7
:1089F0005CCB0B000AD7A33C0AD723414CCD0B001C
:108A0000CECC4CBE98A10B00442F0B004C2F0B007A
:108A1000D8930B0074A70B0010B52DED048B51F803
:108A2000043B90B01C4608AB0193444B00930138C3
:108A300008232EF057F90B980E2866D09FED400AB8
:108A400040F22A612EF096FA0C98F0EE408A002847
:108A500060D00D9B002B62D040F23C412EF0F2FA28
:108A6000DFED387AB4EEE70AF1EE10FAB0EE408AA4
:108A700058D4DFED357AB4EEE70AF1EE10FA51DCA6
:108A8000F5EE408AF1EE10FA04D0F4EEC08AF1EE71
:108A900010FA4FD40D9840F291612EF0D3FAB4EE53
:108AA000C08AF1EE10FAB0EE409A40D40898002344
:108AB000069328B1052205A933F07AFD069BE3B998
:108AC000099840F2FE2201212EF004FA9DF83C1094
:108AD0000E9A0090CDE901219DF82830DDE90512BC
:108AE000B0EE491AF0EE480AB0EE680A204608F0E7
:108AF00099FA10B0BDEC048B10BD059824F00EFF60
:108B00000028DDD1114869F02DFE0C98DFED0C8AAC
